:100000000C94BB060C94FF060C94FF060C94FF06A0
:100010000C94FF060C94FF060C94FF060C94FF064C
:100020000C94FF060C943F190C94FF060C94FF06E9
:100030000C9488330C94FF060C94FF060C94FF0676
:100040000C94FF060C94FF060C940F160C94FF06FC
:100050000C942A0C0C94FF060C94F40B0C94FF06E1
:100060000C94FB1B0C94FF060C941B2F0C94FF06A6
:100070000C9408770C94FF060C940472261C2B1C1D
:10008000301C391C501C671C771C871CA41C901E3C
:10009000671C521D631D921DB01DCD1D271E821EA3
:1000A0006020F220AF212F22982248234F25AC2533
:1000B00019266326AE26FB264C27AE270D28A72837
:1000C00042293C2A3A2F6E2FB12F213039307A3015
:1000D0003131F831F831F831F831F831F831F8319F
:1000E000F831F831F831F831AD31AF31B431CC31CC
:1000F000CE310A0D426174743A00202564204365B4
:100100006C6C732000204C6F77207761726E696E83
:1001100067206C6576656C3A2025642E2564000A9C
:100120000D466F756E6420424C2D4374726C3A20FC
:10013000002564000A0D0A0D2121204D4953534921
:100140004E4720424C2D4354524C3A2025642021E6
:1001500021000A0D3D3D3D3D3D3D3D3D3D3D3D3D8B
:100160003D3D3D3D3D3D3D3D3D3D3D3D3D3D3D3DBF
:100170003D3D3D3D3D3D3D000A0D43616C69627270
:100180006174696E67207072657373757265207330
:10019000656E736F722E2E004F4B0A0D000A0D46CE
:1001A0006C696768742D74696D65202575206D69AB
:1001B0006E2020546F74616C3A2575206D696E0055
:1001C0000A0D436F6E74726F6C3A2000486561646B
:1001D000696E67486F6C64004E6F726D616C2028A9
:1001E0004143432D4D6F646529000A0D3D3D3D3D62
:1001F0003D3D3D3D3D3D3D3D3D3D3D3D3D3D3D3D2F
:100200003D3D3D3D3D3D3D3D3D3D3D3D3D3D3D0A51
:100210000D00416E676C654E69636B2020202020C5
:100220002020416E676C65526F6C6C20202020206E
:1002300020204163634E69636B2020202020202012
:100240002020416363526F6C6C20202020202020EE
:1002500020205961774779726F20202020202020AC
:1002600020204865696768742056616C7565202098
:1002700020204163635A202020202020202020209D
:1002800020204761732020202020202020202020B3
:100290002020436F6D706173732056616C7565200B
:1002A0002020566F6C74616765205B302E31565D7F
:1002B00020205265636569766572204C6576656CB1
:1002C00020204779726F20436F6D70617373202017
:1002D00020204D6F746F722031202020202020209C
:1002E00020204D6F746F722032202020202020208B
:1002F00020204D6F746F722033202020202020207A
:1003000020204D6F746F7220342020202020202068
:1003100020203136202020202020202020202020B6
:1003200020203137202020202020202020202020A5
:100330002020313820202020202020202020202094
:100340002020313920202020202020202020202083
:100350002020536572766F2020202020202020202E
:100360002020486F7665726761732020202020204E
:10037000202043757272656E74205B302E31415DB2
:1003800020204361706163697479205B6D41685D11
:100390002020323420202020202020202020202037
:1003A0002020323520202020202020202020202026
:1003B0002020323620202020202020202020202015
:1003C0002020323720202020202020202020202004
:1003D00020204932432D4572726F72202020202048
:1003E0002020424C204C696D697420202020202060
:1003F00020204750535F4E69636B2020202020202F
:1004000020204750535F526F6C6C2020202020200A
:10041000202021212120494E434F4D504154494233
:100420004C4520212121002E000A0D20444143206B
:100430006F7220493243204552524F522120436867
:1004400065636B204932432C2033567265662C203D
:1004500044414320616E6420424C2D4374726C0011
:100460005B25695D005B25695D002B204D696B7222
:100470006F4B6F70746572202B0048573A56256495
:100480002E25642053573A25642E25642563005396
:10049000657474696E673A2564202573004861723B
:1004A0006477617265204572726F7220313A2564FB
:1004B000202121004D697373696E6720424C2D43E2
:1004C00074726C3A25642121004D6978657220456B
:1004D00072726F722100493243204552524F5221AD
:1004E0002121004865696768743A20202535690034
:1004F000536574706F696E743A2535690050726582
:1005000073737572653A253569004F666673657455
:100510003A20202535690048656967687420636F53
:100520006E74726F6C0044495341424C454400481C
:10053000656967687420636F6E74726F6C004449FC
:100540005341424C4544006163742E2062656172E0
:10055000696E67004E69636B3A20202020202025B9
:10056000356900526F6C6C3A202020202020253500
:100570006900436F6D706173733A202020253569DF
:10058000004B313A25346920204B323A253469201A
:10059000004B333A25346920204B343A2534692006
:1005A000004B353A25346920204B363A25346920F2
:1005B000004B373A25346920204B383A25346920DE
:1005C000004E693A2534692020526F3A253469205B
:1005D0000047733A253469202047693A2534692059
:1005E0000050313A253469202050323A25346920B0
:1005F0000050333A253469202050343A253469209C
:10060000004779726F202D2053656E736F72004E14
:1006100069636B25346920282533692E25692900F3
:10062000526F6C6C25346920282533692E25692981
:100630000047696572253469202825336929004EF1
:1006400069636B2025346920282533692E25782994
:1006500000526F6C6C2025346920282533692E25C3
:1006600078290059617720202534692028253369AD
:1006700029004E69636B20253469202825336929B8
:10068000282533692900526F6C6C20253469202895
:1006900025336929282533692900596177202025C8
:1006A00034692028253369292825336929004143E5
:1006B00043202D2053656E736F72004E69636B206B
:1006C00025346920282533692900526F6C6C202558
:1006D0003469202825336929005A20202020253418
:1006E0006920282533692900566F6C746167653A63
:1006F0002020202533692E253169560043757272FA
:10070000656E743A2020202533692E253169410019
:10071000506F7765723A20202020202534695700D9
:100720004469736368617267653A202535696D4174
:10073000680052656365697665720052432D5253B5
:1007400053493A202020202534690052432D517509
:10075000616C6974793A202534690052432D4368ED
:10076000616E6E656C733A25346900436F6D70611C
:1007700073730048656164696E673A2020253569A6
:100780000056616C75653A2020202025356900539C
:10079000746172743A2020202025356900506F74EE
:1007A00069313A202025336900506F7469323A204C
:1007B0002025336900506F7469333A20202533694E
:1007C00000506F7469343A202025336900506F74EB
:1007D00069353A202025336900506F7469363A2014
:1007E0002025336900506F7469373A20202533691A
:1007F00000506F7469383A202025336900536572C0
:10080000766F202000536574706F696E7420202508
:10081000336900506F736974696F6E3A20253369CC
:100820000052616E67653A2533692D2533690045AD
:10083000787465726E436F6E74726F6C2020004E18
:10084000693A2534692020526F3A253469200047DF
:10085000733A253469202047693A253469200048D5
:10086000693A253469202043663A253469200042DC
:100870004C2D4374726C204572726F727320002588
:10088000336420253364202533642025336420001D
:1008900025336420253364202533642025336420E8
:1008A00000253364202533642025336420253364F8
:1008B0002000424C2054656D7065726174757265DC
:1008C00000253369202533692025336920253369C4
:1008D00020002533692025336920253369202533FD
:1008E00069200025336920253369202533692025B7
:1008F00033692000424C2D4374726C20666F756E14
:1009000064200020256320202025632020202563EB
:10091000202020256320002025632020202563201F
:10092000202025632020202563200020256320200F
:10093000202D2020202D2020202D2000313000319E
:100940003100313200466C696768742D54696D65F9
:10095000202000546F74616C3A2535756D696E0006
:100960004163743A20202535756D696E00287265E3
:1009700073657429000A0D47656E65726174696E4E
:10098000672064656661756C7420506172616D6585
:1009900074657220536574202564000A0D557369CF
:1009A0006E6720506172616D657465722053657465
:1009B000202564000A0D47656E65726174696E6773
:1009C0002064656661756C74204D69786572205489
:1009D00061626C65000A0D4D697865722D436F6E1A
:1009E0006669673A202725732720282575204D6FD3
:1009F000746F727329000A0D3D3D3D3D3D3D3D3D07
:100A00003D3D3D3D3D3D3D3D3D3D3D3D3D3D3D3D16
:100A10003D3D3D3D3D3D000A0D414343206E6F7419
:100A20002063616C69627261746564210D0A000063
:100A3000008F001E01AD013B02CA025803E6037499
:100A40000402058F051B06A7063307BE074808D218
:100A5000085B09E3096B0AF20A780BFD0B810C04B1
:100A60000D860D070E870E060F840F00107B10F504
:100A7000106E11E5115B12CF124213B313231492BF
:100A800014FE146A15D3153B16A11605176717C86F
:100A90001727188318DE1837198E19E319361A87A5
:100AA0001AD61A231B6E1BB61BFD1B411C831CC3CD
:100AB0001C001D3C1D751DAB1DE01D121E421E6F4E
:100AC0001E9A1EC31EE91E0D1F2E1F4D1F691F8477
:100AD0001F9B1FB01FC31FD31FE11FEC1FF51FFB80
:100AE0001FFF1F0020030100005A6B000201014D8F
:100AF0006C01030202E16C020003033E6D253269C2
:100B00002E25316956002533642563202530336452
:100B10006D00537461747573004552524F523A2000
:100B200025326400253469202532693A253032693E
:100B3000002534696D25630025336920253369203C
:100B40002533692025336900253369202533692041
:100B5000253369202533690054656D7065726174B1
:100B600075726573202020200025634320202020FB
:100B700020002532692E2531695620202533692E23
:100B8000253169410025346957202536696D416852
:100B9000002532756D2F73205361743A256420004F
:100BA00020203344004E6F4678004447505300489D
:100BB0006F6D653A2533646D202533642563004EDF
:100BC0006F204E6176694374726C21000A0D77774D
:100BD000772E4D696B726F4B6F707465722E646502
:100BE0002028632920486953797374656D73204701
:100BF0006D6248000A0D74686520757365206F6624
:100C0000207468697320736F6674776172652069F8
:100C100073206F6E6C79207065726D697474656491
:100C2000200A0D6F6E206F726967696E616C204DCE
:100C3000696B726F4B6F707465722D486172647767
:100C4000617265004143542044534C004A65746905
:100C500020736174656C6C6974005370656B747299
:100C6000756D20736174656C6C697420284C6F77A6
:100C7000207265736F6C7574696F6E2900537065AF
:100C80006B7472756D20736174656C6C6974202867
:100C90003230343829005370656B7472756D20736F
:100CA0006174656C6C6974004D756C746973696707
:100CB0006E616C2050504D000A0D52656365697677
:100CC00065723A2000756E6B6E6F776E2E205573CD
:100CD000696E672050504D2E2E2E006E6F7420735B
:100CE0007570706F727465642062792068617264D7
:100CF0007761726521000A0D3D3D3D3D3D3D3D3D25
:100D00003D3D3D3D3D3D3D3D3D3D3D3D3D3D3D3D13
:100D10003D3D3D3D3D3D3D3D3D3D3D000A0D466C6B
:100D200069676874436F6E74726F6C0A0D48617204
:100D300064776172653A25642E25640A0D536F66E7
:100D400074776172653A5625642E25642563200008
:100D50000A0D3D3D3D3D3D3D3D3D3D3D3D3D3D3D26
:100D60003D3D3D3D3D3D3D3D3D3D3D3D3D3D3D3DB3
:100D70003D3D3D3D3D0011241FBECFEFD0E1DEBF24
:100D8000CDBF11E0A0E0B1E0E2E4F2EF02C00590D7
:100D90000D92A63FB107D9F718E0A6EFB1E001C068
:100DA0001D92A53CB107E1F76AEAE2E0F0E081E2DA
:100DB000809357007491AE014F5F5F4F20EF37EF84
:100DC000DA019FE0F9012F5F3F4F84918D9391509D
:100DD00097FFF8CF773911F40000FECFFA019EE0BB
:100DE000819168276095915097FFFACF888968179D
:100DF00021F0773911F40000FECF0C94C0070C9459
:100E0000000080911F06E82FFF27EE0FFF1FE75B12
:100E1000F84F808191818D5E9F4F14F010920301F5
:100E2000808191818A5B9F4FCCF48091030188235C
:100E3000A9F481E080930301809162048F5F809325
:100E40006204853038F088EE93E090932902809315
:100E5000280204C066E970E00E94F23680916204C4
:100E600099279093F0058093EF0508951F93CF93F2
:100E7000DF93182F882389F082EF90E09F938F9360
:100E800084EF92E19F938F93E0912E04F0912F04D1
:100E900009950F900F900F900F908091420682332A
:100EA00008F044C084EF91E00E941A17EC0111236E
:100EB00029F0CE010E9423178823D9F3C2E0D0E0A5
:100EC00026E530E080911E0190911F018217930763
:100ED00030F02196255D3F4FC730D10598F38091C2
:100EE00042069927C89F9001C99F300DD89F300DA9
:100EF0001124209300011123D9F068EC70E08C2FAD
:100F00000E94F236DF93CF938AEF90E09F938F9306
:100F100084EF92E19F938F93E0912E04F0912F0440
:100F200009958DB79EB706968DBF02C080930001CC
:100F3000112311F1809100016AE00E944C78892F01
:100F400099279F938F93809100010E944C78992755
:100F50009F938F9385E091E09F938F9384EF92E12D
:100F60009F938F93E0912E04F0912F0409952DB754
:100F70003EB7285F3F4F2DBFDF91CF911F9108955E
:100F8000CFEFD0E1DEBFCDBF8824992414B815B8C7
:100F900007EE13E00253104017FFFCCF189B06C06A
:100FA000199B02C08DE007C08BE005C0199B02C0F1
:100FB00084E101C08AE08093020181E887B93E9A0A
:100FC0008FEF88B98BE184B981E085B98EE38AB966
:100FD00087E48BB9469A84B7877F84BF809160008D
:100FE0008861809360001092600084EC99E0909397
:100FF00029028093280210921C0310921B03109266
:101000004E0710924D0710921E0310921D0310926E
:10101000200310921F0320910201243128F084EC58
:1010200094E0A0E0B0E004C08BE095E0A0E0B0E088
:1010300080939A0190939B01A0939C01B0939D0192
:101040002A3011F0243110F0289801C0289A0E940B
:1010500083170E9454170E94FC120E946C330E9456
:10106000B31A81E00E94CF2E0E9408630E942D6E69
:101070000E943B76809102018C3010F4299A01C0C5
:10108000299878940E94EE2D80917002826080935E
:101090007002109273020E94144284EF91E00E9449
:1010A0001A178C018091700280FD05C0C8010E9452
:1010B00023178823B9F38FE191E09F938F93B4EFC7
:1010C000AB2EB2E1BB2EBF92AF92E0912E04F09115
:1010D0002F04099580EA9FE00E941A178C01C0E056
:1010E000D0E00F900F900F900F90ABEEEA2EA6E09D
:1010F000FA2EFFE9CF2EF6E0DF2E0E9414428091F7
:10110000700280FD05C0C8010E9423178823B9F32F
:10111000F60180811816ACF40BC00E941442809135
:10112000700280FD05C0C8010E9423178823B9F30F
:10113000C8010E942317882321F4F70180818823A6
:1011400064F7F701808187FF18C02196DF93CF9362
:10115000219781E391E09F938F93BF92AF92E091AB
:101160002E04F0912F0409958091F6018F5F8093F2
:10117000F6018DB79EB706968DBF2196E4E0F0E0AC
:10118000CE0EDF1E88E090E0E80EF91ECC30D105CF
:1011900008F4B3CFC0E0D0E008EE16E0EFE9EE2EA1
:1011A000E6E0FE2EF801838187FD1CC0F7018081F7
:1011B0001816C4F42196DF93CF93219784E391E02E
:1011C0009F938F9384EF92E19F938F93E0912E04EE
:1011D000F0912F04099582E0809326028DB79EB787
:1011E00006968DBFF801838180788383219684E001
:1011F00090E0E80EF91E085F1F4FCC30D10590F249
:1012000082E591E09F938F93C4EFD2E1DF93CF9378
:10121000E0912E04F0912F04099590911D06809184
:10122000F6010F900F900F900F90981728F480916F
:10123000480480618093480488E791E09F938F93EE
:10124000DF93CF93E0912E04F0912F04099588EE5F
:1012500093E00E941A178C010E94B91A0F900F9008
:101260000F900F90C8010E9423178823D9F388E9B3
:1012700091E09F938F93DF93CF93E0912E04F091B1
:101280002F04099580E00E94B437809102010F90ED
:101290000F900F900F908A3011F0843110F0289841
:1012A00001C0289A80ED97E090932902809328024C
:1012B00085E5809364048EE090E00E94802C99275D
:1012C000182F00278FE090E00E94802C080F111D3E
:1012D0001093FC010093FB018AE090E00E94802CB7
:1012E0009927182F00278BE090E00E94802C080F90
:1012F000111D1093FA010093F9010F5F1F4F39F090
:101300008091FB019091FC018F5F9F4F41F41092FF
:10131000FC011092FB011092FA011092F9018091E8
:10132000F9019091FA019F938F938091FB01909125
:10133000FC019F938F938DE991E09F938F93DF93AF
:10134000CF93E0912E04F0912F0409958DB79EB7AD
:1013500008968DBF80EC91E09F938F93DF93CF939E
:10136000E0912E04F0912F04099580912B060F90A7
:101370000F900F900F90E0912E04F0912F0482FFB8
:1013800007C08CEC91E09F938F93DF93CF9308C0BD
:1013900088ED91E09F938F9384EF92E19F938F93D9
:1013A00009950F900F900F900F900E94D71F88E81B
:1013B00093E1909393018093920181E08093630481
:1013C0000E943607809145060E94A1758AEE91E041
:1013D0009F938F93DF93CF93E0912E04F0912F048E
:1013E000099580ED97E00E941A178C018AEF90E032
:1013F0000E941A17EC0183E08093C7050F900F90AD
:101400000F900F908091FE018111FFCFCE010E94BD
:101410002317882339F084E690E00E941A17EC0124
:101420000E94F77680912C02882309F4D5C180911F
:101430001001882309F4D0C110922C02809162041B
:10144000882319F00E94010702C00E9409450E94EA
:101450001442209102012A3011F0243110F0289812
:1014600001C0289A8091210390914804882339F083
:1014700080912103815080932103977F0AC080913E
:101480006F00806280936F0010924A0710924907A4
:1014900098609093480480919201909193010197F4
:1014A0009093930180939201809192019091930186
:1014B000892B21F0809171028823C9F180919201DA
:1014C00090919301892BD9F40E94F92E85E090E048
:1014D000909393018093920180910106909102066E
:1014E00001969093020680930106809148048160E2
:1014F000809348048091C80582608093C8058091DC
:101500000801909109018F5F9F4F19F58091180391
:101510008823F9F080E197E29093290280932802D2
:1015200080E890E0909309018093080112C02A306E
:1015300011F0243110F0289801C0289A80912802D7
:1015400090912902892B29F4809148048E7F809301
:10155000480480912C02882309F03EC180910E013D
:10156000882311F00E949A170E943F130E947A0E5E
:10157000C8010E942317882309F42AC10C5E1F4F5B
:101580008091710290914804882339F09260909381
:1015900048048091C80582600CC09D7F90934804E8
:1015A0008091920190919301079728F08091C8054E
:1015B0008D7F8093C8058091920190919301079748
:1015C00028F0809148048E7F809348048091050123
:1015D000882321F081508093050125C080936E04FB
:1015E0001092F9021092F8021092F7021092F6028D
:1015F0001092F5021092F402809108019091090175
:101600008F5F9F4F81F480912103882361F488E9E3
:101610009AE3909329028093280280E09CE09093C3
:101620000901809308018091ED01893C48F08150C7
:101630008093ED01809148048B7F8093480430C0F3
:10164000809127088823E1F080914804846080938A
:10165000480480910801909109018F5F9F4F81F4A8
:1016600080911803882361F088E99AE39093290216
:101670008093280280E098EA909309018093080102
:101680001092FE031092FD031092FC031092FB03D4
:101690008FEF9FEF90935508809354081092ED01BF
:1016A00080910001282F332780911E0190911F0106
:1016B00082179307CCF48091ED0280628093ED0253
:1016C00080910801909109018F5F9F4FC1F480E7DD
:1016D00097E1909329028093280280E093E0909311
:1016E0000901809308010BC0809128029091290282
:1016F000892B29F48091ED028F7D8093ED020E9469
:10170000146784E08093270280911803882329F4CA
:101710005AEA852E55E0952E12C08091FD018F5F0B
:101720008093FD01813359F41092FD018091F701FE
:101730009091F80101969093F8018093F701089435
:10174000811C911CF2E78F16FBE09F0609F040C058
:10175000882499242091FB013091FC012F5F3F4F99
:101760003093FC012093FB018091F9019091FA01E3
:1017700001969093FA018093F901832F9927682F9E
:101780008EE090E00E94862C8091FB019091FC01FC
:101790009070682F8FE090E00E94862C8091F90174
:1017A0009091FA01892F9927682F8AE090E00E9492
:1017B000862C8091F9019091FA019070682F8BE04E
:1017C00090E00E94862C84E190E00E941A178C0120
:1017D0000E9464670E94446E80912702882309F06A
:1017E00011CE0E9429630ECE1F920F920FB60F9258
:1017F00011248F939F93EF93FF9380910701882388
:10180000E1F48091180290911902019690931902C7
:1018100080931802FC01E35EFA4FE081ED3019F08D
:101820008A3A910539F4109219021092180281E057
:1018300080930701E093C60004C010921902109231
:101840001802FF91EF919F918F910F900FBE0F9013
:101850001F9018951F920F920FB60F9211242F937D
:101860003F934F935F936F937F938F939F93AF9328
:10187000BF93CF93EF93FF9390E08091FE0181306F
:1018800029F48091C6008093CE00CCC08091FE01E7
:10189000823029F48091C60080937104C3C0809186
:1018A000C6008093100250911E025A3A10F0909395
:1018B0001F02809110028D3009F065C080911F02D7
:1018C000823009F060C090931F02852F99278F58AE
:1018D0009B4FFC013297408120911A0230911B02EC
:1018E000241B3109DC0111978C91281B3109C90196
:1018F0009F7090931B0280931A0246E096958795FD
:101900004A95E1F7982F935C90931C022F733070E7
:10191000235C20931D028081981729F48C9128174D
:1019200011F491E006C090E080910D028F5F8093EA
:101930000D02C0910F02CC2309F074C0992309F461
:1019400071C081E080930F02580F50930C025150E8
:10195000E52FFF27EF58FB4F8DE0808380917304C4
:10196000823509F05FC00E94D71F88E190E02CE02B
:101970000FB6F894A895809360000FBE2093600086
:10198000C09326024FC020911F02822F99278130D9
:101990009105F9F0823091051CF4892B21F040C0AB
:1019A000029711F13DC080911002833239F4809189
:1019B0000F02882319F481E080931F0280911002A6
:1019C0008093710481E080931E0280911002992718
:1019D00022C02F5F20931F02E52FFF27EF58FB4FF8
:1019E00080911002808309C0E52FFF27EF58FB4F3D
:1019F0008091100280835A3A20F45F5F50931E0258
:101A000002C010921F022091100280911A02909140
:101A10001B02820F911D90931B0280931A0202C039
:101A200010921F02FF91EF91CF91BF91AF919F91C3
:101A30008F917F916F915F914F913F912F910F9077
:101A40000FBE0F901F901895AC01A0E0B0E09D0173
:101A5000A817B90748F4EDE1F5E08191280F311D91
:101A60001196A417B507C8F33F70FD01E35EFA4F66
:101A7000C90156E0969587955A95E1F7835C808376
:101A80001196FD01E35EFA4F2F733070822F835C55
:101A90008083A25EBA4F8DE08C93109207018091F3
:101AA0001D058093C6000895A0E0B0E0EAE5FDE0E2
:101AB0000C94C5782C859D850E85BB2483E280938C
:101AC0001D059F5990931E0520931F0533E0E32EBB
:101AD000F12C002309F49EC0CF84D888BE016D5E2E
:101AE0007F4FA989BA890150109709F493C01097C4
:101AF000B9F0F601EB0DF11DB3949081119791F4BB
:101B0000002349F1FB016E5F7F4FDB01C080D18074
:101B10006E5F7F4F0D90BC91A02DBB24015002C081
:101B200090E019C01097B9F0F601EB0DF11DB394D8
:101B30004081119791F4002341F1FB016E5F7F4FCB
:101B4000DB01C080D1806E5F7F4F0D90BC91A02DD6
:101B5000BB24015002C040E018C01097B1F0F6015C
:101B6000EB0DF11DB3941081119781F4002371F0F6
:101B7000FB013296DB01CD90DC90BF016E5F7F4FA1
:101B8000A081B181BB24015001C010E0F701E35EE8
:101B9000FA4F892F86958695835C80830894E11C93
:101BA000F11CF701E35EFA4F892F9927837090703B
:101BB00024E0880F991F2A95E1F755279A0194E0B0
:101BC000369527959A95E1F7822B835C808308945C
:101BD000E11CF11CF701E35EFA4F4F705070440FA7
:101BE000551F440F551F812F992726E096958795FD
:101BF0002A95E1F7842B835C80830894E11CF11C17
:101C0000F701E35EFA4F1F73135C10830894E11C25
:101C1000F11C6ACFC7010E94240DE9E00C94E17821
:101C2000A3E07A2F40910C024650442309F458C097
:101C3000E72FFF27EF58FB4F80818D537F5FE72F02
:101C4000FF27EF58FB4F20812D537F5FE72FFF27A2
:101C5000EF58FB4F30813D537F5FE72FFF27EF5851
:101C6000FB4F60816D537F5F9927880F991F880F05
:101C7000991F522F52955F70582B822F99278F7082
:101C80009070F4E0880F991FFA95E1F7232F2695BD
:101C90002695282B832F992783709070E6E0880F74
:101CA000991FEA95E1F7682B41504F3FC9F0EA2FA1
:101CB000FF27EF58FB4F5083AF5F41504F3F81F0FC
:101CC000EA2FFF27EF58FB4F2083AF5F41504F3F74
:101CD00039F0EA2FFF27EF58FB4F6083AF5FA5CFA6
:101CE00084E794E090930B0280930A02A350A093A0
:101CF00009020895A2E0B0E0E0E8FEE00C94CB78A1
:101D000080910F02882309F46BC40E94100E809109
:101D10007204823609F025C38091730499278037B5
:101D2000910509F4C1C081379105C4F48A36910543
:101D300009F48DC28B36910544F48B34910571F111
:101D40008636910509F46CC10CC38D36910509F4F2
:101D50007BC08E36910509F45FC003C384379105BB
:101D6000D1F1853791054CF48137910509F4A3C071
:101D70008337910509F4F1C0F4C28737910509F45E
:101D800028C2883791052CF48537910509F4E4C100
:101D9000E8C28937910509F47AC1E3C2E0910A02E9
:101DA000F0910B02808191819093340380933303EF
:101DB0002091310330913203821B930B845E9D4F3F
:101DC00068E671E00E946C78845B904090933003E9
:101DD00080932F03C6C280910C02A0910A02B09199
:101DE0000B02853140F080E1ECE4F4E00D900192CB
:101DF0008A95E1F70DC08D919D910D90BC91A02D1C
:101E000080934C0490934D04A0934E04B0934F04E0
:101E100080EF809307024BC0809107018823E1F394
:101E20008DE490E09F938F9382E996E09F938F9348
:101E300081E08F938F938EE48F930E94540D8DB722
:101E40009EB707968DBF8DC2A0910A02B0910B027A
:101E50001C91113081F48DE4E2E9F6E00D900192DD
:101E60008A95E1F70E943D2D1983809148048F7E69
:101E70008093480401C01982809107018823E1F30F
:101E800081E090E09F938F93CE0101969F938F9373
:101E900081E08F938F938DE48F930E94540DADB7A3
:101EA000BEB71796ADBF5DC281E0809312028FEF7F
:101EB0008093050156C2E0910A02F0910B02E08185
:101EC0008E2F8A508A3058F48983882311F481E058
:101ED00003C0863010F085E0898361E00EC08E2F4C
:101EE00084518A3070F48983882311F481E003C01F
:101EF000863010F085E0898360E089810E94B12DF1
:101F000012C0E983EF3F19F40E94A22D89838981D1
:101F1000882311F481E003C0863010F085E08983C6
:101F200089810E94952C809107018823E1F383E742
:101F300090E09F938F938EE196E09F938F9381E043
:101F400090E09F938F93CE0101969F938F9382E0B1
:101F50008F9381E08F9381E572C120910A023091C5
:101F60000B02D9018C918150853008F040C0F901F5
:101F700081818535E1F52F5F3F4F83E7EEE1F6E0A4
:101F8000D9010D9001928A95E1F7F90182910E94A1
:101F9000D92C80915F069927AA27BB27BC01CD01C8
:101FA00024EC39E040E050E00E942D78DC01CB01C8
:101FB0008093D9019093DA01A093DB01B093DC0107
:101FC000809160069927AA27BB27BC01CD010E94FA
:101FD0002D78DC01CB018093D5019093D601A0939D
:101FE000D701B093D8010E94A22D898301C0198224
:101FF000809107018823E1F381E090E09F938F9324
:10200000CE0101969F938F9381E08F938F9383E509
:102010008F930E94540D8DB79EB707968DBF26C033
:10202000E0910A02F0910B02E0818E2F8150853001
:1020300018F48E2F0E94952C0E94A22D89838091E6
:1020400007018823E1F381E090E09F938F93CE0115
:1020500001969F938F9381E08F938F9386E48F9364
:102060000E94540DADB7BEB71796ADBF809118034F
:10207000882329F46EE670E089810E94F23680E0C0
:102080000E943607809145060E94A1756AC1E091C1
:102090000A02F0910B028081992787FD9095909319
:1020A0006407809363078181992787FD90959093BA
:1020B0006607809365078281992787FD90959093A5
:1020C0006807809367078381992787FD9095909390
:1020D0006A07809369078481992787FD909590937B
:1020E0006C0780936B078581992787FD9095909366
:1020F0006E0780936D078681992787FD9095909351
:10210000700780936F078781992787FD909590933B
:102110007207809371078085992787FD909590932A
:102120007407809373078185992787FD9095909315
:102130007607809375078285992787FD9095909300
:102140007807809377078385992787FD90959093EB
:102150007A078093790705C1E0910A02F0910B029A
:1021600080810E94C5328A83882319F481E08983A3
:1021700001C01982809107018823E1F388E090E093
:102180009F938F9380EE96E09F938F9321E030E0B2
:102190003F932F9380910A0290910B029F938F930C
:1021A0003F932F93CE0102969F938F933F932F934C
:1021B000CE01820F931F9F938F9384E08F9381E0D2
:1021C0008F9385E58F930E94540DEDB7FEB77396FC
:1021D0003CC080910902893008F4C3C020910A02F2
:1021E00030910B022F5F3F4F88E0A0EEB6E0F9017F
:1021F00001900D928A95E1F7D9018E910E941B32D0
:102200008A83882319F481E0898301C0198280912F
:1022100007018823E1F321E030E03F932F93CE01C3
:1022200002969F938F933F932F93CE01820F931F1C
:102230009F938F9382E08F9381E08F9387E58F93B5
:102240000E94540DEDB7FEB73B96EDBF8AC00E94C9
:1022500054758983823019F0843009F082C0F89473
:102260008091C1008F738093C1008091C9008F73EA
:102270008093C9008091C100877E8093C1008091C6
:10228000C900877E8093C9008091C80087FF03C082
:102290008091CE00F9CF8091C00087FF03C080916C
:1022A000C600F9CFE0910A02F0910B0280818823E9
:1022B00059F581E08093FE011092CD0080E490E01A
:1022C0008093CC008091CD008093C5008091CC009C
:1022D0008093C4008091CA008F7D8093CA00809152
:1022E000CA008F7E8093CA008091C9008B7F809343
:1022F000C9008091CA0084608093CA008091CA009E
:1023000082608093CA0003C082E08093FE018091C6
:10231000CA00877F8093CA008091C200877F809324
:10232000C2008091C9008E7F8093C9008091C10056
:1023300088618093C1008091C90088618093C90041
:102340008091C10080688093C1008091C90080683D
:102350008093C90010926E0010926F00109270006E
:1023600078948091730499278436910509F4CDC03F
:1023700085369105ACF48136910509F481C0823629
:1023800091052CF48B34910509F45DC021C182368E
:10239000910509F482C08336910509F491C018C1F2
:1023A0008C36910509F4FFC08D3691054CF48736C3
:1023B000910509F40AC18836910509F4C4C008C121
:1023C0008437910529F08637910509F4FAC000C1D8
:1023D00080910C02A0910A02B0910B02803140F072
:1023E00080E1ECE4F4E00D9001928A95E1F70DC0F4
:1023F0008D919D910D90BC91A02D80934C04909354
:102400004D04A0934E04B0934F048091070188239C
:10241000E1F31F92809104018F9384E58F930E94D2
:10242000540D8AEF809307028FEF8093050180EAB5
:102430009FE00E941A17909300028093FF010F9073
:102440000F900F90C5C0E0910A02F0910B028081BD
:102450009181909334038093330320913103309121
:102460003203821B930B845E9D4F68E671E00E94ED
:102470006C78845B90409093300380932F03A8C0C6
:10248000E0910A02F0910B02808180930601803274
:1024900098F08FE1809306010FC0A0910A02B091DD
:1024A0000B028BE0E4E6F4E00D9001928A95E1F7EF
:1024B00080916D04809309068FEF8093050188C099
:1024C0008091030290910402892B89F4E0910A0221
:1024D000F0910B02E081EE2351F08AE0E89FC00109
:1024E00011240E941A1790933F0480933E04E091B8
:1024F0000A02F0910B0290818AE0989FC00111249A
:10250000909304028093030215C08FEF809305011E
:10251000E0910A02F0910B0290818AE0989FC0013D
:1025200011249093060280930502892B19F081E013
:102530008093140280EA9FE00E941A179093000291
:102540008093FF0145C08FEF80930501E0910A025F
:10255000F0910B02908197FD08C082E080931102F8
:1025600010920202109201021AC0909580916902A5
:10257000892B8093690291818AE0989FC001112480
:10258000909302028093010284E08093110280EA1A
:102590009FE00E941A17909300028093FF0181E050
:1025A0008093150215C08FEF80930501E0910A0218
:1025B000F0910B02808180936A0281E08093160281
:1025C00007C081E08093130203C081E0809317026B
:1025D00010920F0210920B0210920A02109209023E
:1025E000E3E0CE5F0C94E778982F8091C00085FFE0
:1025F000FCCF9093C60008950F931F9388E18093BA
:10260000C1008091C00082608093C0008091C100B1
:1026100080688093C1008091C10080648093C10074
:1026200000E010E00093C5008AE290E08093C400CF
:1026300080910502909106020E941A17909341041E
:10264000809340048CED90E00E941A1790937004E0
:1026500080936F041092420482E5809343041092A9
:1026600046048BE0809344041092450410930B02BF
:1026700000930A02109209021F910F910895A0E1A0
:10268000B0E0E5E4F3E10C94C87880910701882379
:1026900009F4C1C28091FF01909100020E942317AA
:1026A000882361F010920202109201021092060239
:1026B000109205021092040210920302809101020E
:1026C00090910202892B41F080911B0590911C058D
:1026D0000E942317882329F480911502882309F486
:1026E00060C080910701882309F45BC080911102CA
:1026F00001E211E08430A8F00E94EB1F80E590E039
:102700009F938F931F930F9381E08F938F9388E410
:102710008F930E94540D2DB73EB7295F3F4F2DBFB9
:1027200034C010926B0282E194E09F938F9380EE0D
:102730009FE19F938F93E0912E04F0912F040995D0
:1027400084E190E09F938F931F930F9381E090E03B
:102750009F938F9381E192E09F938F9382E08F9379
:1027600081E08F9388E48F930E94540D8091110231
:10277000982F8F5F809311022DB73EB7215F3F4F97
:102780002DBF943010F010921102809101029091AF
:1027900002020E941A1790931C0580931B05109249
:1027A000150280911602882351F180910701882338
:1027B00031F10E94EB1F80E590E09F938F9381E2BF
:1027C00091E09F938F9321E030E03F932F9380E23D
:1027D00091E09F938F933F932F938AE692E09F938C
:1027E0008F9383E08F9381E08F938CE48F930E948B
:1027F000540D109216028DB79EB70F968DBF809123
:1028000013028823D1F0809107018823B1F08AE078
:1028100090E09F938F9382E494E09F938F9381E065
:102820008F938F9386E58F930E94540D109213021D
:102830002DB73EB7295F3F4F2DBF809117028823E8
:10284000D9F0809107018823B9F08BE090E09F9345
:102850008F9384E694E09F938F9381E08F93809190
:1028600004018F9387E48F930E94540D10921702F6
:102870008DB79EB707968DBF80916F0490917004BD
:102880000E942317882309F461C0809107018823DF
:1028900009F45CC080913A069927880F991F880F28
:1028A000991F7C010027F7FC0095102F809175037C
:1028B00090917603A0917703B0917803BC01CD018C
:1028C000A80197010E94A17830935D0420935C04D5
:1028D00080916D0390916E03A0916F03B09170038E
:1028E000BC01CD01A80197010E94A17830935F043B
:1028F00020935E0480910203809360048091010321
:102900008093610488E090E09F938F938CE594E03E
:102910009F938F9381E08F9383E08F938BE68F93C8
:102920000E94540D809162042DB73EB7295F3F4F3E
:102930002DBF853018F086E08093620483E690E036
:102940000E941A179093700480936F04809105027F
:1029500090910602892B41F08091400490914104AE
:102960000E942317882321F480911402882339F1CF
:1029700080910701882319F10E94E83582E490E0F4
:102980009F938F9387EC95E09F938F9381E08F9334
:102990008F9384E48F930E94540D109214028DB78C
:1029A0009EB707968DBF8091050290910602009711
:1029B00031F00E941A179093410480934004809153
:1029C000030290910402892B09F4B8C080913E045F
:1029D00090913F040E942317882309F4AFC080918F
:1029E0000701882309F4AAC080913A069927880F25
:1029F000991F880F991F7C010027F7FC0095102F65
:102A00008091750390917603A0917703B09178033C
:102A1000BC01CD01A80197010E94A1783093310437
:102A20002093300480916D0390916E03A0916F0309
:102A3000B0917003BC01CD01A80197010E94A1785B
:102A4000309333042093320420910F083091100802
:102A50004091110850911208DA01C90163E0880F12
:102A6000991FAA1FBB1F6A95D1F7820F931FA41F3E
:102A7000B51F820F931FA41FB51F20919A0130919B
:102A80009B0140919C0150919D01BC01CD010E9490
:102A9000A178309335042093340480913D039091C4
:102AA0003E03A0913F03B091400339E0B595A7954F
:102AB000979587953A95D1F780933604809139039D
:102AC00090913A03A0913B03B0913C0329E0B59566
:102AD000A795979587952A95D1F78093370480918C
:102AE000450390914603A0914703B091480309E044
:102AF000B595A795979587950A95D1F78093380452
:102B00008EE090E09F938F9380E394E09F938F9368
:102B100081E08F938F9383E48F930E94540D809173
:102B20000302909104020E941A1790933F0480932D
:102B30003E042DB73EB7295F3F4F2DBF8091060160
:102B40008F3F71F1992714E0880F991F1A95E1F7CB
:102B50008E5E9D4F40E150E0BC01CE0101960E9487
:102B60005B7780E190E09F938F93CE0101969F93D6
:102B70008F9381E090E09F938F9386E091E09F9305
:102B80008F9382E08F9381E08F9381E48F930E94F3
:102B9000540D8FEF809306018DB79EB70B968DBFB6
:102BA000809109068823D1F0809107018823B1F034
:102BB00081E090E09F938F9389E096E09F938F93BD
:102BC00081E08F938F9382E48F930E94540D109233
:102BD00009062DB73EB7295F3F4F2DBF80911202E6
:102BE0008823C9F0809107018823A9F084E390E04D
:102BF0009F938F9389E497E09F938F9381E08F93C6
:102C00008F9380E58F930E94540D109212028DB71E
:102C10009EB707968DBFE6E0C05F0C94E4781F92E4
:102C20000F920FB60F9211242F933F935F936F93E0
:102C30007F938F939F93AF93BF93EF93FF9320E086
:102C400080912702882329F0809127028150809368
:102C5000270280911104882319F081508093110478
:102C600080912F02815080932F028F3F09F05BC02B
:102C700089E080932F0280912D0290912E0201967F
:102C800090932E0280932D0280910F018F5F8170AF
:102C900080930F01882319F481E080932C023499EA
:102CA00003C081E080933002809128029091290234
:102CB000892B21F180912802909129020B9750F0E5
:102CC00080912802909129020A979093290280937B
:102CD000280204C010922902109228028091280232
:102CE00090912902209108013091090182239323B8
:102CF000892B11F021E008C020E006C08FEF9FEF84
:102D0000909309018093080180910201222331F000
:102D10008A3011F45A9A07C0479A05C08A3011F4D4
:102D20005A9801C0479880913002882309F472C0F4
:102D30002091ED01222309F06DC080912B0683FFC5
:102D400069C086B19927FC01E071F07084FF14C05E
:102D500080912A0290912B02019690932B028093EE
:102D60002A0280912A0290912B02895E934008F4F6
:102D700051C0209330024EC080912A0290912B02C4
:102D8000892B09F443C080912A0290912B028A5624
:102D90009140E0F580912A0290912B0269E270E067
:102DA0000E94587880912A0290912B02860F971FDB
:102DB00090932B0280932A0280912A0290912B02F9
:102DC0000B9750F080912A0290912B020A979093D2
:102DD00034038093330304C0F0933403E09333034C
:102DE0008091330390913403209131033091320369
:102DF000821B930B845E9D4F68E671E00E946C78A5
:102E0000845B90409093300380932F0310922B02A9
:102E100010922A02FF91EF91BF91AF919F918F91F4
:102E20007F916F915F913F912F910F900FBE0F9007
:102E30001F90189520912D0230912E02280F391FD6
:102E4000C9010196089520912D0230912E02821B16
:102E5000930B892F99278695807490700895CF934E
:102E6000DF930E941A17EC01CE010E9423178823DA
:102E7000D9F3DF91CF910895CF93DF930E941A1772
:102E8000EC0109C080911001882329F09093100172
:102E90008FEC80937A00CE010E942317982F88230D
:102EA00089F3DF91CF9108959FB7F8945F983E9A88
:102EB000469A8091B0008F708093B0008091B000EE
:102EC00083608093B0008091B1008B738093B100D8
:102ED0008091B1008B608093B1001092B2008FEFAF
:102EE0008093B3008091B00080688093B00080919F
:102EF00070008A7F80937000809170008260809360
:102F000070009FBF08958AE090E00E941A17909386
:102F100036028093350282E085BD83EA84BD17BC0A
:102F200084EB88BD86E086BD80916E0081608093D1
:102F30006E000895A0E0B0E0E0EAF7E10C94C778F5
:102F400080915506E82FFF27E056FE4F9681D080EE
:102F500080910E01A92FBB27A7FDB095CB2FDB2FAA
:102F6000813009F0C9C020917503309176034091FA
:102F7000770350917803BD01CE010E942D7897FF11
:102F800004C061587F4F8F4F9F4F7B018C0167E0DA
:102F900015950795F794E7946A95D1F78D2D9927A4
:102FA00087FD9095A92FB92F20916D0330916E0365
:102FB00040916F0350917003BC01CD010E942D78A8
:102FC00097FF04C061587F4F8F4F9F4F57E09595F3
:102FD0008795779567955A95D1F7F801E701C61B54
:102FE000D70BE80BF90B80914C069927AA27BB2732
:102FF000BC01CD019E01AF010E942D7897FF04C056
:1030000061507E4F8F4F9F4FFC01EB0149E0F595DA
:10301000E795D795C7954A95D1F78091C50199272E
:1030200036E0880F991F3A95E1F740910C015091D5
:103030000D01209154063327841B950BB9010E9482
:103040006C7880910C0190910D01860F971F9093E1
:103050000D0180930C0180910C0190910D0197FD61
:103060000F9624E0959587952A95E1F79093230292
:10307000809322028091830680FF07C08091220204
:10308000909123028C0F9D1F06C080912202909187
:1030900023028C1B9D0B909323028093220280912C
:1030A0004D06282F3327220F331F220F331F809105
:1030B000220290912302821793077CF080914E06A2
:1030C000282F3327220F331F220F331F8091220214
:1030D000909123022817390724F430932302209378
:1030E000220280910201843108F4C2C080910E0155
:1030F0008F5F80930E01BEC020916D0330916E03EF
:1031000040916F0350917003BD01CE010E942D7854
:1031100097FF04C061587F4F8F4F9F4F7B018C01F9
:10312000C7E015950795F794E794CA95D1F78D2DCB
:10313000992787FD9095A92FB92F2091750330917C
:1031400076034091770350917803BC01CD010E9432
:103150002D789B01AC0197FF04C021583F4F4F4F82
:103160005F4FB7E05595479537952795BA95D1F7B5
:103170002E0D3F1D401F511F809150069927AA27F1
:10318000BB27BC01CD010E942D7897FF04C0615080
:103190007E4F8F4F9F4FFC01EB01A9E0F595E7951E
:1031A000D795C795AA95D1F78091C401992776E064
:1031B000880F991F7A95E1F740910A0150910B0110
:1031C000209154063327841B950BB9010E946C781B
:1031D00080910A0190910B01860F971F90930B012C
:1031E00080930A0180910A0190910B0197FD0F963F
:1031F00064E0959587956A95E1F790932102809315
:1032000020028091830681FF07C080912002909167
:1032100021028C0F9D1F06C08091200290912102F7
:103220008C1B9D0B9093210280932002809151066C
:10323000282F3327220F331F220F331F80912002A4
:1032400090912102821793077CF080915206282FDB
:103250003327220F331F220F331F809120029091BA
:1032600021022817390724F43093210220932002E9
:1032700010920E01E7E0CDB7DEB70C94E3781F9211
:103280000F920FB60F9211242F933F934F935F939A
:103290008F939F93EF93FF9380910201909131025E
:1032A000843108F04CC0992309F01CC18091B00012
:1032B00086FF24C08091B0008F7B8093B000809106
:1032C00022029091230287559E4F9093250280936E
:1032D000240225E08D3D920718F08CED95E005C0A5
:1032E0008757914030F487E791E0909325028093CF
:1032F00024028091240290912502BAC08091B000EE
:1033000080648093B00080915306282F33278DED81
:1033100096E0289FA001299F500D389F500D112441
:10332000CA012091320230913302821B930B909399
:1033300025028093240281E080930E01D0C099235E
:1033400009F0D0C08091B00086FF97C08091B00096
:103350008F7B8093B000E0913402EE23F1F48091F2
:103360005306282F33278DED96E0289FA001299F33
:10337000500D389F500D1124CA0120913202309116
:103380003302821B930B90932502809324021092A8
:10339000330210923202469AA2C089EA93E09093D7
:1033A0002502809324028E2F992783309105D9F02E
:1033B0008430910534F48130910549F0029761F031
:1033C00020C08430910591F0059799F01AC0809142
:1033D00022029091230204C0809120029091210248
:1033E00087559E4F1DC08091DD0705C08091B707AE
:1033F00002C08091E5079927880F991F880F991FB0
:10340000EFCFFF27EE0FFF1FE75BF84F20813181E1
:10341000220F331F8091240290912502820F931F67
:10342000909325028093240280912402909125029A
:1034300055E08D3D950718F08CED95E005C0875758
:10344000914030F487E791E0909325028093240225
:1034500020912402309125022C5B304030932502CC
:10346000209324028091320290913302820F931FA5
:10347000909333028093320232C08091B000806416
:103480008093B0008CEB90E090932502809324020F
:10349000809132029091330284549F4F9093330273
:1034A0008093320280912602882321F080912103AB
:1034B000833320F480912602823011F4469801C0B3
:1034C000469A809134028F5F809334029091530624
:1034D000981728F481E080930E011092340281E065
:1034E00080933102209124023091250241E02F3750
:1034F000340730F08FEF8093B3002F5F30400FC060
:103500002F3F3105C9F0C0F0A9014F5F50404F3740
:10351000510550F480E88093B30020583040309338
:1035200025022093240212C08FEF8093B3005093A2
:103530002502409324020AC0809124028093B300A4
:10354000109225021092240210923102FF91EF9105
:103550009F918F915F914F913F912F910F900FBE4F
:103560000F901F90189510927C008FEC80937A003A
:103570000895CF93DF9310923B0283E090E00E9486
:10358000802CC82FDD27C531D10508F02A97C7BD8B
:1035900084E690E00E943C178091140190911501FF
:1035A0008052934010F4C0E0D0E0CA3FD105F8F457
:1035B000C7BD82E390E00E943C1787E294E09F93AE
:1035C0008F9384EF92E19F938F93E0912E04F0917B
:1035D0002F04099580911401909115010F900F907F
:1035E0000F900F908052934010F02196DECFC09341
:1035F0001A066C2F83E090E00E94862C80912B06A7
:1036000080FF0AC080911A068A508B3E28F0809174
:103610004704806480934704C7BD8CE291E00E9418
:103620003C17DF91CF910895EF92FF921F93CF93B4
:1036300010E080ED97E00E941A177C01CCE813306F
:1036400019F4CB3008F0C9E010E080914B02909162
:103650004C028C5F934024F48091130181500AC086
:1036600080914B0290914C028750944034F08091AD
:1036700013018F5F8093130101C011E08091490213
:1036800090914A028C5F934024F480911201815002
:103690000AC08091490290914A028750944034F0C8
:1036A000809112018F5F8093120101C01F5F809192
:1036B0004702909148028C5F934024F4809111015D
:1036C00081500AC0809147029091480287509440EF
:1036D000C4F0809111018F5F8093110113C089E2C2
:1036E00094E09F938F9384EF92E19F938F93E09167
:1036F0002E04F0912F0409950F900F900F900F90CA
:103700005FC01F5F82E180937602809170028E7F9E
:103710008093700285EA8093BC00809113018A3007
:1037200040F4809147048160809347048AE080934D
:10373000130180911301863F40F08091470481601E
:103740008093470485EF80931301809112018A30A2
:1037500040F4809147048260809347048AE080931C
:10376000120180911201863F40F0809147048260EF
:103770008093470485EF80931201809111018A3074
:1037800040F4809147048460809347048AE08093EA
:10379000110180911101863F40F0809147048460BF
:1037A0008093470485EF80931101809176028823EE
:1037B00039F0C7010E942317882309F090CFF5CF75
:1037C000109210018FEC80937A0080911001882371
:1037D000E1F3CA3020F48AE090E00E943C17C15027
:1037E00009F02DCF86E490E00E943C17CF911F9105
:1037F000FF90EF9008951F920F920FB60F92112431
:10380000AF92BF92CF92DF92EF92FF920F931F93EE
:103810002F933F934F935F936F937F938F939F93D8
:10382000AF93BF93EF93FF9380915402282F3327D8
:10383000442755278F5F80935402F90122313105C7
:1038400008F08CC3E25CFF4F0C94F3788091780011
:103850009091790046C080917800909179002CC1B8
:10386000809178009091790090935702809356024E
:1038700057C180917E0390917F0320917800309111
:103880007900821B930B90930B0680930A0680911C
:103890000A0690910B0690936102809360025EC1CC
:1038A000809178009091790020918003309181037C
:1038B000821B930B9093190680931806809118062B
:1038C00090911906909363028093620249C380919C
:1038D0005A0290915B022091780030917900820F1A
:1038E000931F90935B0280935A0281E03AC38091C8
:1038F0005802909159022091780030917900820FFE
:10390000931F909359028093580284E02AC38091B8
:103910001E0190911F019C01220F331F280F391F98
:10392000809178009091790063E070E00E9458786F
:10393000260F371F369527953695279530931F010B
:1039400020931E0185E00DC380917800909179004D
:1039500040917A0350917B03841B950B9093420214
:10396000809341028091410290914202029704F1BA
:1039700022E04E3E520784F4209155022B5F2093A3
:10398000550225508091EE029091EF02845F9140A4
:1039900018F4215F2093550280915502853684F1F9
:1039A0004F5F5F4F50937B0340937A03845626C04A
:1039B00080914102909142028F5F9F4F0CF532E05F
:1039C00047325307ECF020915502255020935502C1
:1039D0002B5F8091EE029091EF02845F914018F48A
:1039E0002F5020935502809155028C394CF4415050
:1039F000504050937B0340937A038C598093550237
:103A000081E08093400280917800909179009093BA
:103A100011068093100680914102909142029C0110
:103A2000442737FD4095542F8091350390913603FC
:103A3000A0913703B0913803820F931FA41FB51FC5
:103A40008093350390933603A0933703B0933803E4
:103A5000209135033091360340913703509138035C
:103A600057FF04C021503C4F4F4F5F4F0AE0559520
:103A70004795379527950A95D1F780913503909111
:103A80003603A0913703B0913803821B930BA40B2C
:103A9000B50B8093350390933603A0933703B0930F
:103AA00038032EC1809158029091590220917800DC
:103AB00030917900820F931F90935902809358029E
:103AC0001092530250C2809102018A3071F48091A9
:103AD0007800909179002091560230915702820F20
:103AE000931F01969695879517C040915602509165
:103AF0005702843158F02091780030917900240FDA
:103B0000351F8FEF97E0821B930B06C080917800E2
:103B100090917900840F951F9093480280934702FB
:103B200086E01FC280917E0390917F0320917800F0
:103B300030917900821B930B90930B0680930A06B9
:103B400080910A0690910B062091600230916102EB
:103B5000820F931F909346028093450287E001C233
:103B600080917800909179002091800330918103B9
:103B7000821B930B90931906809318068091180668
:103B8000909119062091620230916302820F931F77
:103B90009093440280934302E3C120915A023091F2
:103BA0005B028091780090917900280F391F309343
:103BB0005B0220935A02809102018A3019F4220F8D
:103BC000331F04C0220F331F220F331F30935B02B9
:103BD00020935A0220915A0230915B02C90137FDAD
:103BE0000796A3E095958795AA95E1F790934C02E7
:103BF00080934B0280915C0290915D02820F931F33
:103C000097FD01969595879590935D0280935C0250
:103C100020918A0330918B03821B930B90931D019B
:103C200080931C01209151023091520280911C011D
:103C300090911D01280F391F37FF02C02F5F3F4FA2
:103C40003595279530935202209351024ECE209104
:103C50005802309159028091780090917900280F94
:103C6000391F3093590220935802809102018A3003
:103C700019F4220F331F04C0220F331F220F331FEA
:103C800030935902209358022091580230915902E2
:103C9000C90137FD079663E0959587956A95E1F729
:103CA00090934A028093490280915E0290915F0254
:103CB000820F931F97FD01969595879590935F02CC
:103CC00080935E022091880330918903821B930BBD
:103CD00090931B0180931A0120914F023091500262
:103CE00080911A0190911B01280F391F37FF02C0E4
:103CF0002F5F3F4F359527953093500220934F0209
:103D000083E02FC11092540281E0809310018091D2
:103D100037029091380201969093380280933702CF
:103D2000809178009091790090931501809314010F
:103D30008091140190911501AA27BB27A0906402DD
:103D4000B0906502C0906602D0906702A80EB91EBE
:103D5000CA1EDB1EA0926402B0926502C092660287
:103D6000D0926702809168028F5F809368028231EF
:103D700008F4F6C08091160190911701A0911801E6
:103D8000B09119017C018D0123E0EE0CFF1C001F96
:103D9000111F2A95D1F7E81AF90A0A0B1B0BEA0C36
:103DA000FB1C0C1D1D1D80913B02992787FD9095E2
:103DB000A92FB92FBC01CD0126EC34E240E050E040
:103DC0000E942D78DC01CB01E81AF90A0A0B1B0BC3
:103DD000D801C7010496A11DB11DB7FF05C0D801C8
:103DE000C7010B96A11DB11D13E0B595A795979539
:103DF00087951A95D1F78093160190931701A09398
:103E00001801B093190180911206909113067C015C
:103E10000027F7FC0095102F809116019091170153
:103E2000A0911801B0911901E81AF90A0A0B1B0BAD
:103E3000E0921303F09214030093150310931603FA
:103E400020913C0230913D0240913E0250913F0250
:103E500057FF04C0215F3F4F4F4F5F4FF4E0559530
:103E6000479537952795FA95D1F780913C02909127
:103E70003D02A0913E02B0913F02821B930BA40B26
:103E8000B50B80933C0290933D02A0933E02B09309
:103E90003F0280913C0290913D02A0913E02B09180
:103EA0003F028E0D9F1DA01FB11F80933C02909377
:103EB0003D02A0933E02B0933F028091390290915F
:103EC0003A02AC01E5E0440F551FEA95E1F7481BC3
:103ED000590B80913C0290913D02A0913E02B0911D
:103EE0003F02B7FF03C00F96A11DB11D74E0B59549
:103EF000A795979587957A95D1F7209113033091DF
:103F00001403281B390B63E0220F331F6A95E1F776
:103F1000240F351F37FF02C0215E3F4F45E0359526
:103F200027954A95E1F730933A0220933902D6015A
:103F3000C501D7FE03C00196A11DB11DB595A7957A
:103F4000979587958093640290936502A09366028B
:103F5000B093670289E08093680202C01092540215
:103F600082E0809353028091530280937C00809181
:103F70005402882319F08FEC80937A00FF91EF911F
:103F8000BF91AF919F918F917F916F915F914F9171
:103F90003F912F911F910F91FF90EF90DF90CF9065
:103FA000BF90AF900F900FBE0F901F90189590E2AA
:103FB000E1E2F1E08FE49193815087FFFCCF089517
:103FC00090916B02E1E2F1E0E90FF11D80839F5FC8
:103FD00090936B020895EF92FF920F931F93CF93EC
:103FE000DF932091690220FF0AC080916A02882332
:103FF00011F0815002C08091200180936A0221FF5C
:104000000CC090916A0280912001981719F41092C7
:104010006A0203C09F5F90936A02822F992780FFF4
:1040200004C081FF02C010926A020E94D71F8091D3
:104030006A02282F332750EEE52E5FE1F52EC0915E
:104040002E04D0912F048A3098F481E180936B0282
:104050003F932F9380E694E09F938F93FF92EF928C
:10406000FE0109952DB73EB72A5F3F4F2DBF11C006
:1040700080E180936B023F932F9385E694E09F93BA
:104080008F93FF92EF92FE0109958DB79EB706962A
:104090008DBF20916A02822F9927AA27BB27FC0196
:1040A000429710F00C949C2AE05BFF4F40EEE42E08
:1040B0004FE1F42EC0912E04D0912F040C94F3788C
:1040C00010926B028AE694E09F938F9300EE1FE1BB
:1040D000FF92EF92FE01099584E180936B020F90AD
:1040E0000F900F900F9081E690E09F938F9382E561
:1040F00090E09F938F931F921F92809102016AE03C
:104100000E944C78892F99279F938F938091020169
:104110000E944C7899279F938F938AE794E09F930E
:104120008F93FF92EF92E0912E04F0912F04099566
:1041300088E280936B022DB73EB7225F3F4F2DBFC1
:1041400083E996E09F938F930E94A22D99279F93D6
:104150008F938FE894E09F938F93FF92EF92E0917B
:104160002E04F0912F0409958DB79EB708968DBF48
:1041700090914704992351F08CE380936B02892F2F
:1041800099279F938F938DE994E081C69091710256
:10419000992371F08CE380936B02892F99279F9369
:1041A0008F9384EB94E09F938F931F930F9391C011
:1041B0008091480484FF07C08CE380936B0289ECF4
:1041C00094E00C942E2A809192019091930106978D
:1041D00010F00C94A52A8CE380936B0286ED94E09A
:1041E0000C942E2A80912B0630EEE32E3FE1F32E25
:1041F000C0912E04D0912F0480FF74C010926B02E6
:104200008091130390911403A0911503B0911603AC
:10421000BC01CD0125E030E040E050E00E94A178F3
:104220003F932F9383EE94E09F938F93FF92EF92AF
:10423000FE01099584E180936B022DB73EB72A5F9A
:104240003F4F2DBF80910F0390911003A091110358
:10425000B0911203BC01CD0125E030E040E050E018
:104260000E94A1783F932F9380EF94E09F938F93C8
:10427000FF92EF92E0912E04F0912F04099588E2CD
:1042800080936B028DB79EB706968DBF8091140107
:10429000909115019F938F938DEF94E09F938F934F
:1042A000FF92EF92E0912E04F0912F0409958CE398
:1042B00080936B022DB73EB72A5F3F4F2DBF87B566
:1042C00099279F938F938AE095E09F938F93FF9216
:1042D000EF92E0912E04F0912F0409958DB79EB7CF
:1042E000069633C710926B0287E195E09F938F93F8
:1042F000FF92EF92FE01099584E180936B020F908B
:104300000F900F900F9086E295E09F938F93FF920E
:10431000EF92E0912E04F0912F04099588E28093AA
:104320006B020F900F900F900F908FE295E09F938C
:104330008F93FF92EF92E0912E04F0912F04099554
:104340008CE380936B020F900F900F900F908EE391
:1043500095E09F938F93FF92EF920C94322A1092E4
:104360006B0287E495E09F938F9300EE1FE1FF922D
:10437000EF92FE01099584E180936B020F900F90FC
:104380000F900F908091750390917603A091770321
:10439000B0917803B7FF04C081509C4FAF4FBF4F1F
:1043A0002AE0B595A795979587952A95D1F7BF935C
:1043B000AF939F938F9384E595E09F938F931F9383
:1043C0000F93E0912E04F0912F04099588E28093D9
:1043D0006B022DB73EB7285F3F4F2DBF80916D0315
:1043E00090916E03A0916F03B0917003B7FF04C06A
:1043F00081509C4FAF4FBF4FCAE0B595A795979599
:104400008795CA95D1F7BF93AF939F938F9383E618
:1044100095E09F938F931F930F93E0912E04F0915B
:104420002F0409958CE380936B028DB79EB7089695
:104430008DBF80913303909134039F938F9382E7D4
:1044400095E09F938F931F930F93E0912E04F0912B
:104450002F0409952DB73EB72A5F3F4F11C7109221
:104460006B0280914D0790914E079F938F9380919F
:104470004B0790914C079F938F9381E895E09F9312
:104480008F93FF92EF92FE01099584E180936B0276
:104490008DB79EB708968DBF8091510790915207B6
:1044A0009F938F9380914F07909150079F938F9385
:1044B00081E995E09F938F93FF92EF92E0912E0414
:1044C000F0912F04099588E280936B022DB73EB7D7
:1044D000285F3F4F2DBF80915507909156079F93BE
:1044E0008F9380915307909154079F938F9381EA04
:1044F00095E09F938F93FF92EF92E0912E04F091BD
:104500002F0409958CE380936B028DB79EB70896B4
:104510008DBF8091590790915A079F938F938091F7
:104520005707909158079F938F9381EB95E0A2C016
:1045300010926B0280912006E82FFF27EE0FFF1FDD
:10454000E75BF84F808191819F938F9380911F0645
:10455000E82FFF27EE0FFF1FE75BF84F8081918167
:104560009F938F9381EC95E09F938F93FF92EF92AF
:10457000FE01099584E180936B028DB79EB7089682
:104580008DBF80912206E82FFF27EE0FFF1FE75B0C
:10459000F84F808191819F938F9380912106E82F1E
:1045A000FF27EE0FFF1FE75BF84F8081918188584E
:1045B0009F4F9F938F9381ED95E09F938F93FF92F1
:1045C000EF92E0912E04F0912F04099588E28093F8
:1045D0006B022DB73EB7285F3F4F2DBF8091240659
:1045E000E82FFF27EE0FFF1FE75BF84F80819181D7
:1045F00082599F4F9F938F9380912306E82FFF2727
:10460000EE0FFF1FE75BF84F8081918182599F4F2A
:104610009F938F9381EE95E09F938F93FF92EF92FC
:10462000E0912E04F0912F0409958CE380936B02A6
:104630008DB79EB708968DBF80912606E82FFF277D
:10464000EE0FFF1FE75BF84F8081918182599F4FEA
:104650009F938F9380912506E82FFF27EE0FFF1F72
:10466000E75BF84F8081918182599F4F9F938F9391
:1046700081EF95E09F938F93FF92EF92E0912E044C
:10468000F0912F0409952DB73EB7285F3F4FF8C52D
:1046900010926B0281E096E09F938F9300EE1FE1F2
:1046A000FF92EF92FE010995809102010F900F9009
:1046B0000F900F908A3009F09DC084E180936B02C7
:1046C00080918A0390918B039C0197FF02C0295F20
:1046D0003F4F287F821B930B9F938F9380918A0378
:1046E00090918B0397FD0796A3E095958795AA95E2
:1046F000E1F79F938F9320918A0330918B0337FFCB
:1047000002C0295F3F4FF3E035952795FA95E1F711
:1047100080914B0290914C02821B930B9F938F933D
:104720008FE096E09F938F931F930F93E0912E0459
:10473000F0912F04099588E280936B028DB79EB7A4
:104740000A968DBF80918803909189039C0197FF01
:1047500002C0295F3F4F287F821B930B9F938F934B
:10476000809188039091890397FD0796E3E09595E2
:104770008795EA95E1F79F938F9320918803309175
:10478000890337FF02C0295F3F4F73E035952795B6
:104790007A95E1F78091490290914A02821B930B2E
:1047A0009F938F9380E296E09F938F931F930F9335
:1047B000E0912E04F0912F0409958CE380936B0215
:1047C0002DB73EB7265F3F4F2DBF80918603909156
:1047D00087039F938F938091860390918703209105
:1047E000470230914802821B930B9F938F9381E382
:1047F00096E0A7C38B3019F0843108F4ADC084E192
:1048000080936B0280918A0390918B039C0197FFA8
:1048100002C0215F3F4F207F821B930B97FD0196C3
:10482000959587959F938F9380918A0390918B03A1
:1048300097FD0F9654E0959587955A95E1F79F93CC
:104840008F9320918A0330918B0337FF02C0295F39
:104850003F4F43E0359527954A95E1F780914B020C
:1048600090914C02821B930B9F938F938FE396E062
:104870009F938F931F930F93E0912E04F0912F0439
:10488000099588E280936B022DB73EB7265F3F4FB4
:104890002DBF80918803909189039C0197FF02C0EE
:1048A000215F3F4F207F821B930B97FD01969595CB
:1048B00087959F938F93809188039091890397FDAB
:1048C0000F96C4E095958795CA95E1F79F938F93CE
:1048D000209188033091890337FF02C0295F3F4F41
:1048E000B3E035952795BA95E1F78091490290910B
:1048F0004A02821B930B9F938F9381E596E09F93CF
:104900008F931F930F93E0912E04F0912F0409953C
:104910008CE380936B028DB79EB70A968DBF809112
:1049200086039091870397FD0196959587959F93B0
:104930008F93809186039091870320914702309155
:104940004802821B930B9F938F9383E696E09F937D
:104950008F931F930F9392CE8D3009F0F6C584E1AB
:1049600080936B028091130199279F938F9380917D
:104970008A0390918B0397FD0F96F4E095958795A8
:10498000FA95E1F79F938F9320918A0330918B03DF
:1049900037FF02C0295F3F4FE3E035952795EA9541
:1049A000E1F780914B0290914C02821B930B9F93F5
:1049B0008F9382E796E09F938F931F930F93E091DD
:1049C0002E04F0912F04099588E280936B028DB735
:1049D0009EB70A968DBF8091120199279F938F935E
:1049E000809188039091890397FD0F9674E09595C7
:1049F00087957A95E1F79F938F9320918803309163
:104A0000890337FF02C0295F3F4F63E03595279543
:104A10006A95E1F78091490290914A02821B930BBB
:104A20009F938F9386E896E09F938F931F930F93A6
:104A3000E0912E04F0912F0409958CE380936B0292
:104A40002DB73EB7265F3F4F2DBF809111019927AB
:104A50009F938F93809186039091870397FD019692
:104A6000959587959F938F93809186039091870367
:104A70002091470230914802821B930B9F938F93A2
:104A80008AE996E09F938F931F930F93E0912E04F2
:104A9000F0912F0409958DB79EB70A9656C31092D0
:104AA0006B028EEA96E09F938F93FF92EF92FE0146
:104AB000099584E180936B020F900F900F900F90F7
:104AC00080918003909181039F938F938091430203
:104AD000909144029F938F938BEB96E09F938F93DB
:104AE000FF92EF92E0912E04F0912F04099588E255
:104AF00080936B022DB73EB7285F3F4F2DBF80914B
:104B00007E0390917F039F938F93809145029091B4
:104B100046029F938F938AEC96E09F938F93FF9228
:104B2000EF92E0912E04F0912F0409958CE380938D
:104B30006B028DB79EB708968DBF80917A039091D6
:104B40007B039F938F9380914102909142029F93A8
:104B50008F9389ED96E08ECD10926B0280911E01AD
:104B600090911F016AE070E00E946C789F938F9390
:104B700080911E0190911F016AE070E00E946C78A4
:104B80007F936F9388EE96E09F938F93FF92EF92BF
:104B9000FE01099584E180936B028DB79EB708965C
:104BA0008DBF80919108909192086AE070E00E9418
:104BB00058789F938F9380919108909192086AE022
:104BC00070E00E9458787F936F938CEF96E09F93EC
:104BD0008F93FF92EF92E0912E04F0912F040995AC
:104BE00088E280936B022DB73EB7285F3F4F2DBF01
:104BF00080919308909194089F938F9380E197E020
:104C00009F938F93FF92EF92E0912E04F0912F04E7
:104C100009958CE380936B028DB79EB706968DBF86
:104C200080919508909196089F938F9380E297E0EA
:104C30002EC110926B0282E397E09F938F93FF92B5
:104C4000EF92FE01099584E180936B020F900F9023
:104C50000F900F908091490790914A079F938F93EF
:104C60008BE397E09F938F93FF92EF92E0912E0456
:104C7000F0912F04099588E280936B028DB79EB75F
:104C800006968DBF8091210399279F938F938BE484
:104C900097E09F938F93FF92EF92E0912E04F09113
:104CA0002F0409958CE380936B022DB73EB72A5FE2
:104CB0003F4F2DBF80914807992701979F938F936E
:104CC0008BE597E002CB10926B028BE697E09F9307
:104CD0008F93FF92EF92FE01099584E180936B021E
:104CE0000F900F900F900F9080912F0390913003B1
:104CF0009F938F9383E797E09F938F93FF92EF9219
:104D0000E0912E04F0912F04099588E280936B02C4
:104D10002DB73EB72A5F3F4F2DBF8091330390914F
:104D200034039F938F9381E897E09F938F93FF9233
:104D3000EF92E0912E04F0912F0409958CE380937B
:104D40006B028DB79EB706968DBF8091310390910F
:104D500032039F938F938FE897E099C010926B0274
:104D60008091220399279F938F938DE997E09F93DA
:104D70008F93FF92EF92FE01099584E180936B027D
:104D80008DB79EB706968DBF8091230399279F9379
:104D90008F9389EA97E09F938F93FF92EF92E09130
:104DA0002E04F0912F04099588E280936B022DB7B1
:104DB0003EB72A5F3F4F2DBF8091240399279F93D1
:104DC0008F9385EB97E09F938F93FF92EF92E09103
:104DD0002E04F0912F0409958CE380936B028DB71C
:104DE0009EB706968DBF8091250399279F938F9339
:104DF00081EC97E04CC010926B02809126039927BA
:104E00009F938F938DEC97E09F938F93FF92EF92F8
:104E1000FE01099584E180936B028DB79EB70696DB
:104E20008DBF8091270399279F938F9389ED97E0FA
:104E30009F938F93FF92EF92E0912E04F0912F04B5
:104E4000099588E280936B022DB73EB72A5F3F4FEA
:104E50002DBF8091280399279F938F9385EE97E02C
:104E60009F938F93FF92EF92E0912E04F0912F0485
:104E700009958CE380936B028DB79EB706968DBF24
:104E80008091290399279F938F9381EF97E09F93B8
:104E90008F93FF92EF92D9CA10926B028DEF97E039
:104EA0009F938F9300EE1FE1FF92EF92FE01099511
:104EB00084E180936B020F900F900F900F90809180
:104EC000C50199279F938F9385E098E09F938F93D7
:104ED000FF92EF92E0912E04F0912F04099588E261
:104EE00080936B028DB79EB706968DBF809122028C
:104EF0009091230297FD03969595879595958795B3
:104F00009F938F9383E198E09F938F931F930F93C9
:104F1000E0912E04F0912F0409958CE380936B02AD
:104F20002DB73EB72A5F3F4F2DBF80914E06992780
:104F30009F938F9380914D0699279F938F9381E242
:104F400098E09F938F931F930F93E0912E04F0911D
:104F50002F0409958DB79EB70896F7C010926B0283
:104F60008FE298E09F938F93FF92EF92FE01099555
:104F700084E180936B020F900F900F900F908091BF
:104F80006804992787FD90959F938F93809167047C
:104F9000992787FD90959F938F938FE398E09F9338
:104FA0008F93FF92EF92E0912E04F0912F040995D8
:104FB00088E280936B022DB73EB7285F3F4F2DBF2D
:104FC00080916904992787FD90959F938F93809195
:104FD0006A0499279F938F938FE498E09F938F9310
:104FE000FF92EF92E0912E04F0912F0409958CE34B
:104FF00080936B028DB79EB708968DBF80916E042B
:1050000099279F938F9380916B04992787FD9095A3
:105010009F938F938FE598E02DCB10926B028FE6D4
:1050200098E09F938F93FF92EF92FE01099584E1A0
:1050300080936B020F900F900F900F908091030759
:1050400099278F7790709F938F938091FB06992774
:105050008F7790709F938F938091F30699278F7726
:1050600090709F938F938091EB0699278F77907024
:105070009F938F938FE798E09F938F93FF92EF9288
:10508000E0912E04F0912F04099588E280936B0241
:105090008DB79EB70C968DBF8091230799278F7788
:1050A00090709F938F9380911B0799278F779070B3
:1050B0009F938F938091130799278F7790709F9379
:1050C0008F9380910B0799278F7790709F938F9381
:1050D00080E998E09F938F93FF92EF92E0912E04E6
:1050E000F0912F0409958CE380936B022DB73EB7A6
:1050F000245F3F4F2DBF8091430799278F77907092
:105100009F938F9380913B0799278F7790709F9300
:105110008F938091330799278F7790709F938F9308
:1051200080912B0799278F7790709F938F9381EAB7
:1051300098E09F938F93FF92EF92E0912E04F0916D
:105140002F0409958DB79EB70C968DBFFEC11092A6
:105150006B0282EB98E09F938F93FF92EF92FE0198
:10516000099584E180936B020F900F900F900F9040
:1051700080910707992787FD90959F938F93809142
:10518000FF06992787FD90959F938F938091F7064F
:10519000992787FD90959F938F938091EF0699278C
:1051A00087FD90959F938F9381EC98E09F938F93C9
:1051B000FF92EF92E0912E04F0912F04099588E27E
:1051C00080936B022DB73EB7245F3F4F2DBF809178
:1051D0002707992787FD90959F938F9380911F07AD
:1051E000992787FD90959F938F9380911707992713
:1051F00087FD90959F938F9380910F07992787FD47
:1052000090959F938F9382ED98E09F938F93FF9259
:10521000EF92E0912E04F0912F0409958CE3809396
:105220006B028DB79EB70C968DBF8091470799276B
:1052300087FD90959F938F9380913F07992787FDD6
:1052400090959F938F9380913707992787FD90952D
:105250009F938F9380912F07992787FD90959F9318
:105260008F9383EE98E09F938F93FF92EF92E0915C
:105270002E04F0912F0409952DB73EB7245F3F4FC0
:105280002DBF63C110926B0284EF98E09F938F93C0
:1052900000EE1FE1FF92EF92FE01099584E18093F9
:1052A0006B020F900F900F900F9080910307881F53
:1052B0008827881F97E0899FC00111248D969F93AE
:1052C0008F938091FB06881F8827881F96E0899F0F
:1052D000C00111248D969F938F938091F306881FB0
:1052E0008827881F95E0899FC00111248D969F9380
:1052F0008F938091EB06881F8827881F9927880F36
:10530000991F880F991F8D969F938F9383E099E043
:105310009F938F93FF92EF92E0912E04F0912F04D0
:10532000099588E280936B028DB79EB70C968DBF6E
:1053300080912307881F8827881F9BE0899FC001D1
:1053400011248D969F938F9380911B07881F882728
:10535000881F9AE0899FC00111248D969F938F9397
:1053600080911307881F8827881F99E0899FC001B3
:1053700011248D969F938F9380910B07881F882708
:10538000881F992723E0880F991F2A95E1F78D96AA
:105390009F938F9387E199E09F938F93FF92EF9272
:1053A000E0912E04F0912F0409958CE380936B0219
:1053B0002DB73EB7245F3F4F2DBF80912B07881F2D
:1053C0008827881F9CE0899FC00111248D969F9398
:1053D0008F938BE299E09F938F93FF92EF92E091EE
:1053E0002E04F0912F040995809133072DB73EB715
:1053F0002A5F3F4F2DBF87FF12C080E480936B026E
:105400008CE399E09F938F93FF92EF92E0912E04AB
:10541000F0912F0409950F900F900F900F908091AD
:105420003B0787FF12C084E480936B028FE399E00F
:105430009F938F931F930F93E0912E04F0912F046D
:1054400009950F900F900F900F908091430787FF61
:105450007CC088E480936B0282E499E09F938F93F1
:105460001F930F93E0912E04F0912F0409950F9054
:105470000F900F900F9069C010926B0285E499E035
:105480009F938F93FF92EF92FE01099584E18093A1
:105490006B020F900F900F900F908091F9019091F7
:1054A000FA019F938F9383E599E09F938F93FF92E7
:1054B000EF92E0912E04F0912F04099588E28093F9
:1054C0006B028DB79EB706968DBF8091FB019091C0
:1054D000FC019F938F9380E699E09F938F93FF92B7
:1054E000EF92E0912E04F0912F04099589E48093C6
:1054F0006B022DB73EB72A5F3F4F2DBF8DE699E077
:105500009F938F93FF92EF92E0912E04F0912F04DE
:105510000995809169020F900F900F900F9083FF73
:1055200014C01092FC011092FB0160E070E08EE06C
:1055300090E00E94902C09C080912001281719F456
:1055400021502093200110926A0210926902E6E035
:10555000CDB7DEB70C94E4784AEA20E030E02617B5
:10556000370740F4FC018191480F2F5F3F4F26170A
:105570003707C8F3842F99270895AC019AEA20E0F1
:1055800030E02617370750F4DA01A20FB31F0E944C
:10559000F978802D980F2F5F3F4FF3CF892F9927F0
:1055A000089581E08093210682E08093200683E0C5
:1055B00080931F0684E08093220685E08093230673
:1055C00086E08093240687E08093250688E0809318
:1055D000260689E0809327068AE0809328068BE0E0
:1055E000809329068CE080932A06089595E5909390
:1055F0001E0680910201843170F08AE080933E069D
:10560000109262068BE180933A068EE480935F06E7
:10561000809360060DC083E080933E0680E2809315
:1056200062068EE180933A0690935F06909360063F
:105630008AE680932B0683E08093840681E0809342
:1056400045061092810610927E0668E06093380647
:1056500086EE8093390680E880933B065EE15093A6
:105660002C068FEF80932E069FE090932F06509389
:105670002D06109231066093320680E48093330643
:105680001092340690933006109247061092480606
:105690001092490610924A0610926406109265060E
:1056A000109266061092670638E730934B0648E280
:1056B00040934C0672E07093830690934D0627EF5B
:1056C00020934E0685E0809353068DE7809356061F
:1056D000809357068093580630934F069AE590932F
:1056E0005006109251062093520640935406109291
:1056F00055068FE58093680683EF80936A068AEAF1
:1057000080936C0680936D0684E180936906809394
:105710006B0682E38093590690935A0680935B064A
:10572000109282068EEF80936E0624E620936F0619
:105730009093700690937106909372068BE4809319
:10574000730680937406809375061092760686E041
:1057500080937706609378069093790650937A0643
:1057600020937B0620937C0670937D0610927F0623
:105770001092800681E2809342068DE28093430678
:10578000909344060895CF93DF930E94F62A8EE00B
:105790008093350620E1209336063CE030933706AF
:1057A00090E590933C0686E980933D0690933F06F2
:1057B0008093400686E08093410680E2809346060F
:1057C0008AE580935C0690935D0681E080935E0697
:1057D0002093610684E680936306A5E8B6E0E1E7DE
:1057E000F1E0ED01019009923A95E1F763E770E08D
:1057F000CD01875690400E94AC2A80939106DF919C
:10580000CF910895CF93DF930E94F62A8AE0809388
:10581000350680E18093360626E0209337069AE528
:1058200090933C0688E780933D0690933F068093D3
:1058300040062093410620E22093460690935C06A2
:1058400080E580935D068CE380935E06209361067D
:105850008BE480936306A5E8B6E08CE0E8E7F1E02E
:10586000ED01019009928A95E1F763E770E0CD01BF
:10587000875690400E94AC2A80939106DF91CF9189
:105880000895CF93DF930E94F62A88E0809335062F
:1058900030E13093360626E02093370694E6909365
:1058A0003C0688E780933D0690933F068093400630
:1058B00020934106309346068AE580935C0680E596
:1058C00080935D0696E490935E0680E28093610685
:1058D00090936306A5E8B6E08CE0E0E8F1E0ED0126
:1058E000019009928A95E1F763E770E0CD01875650
:1058F00090400E94AC2A80939106DF91CF91089549
:10590000DC010E94F978802D99270895DC01062E8C
:105910000E940B790895DC010E940679CF01089559
:10592000DC010B010E9417790895FF920F931F93DA
:10593000CF93DF93982F8150853008F093E084E770
:10594000F82E9F9D80011124E801609763E770E0C5
:10595000CE010E94BD2A982FD801AD59BF4F0E9499
:10596000F978802D891731F4DE010E94F978802DB5
:10597000853519F080E090E00AC0EEE1F6E0DE0146
:105980001F2C0E9401790E94556781E090E0E5E0BC
:10599000CDB7DEB70C94E578863010F085E003C013
:1059A000882309F481E0A2E0B0E0082E0E940B7980
:1059B00008951F93CF93DF93182FCEE1D6E0809107
:1059C0001E06853591F5163010F015E002C0112342
:1059D00061F163E770E08EE196E00E94AC2A80936B
:1059E000910684E7189FD00111245097FE01182ECC
:1059F0000E941C79EFE1F6E0A0E5B0E02CE030E099
:105A0000122E0E941C79B9018FE196E00E94AC2A07
:105A1000ACE5B0E0082E0E940B79812F0E94CC2CBF
:105A20000E94556781E090E002C080E090E0DF9145
:105A3000CF911F9108956DE470E088EE93E00E948D
:105A4000BD2AA5E3B4E00E94F978902D981739F4A7
:105A5000A8EEB3E00E94F978802D813019F080E043
:105A600090E00895E2E9F6E0A8EEB3E08EE4182EA7
:105A70000E94017981E090E00895CF93DF93C2E91D
:105A8000D6E080919206813089F46DE470E0CE0119
:105A90000E94AC2A8093DF06A8EEB3E08EE4FE01FC
:105AA000182E0E941C7981E090E002C080E090E016
:105AB000DF91CF910895CF93DF9381E08093920699
:105AC000E2E9F6E08FE0158616861786108A815087
:105AD000349687FFF8CF80E480939F068093A006DA
:105AE0001092A1068093A2068093A30690EC909357
:105AF000A4061092A5068093A6068093A70610928E
:105B0000A8069093A9069093AA068093AB061092DC
:105B1000AC068093AD069093AE06A3E9B6E087E0AD
:105B2000EAE8F1E0ED01019009928A95E1F76DE470
:105B300070E0CD0101970E94AC2A8093DF06DF91CF
:105B4000CF910895A2E0B0E00E94F978802D8630D0
:105B500030F083E0A2E0B0E0082E0E940B79992794
:105B600008951F93CF93C82F162F863010F0C5E0ED
:105B700003C0882309F4C1E08C2F99278230910556
:105B800041F08330910544F4019731F40E94C32B16
:105B900005C00E94022C02C00E94412C1123B1F0CA
:105BA0006CE070E080E590E00E94BD2AACE5B0E0DA
:105BB0000E94F978902D981749F4EFE1F6E0A0E5FE
:105BC000B0E08CE0182E0E94017902C00E94D12A18
:105BD0008C2F0E94D92CCF911F910895DF92EF92C4
:105BE000FF920F931F93CF93FF24DF2CEF2C81E0C4
:105BF00090E00E94802C853539F031E0E32E65E598
:105C000081E090E00E94862C6CE070E080E590E0FE
:105C10000E94BD2AC82FACE5B0E00E94F978802D23
:105C20008C1711F421E0D22EC1E001E010E0EE204B
:105C300029F48C2F0E94952C8823B1F591E0F92E40
:105C40001F930F9385E799E09F938F9384EF92E1E1
:105C50009F938F93E0912E04F0912F0409958DB7B7
:105C60009EB706968DBF0230110549F0033011052D
:105C70004CF40130110531F40E94C32B05C00E9481
:105C8000022C02C00E94412CDD2049F0EFE1F6E039
:105C9000A0E5B0E08CE0182E0E94017902C00E94BD
:105CA000D12A8C2F0E94D92CCF5F0F5F1F4FC63097
:105CB00008F4BDCFFF2019F083E00E94CC2C0E9495
:105CC000A22DC82F0E94952C8C2F99279F938F93DC
:105CD0008BE999E09F938F9304EF12E11F930F9349
:105CE000E0912E04F0912F0409958DB79EB706968A
:105CF0008DBFEE2021F40E941B2D882399F484EBA4
:105D000099E09F938F931F930F93E0912E04F0914E
:105D10002F0409950E945B2D0E943D2D0F900F903E
:105D20000F900F9010921D0690E0EFE9F6E0CFE0A3
:105D30008081349618160CF49F5FC150C7FFF8CFCE
:105D400090931D06892F99279F938F9383E996E05F
:105D50009F938F9385ED99E09F938F931F930F935C
:105D6000E0912E04F0912F0409958DB79EB7089607
:105D70008DBF86EF99E09F938F931F930F93E091D0
:105D80002E04F0912F0409950F900F900F900F9013
:105D9000CF911F910F91FF90EF90DF900895982F72
:105DA0002FB7F8943998389A88B1836088B9809170
:105DB000B9008C7F8093B9008AE28093B80010927A
:105DC00076021092740210927302992379F0E8EE31
:105DD000F6E08BE010821182128213821482158207
:105DE000168217828150389687FFF4CF78942FBFA0
:105DF00008951092760284E98093BC0080E8809335
:105E0000BC001092BD001092BA001092BB0010921C
:105E1000B9001092B8001092720280E00E94CF2E5A
:105E20001092BB0085E88093BC0080917002826074
:105E30008093700208951F920F920FB60F92112453
:105E40002F933F934F935F938F939F93EF93FF9382
:105E500080917602282F3327442755278F5F809320
:105E60007602F9012731310508F0C2C2EE59FF4F21
:105E70000C94F37881E08093720209C080917402DF
:105E80008C3090F4809174028F5F809374028091C3
:105E90007402E82FFF27EE0FFF1FEE0FFF1FEE56D5
:105EA000F94F8585181654F7809174028C3070F084
:105EB00010926F0210926E021092740285E080932D
:105EC000760280917302880F8D5A04C0809174020B
:105ED000880F8E5A8093BB0085E87FC28091740240
:105EE000E82FFF2783E0EE0FFF1F8A95E1F7E851C7
:105EF000F94F81818093BB0085E88093BC0080913D
:105F00007402E82FFF27EE0FFF1FEE0FFF1FEE0FAB
:105F1000FF1FE851F94F808180FF91C0809174028A
:105F2000E82FFF27EE0FFF1FEE0FFF1FEE0FFF1FE3
:105F3000E851F94F8281882329F080911D0687302E
:105F400008F46CC280916E0290916F02892B09F067
:105F500065C280916C0290916D02892B09F05EC23E
:105F60006EC08091740221E030E002C0220F331F26
:105F70008A95E2F780916C0290916D022823392373
:105F8000232B79F080917402E82FFF27EE0FFF1F7B
:105F9000EE0FFF1FEE0FFF1FE851F94F80E18483E2
:105FA0000DC080917402E82FFF27EE0FFF1FEE0F48
:105FB000FF1FEE0FFF1FE851F94F1482809174020A
:105FC000E82FFF2753E0EE0FFF1F5A95E1F7E85146
:105FD000F94F8481282F332743E0220F331F4A953E
:105FE000E1F780917402E82FFF2793E0EE0FFF1F87
:105FF0009A95E1F7E851F94F82818770822B80935F
:10600000BB0085E88093BC002091740281E090E0A1
:1060100002C0880F991F2A95E2F720916E023091F5
:106020006F0282239323892B51F080EE96E09093A8
:106030007A028093790288E080937B02EFC184E04A
:1060400089C1E0917902F0917A0281918093BB003D
:1060500085E88093BC00F0937A02E0937902809106
:106060007B02815080937B02882309F4D7C183E0AF
:1060700071C18091B900803351F5809177028823F6
:1060800029F4809174028F5F80937702809174026B
:10609000E82FFF2783E0EE0FFF1F8A95E1F7E85115
:1060A000F94F838199278F7790708F3791057CF412
:1060B00080917402E82FFF27EE0FFF1FEE0FFF1FE6
:1060C000EE0FFF1FE851F94F83818F5F838310929A
:1060D000760284E98093BC008AE090E0909393017B
:1060E00080939201809174028F5F8093740210926A
:1060F00076026DC18091B9008034C9F1809173023C
:10610000E82FFF27EE0FFF1FEE0FFF1FEE0FFF1F01
:10611000E851F94F83818F778383809173028F5F7A
:1061200080937302809173028C30A0F010927302FE
:1061300010926D0210926C02809178028F5F8093B2
:1061400078028C3038F010927802809170028D7F46
:10615000809370028091700281608093700210922F
:10616000760284E98093BC001092720273C0809121
:106170007302E82FFF27EE0FFF1FEE0FFF1FEE0F3A
:10618000FF1FE851F94F83818068838380917302F8
:10619000E82FFF27EE0FFF1FEE0FFF1FEE0FFF1F71
:1061A000E851F94F808180FF2FC080917302E82F62
:1061B000FF2753E0EE0FFF1F5A95E1F7E851F94F23
:1061C00084819927009751F04097D9F580EE96E0A9
:1061D00090937A028093790288E031C080917302B3
:1061E000992743E0880F991F4A95E1F78351994F0A
:1061F00090937A0280937902909173028091780251
:106200009817E1F483E01BC080917302992733E073
:10621000880F991F3A95E1F78351994F90937A022D
:10622000809379028091700281FD06C09091730283
:1062300080917802981711F482E001C081E0809388
:106240007B0280917B02813011F485E801C085ECEE
:106250008093BC0080917702809371021092770244
:10626000DDC0E0917902F0917A028091BB008083D9
:106270008091790290917A02019690937A028093AC
:10628000790280917B02815080937B02823010F0F2
:1062900085EC5DC0813011F485E859C080917002B1
:1062A00081FF2DC08091ED0280FD1DC080917302A1
:1062B000E82FFF2723E0EE0FFF1F2A95E1F7E851B3
:1062C000F94F86818A3F79F480917302E82FFF2786
:1062D00093E0EE0FFF1F9A95E1F7E851F94F8081A7
:1062E000816080830CC080917302E82FFF2783E0D8
:1062F000EE0FFF1F8A95E1F7E851F94F1082809168
:1063000073028F5F80937302809173028C30A0F0D0
:106310001092730210926D0210926C0280917802BA
:106320008F5F809378028C3038F0109278028091E1
:1063300070028D7F809370021092760284E98093C0
:10634000BC008091700281608093700265C0809370
:10635000BC0086E08093760261C088E9BBCD809165
:106360007502880F805FB6CD8091750299278130C4
:10637000910561F0823091051CF4892B21F04EC00B
:10638000029739F04BC080911301A4CD8091120186
:10639000A1CD809111019ECD80E89CCD1092760216
:1063A00084E98093BC00109272028AE090E090939E
:1063B00093018093920180917502823088F48091DC
:1063C00075028F5F8093750282E1809376028091DF
:1063D00070028E7F8093700285EA8093BC001EC09D
:1063E000109275028091700281608093700216C0D5
:1063F0001092760284E98093BC00809170028160E3
:10640000809370028AE090E09093930180939201D0
:10641000109274021092730210927202FF91EF9127
:106420009F918F915F914F913F912F910F900FBE50
:106430000F901F9018951F93CF93DF93182F809183
:106440001803882321F480910702882319F081E042
:1064500090E097C01D3008F092C01123B1F0E12FF9
:10646000FF2723E0EE0FFF1F2A95E1F7E851F94FD0
:1064700035978081359688230CF081C038978081CC
:1064800080FD03C083E090E07CC08091E006823014
:1064900019F084E090E075C067E070E080EE96E06F
:1064A0000E94AC2A9091E706891719F085E090E0E8
:1064B00068C080ED97E00E941A17EC01809170028D
:1064C00080FD05C0CE010E9423178823B9F3112354
:1064D00019F48FEF90E00BC0212F3327215030406B
:1064E00081E090E002C0880F991F2A95E2F790930F
:1064F0006F0280936E02A1E0B0E0E8EEF6E040E0CB
:1065000050E06BE0CD01042E02C0880F991F0A9461
:10651000E2F720916E0230916F0282239323892B40
:1065200011F01182128261504F5F5F4F389667FF02
:10653000E9CF1092740210927602809170028E7FE1
:106540008093700285EA8093BC008091700280FD88
:1065500005C0CE010E9423178823B9F380916E02F3
:1065600090916F02892B29F0CE010E942317882376
:1065700011F380916E0290916F02009711F082E00A
:1065800090E0DF91CF911F9108950F931F93CF93C8
:10659000DF93982F80911803882321F480910702BC
:1065A000882319F081E090E092C09D30A0F49923F7
:1065B00019F486E090E08BC0C92FDD27FE0133E09F
:1065C000EE0FFF1F3A95E1F7E851F94F35978081BB
:1065D000359687FD03C082E090E079C038978081CE
:1065E00080FD03C083E090E072C080ED97E00E94E0
:1065F0001A178C018091700280FD05C0C8010E94AD
:1066000023178823B9F3219721E030E0C90102C0A4
:10661000880F991FCA95E2F790936D0280936C02E0
:10662000D901E8EEF6E040E050E06BE0CD01042E49
:1066300002C0880F991F0A94E2F720916C023091F2
:106640006D0282239323892B11F0118212826150F3
:106650004F5F5F4F389667FFE9CF10927302109239
:10666000E0061092E70610927602809170028E7F0B
:106670008093700285EA8093BC008091700280FD57
:1066800005C0C8010E9423178823B9F380916C02CA
:1066900090916D02892B29F0C8010E94231788234D
:1066A00011F38091E006823019F084E090E00FC091
:1066B00067E070E080EE96E00E94AC2A9091E706D9
:1066C000891719F085E090E002C080E090E0DF914A
:1066D000CF911F910F91089589E1ADE7B7E0E9E40B
:1066E000F7E011821082329611961C921E92129639
:1066F000815087FFF6CF1092870310928603109285
:1067000089031092880310928B0310928A030895D4
:106710001F920F920FB60F9211240F931F932F9376
:106720003F934F935F936F937F938F939F93AF9319
:10673000BF93CF93DF93EF93FF938091840682FD05
:10674000CFC0409186005091870080917D0290914A
:106750007E02481B590B8091860090918700909390
:106760007E0280937D02CA018D549440A0917F02E5
:10677000B0918002835F9A4178F480917F02809388
:106780004807149714F01092940181E090E09093E0
:10679000800280937F0207C2AD30B1050CF003C2C6
:1067A000CA018B5F9040845B914008F074C0425DE9
:1067B0005140FD01EA0FFB1FE75BF84F808191819B
:1067C000FA01E81BF90BCF01F7FF03C09095819503
:1067D0009F4F06975CF480912103883C20F48091C0
:1067E0002103865F01C088EC80932103FD01EA0F3D
:1067F000FB1FE75BF84F808191819C01220F331FC3
:10680000280F391F240F351F37FF02C02D5F3F4F60
:10681000E901D595C795D595C795CA0101968C17FD
:106820009D0714F4219706C041505040C417D50766
:106830000CF4219680912103833CE0F08D010A0F36
:106840001B1FF801E75BF84F808191819E01281B97
:10685000390BC90163E070E00E946C78CB01880FAE
:10686000991F860F971F0358184FD80111969C93B4
:106870008E9307C0AA0FBB1FA358B84F11961C9246
:106880001E92E0917F02F0918002EE0FFF1FE75B06
:10689000F84FD183C08320917F02309180022F5F17
:1068A0003F4F3093800220937F0280910201843118
:1068B00008F079C12530310511F45D9A01C05D9869
:1068C00080917F02909180028630910511F45C9A4C
:1068D00001C05C98079711F45B9A65C15B9863C12E
:1068E00040918600509187008091810290918202B0
:1068F000481B590B809186009091870090938202EB
:1069000080938102CA018D5494406091EB02835FB1
:106910009A4108F07AC060937C0280917C028430B6
:1069200008F453C09091480780917C02981709F0B1
:106930004CC05091EC025B3008F43FC010929401BF
:106940001092EB0240E05F31C0F0E42FFF27EE0F22
:10695000FF1F9F0129543D4FDF01A75BB84F8D9169
:106960009C91D9018D939C93DF01A358B84F8D91D1
:106970009C91EF52FD4F91838083E42FFF27EE0F10
:10698000FF1F9F01275B384FDF01AD57BD4F8D9132
:106990009C91D90111969C938E93DF01A356BD4F14
:1069A0008D919C91E358F84F91838083842F8F5F62
:1069B000482F8D3040F28093EB028091EC028F3FA4
:1069C000B9F08F5F8093EC0213C08091EC028536A2
:1069D00020F08AE08093EC0202C01092EC028091D9
:1069E00002018A3011F0843110F0289A01C02898F1
:1069F00081E08093EB0280911803882309F0D3C0D3
:106A000080917C0280934807CEC06D3008F0A3C00F
:106A1000CA018B5F9040845B914008F07EC0425D6C
:106A20005140E62FFF27EE0FFF1FED57FD4F8081EE
:106A30009181FA01E81BF90BCF0105960B97B0F491
:106A40008091EC028A3120F080912103865F05C09D
:106A50008B3028F0809121038E5F809321038091F9
:106A60002103893C18F088EC80932103E62FFF274F
:106A7000EE0FFF1FED57FD4F808191819C01220F8A
:106A8000331F280F391F240F351F37FF02C02D5F1A
:106A90003F4FE901D595C795D595C795CA01019690
:106AA0008C179D0714F4219706C041505040C4171D
:106AB000D5070CF42196809121038E3BD8F0E62F68
:106AC000FF27EE0FFF1FDF01AD57BD4F8D919C914A
:106AD0009E01281B390BC90163E070E00E946C78AD
:106AE000CB01880F991F860F971FE356FD4F9183A7
:106AF000808308C0E62FFF27EE0FFF1FE356FD4FF0
:106B0000118210828091EB02E82FFF27EE0FFF1F0A
:106B1000ED57FD4FD183C08309C0809102018A30B7
:106B200011F0843110F0289A01C028988091020158
:106B3000843188F48091EB02853011F45D9A05C0B0
:106B40005D98863011F45C9A05C05C98873011F42A
:106B50005B9A01C05B988091EB02843120F48F5FD7
:106B60008093EB0220C08431F1F4809102018A30DD
:106B700011F0843110F0289A01C028988EE180939A
:106B8000EB022CE0CDE7D7E0A7EBB2E0E9E4F7E0D9
:106B90008D919D91918380833296198218822296DD
:106BA000215027FFF5CFFF91EF91DF91CF91BF915A
:106BB000AF919F918F917F916F915F914F913F9195
:106BC0002F911F910F910F900FBE0F901F9018954E
:106BD000EF92FF920F931F9380913A069927880FA7
:106BE000991F880F991F7C010027F7FC0095102F33
:106BF0008091750390917603A0917703B09178030B
:106C0000BC01CD01A80197010E94A1783093CA056B
:106C10002093C90580916D0390916E03A0916F033D
:106C2000B0917003BC01CD01A80197010E94A17829
:106C30003093CC052093CB058091030890910408F4
:106C400097FD039695958795959587959093CE0595
:106C50008093CD05809113089091140897FD0396B9
:106C600095958795959587959093D0058093CF05B9
:106C700080918603909187032091470230914802CA
:106C8000821B930B9093D2058093D10580911303BF
:106C900090911403A0911503B0911603BC01CD018E
:106CA00025E030E040E050E00E94A1783093D40528
:106CB0002093D30580914102909142029093D60592
:106CC0008093D50580913303909134039093DA0536
:106CD0008093D90580911E0190911F019093DC054E
:106CE0008093DB058091210399279093DE058093A3
:106CF000DD0580910F0890911008A0911108B091C6
:106D0000120820919A0130919B0140919C01509171
:106D10009D01BC01CD010E94A1783093E005209334
:106D2000DF058091E90699279093E2058093E105BC
:106D30008091F10699279093E4058093E305809173
:106D4000F90699279093E6058093E5058091010760
:106D500099279093E8058093E7058091220290910E
:106D600023029093F2058093F10580919108909110
:106D700092089093F6058093F5058091950890917F
:106D800096089093F8058093F705809197089927C6
:106D900090930406809303068091FD039091FE0377
:106DA00090930606809305068091FB039091FC0367
:106DB000909308068093070680914704882321F466
:106DC00080914804882321F08091C805816003C028
:106DD0008091C8058E7F8093C8051F910F91FF9009
:106DE000EF9008951F93CF93DF93182FEB018091BD
:106DF00018038823A1F411501F3F89F0D093290272
:106E0000C09328028091280290912902892BD1F702
:106E1000CE018C0F9D1F0E942F17115078F7DF9124
:106E2000CF911F910895CF93DF93809102018D3010
:106E300011F40E94141B10927A0080914B029091E1
:106E40004C029093CA078093C907809149029091A0
:106E50004A029093BB078093BA07809147029091B2
:106E600048029093090880930808209143023091CA
:106E70004402C901880F991F880F991F820F931F21
:106E8000820F931F9093040880930308209145027A
:106E900030914602C901880F991F880F991F820FF0
:106EA000931F820F931F90931408809313088FEC05
:106EB00080937A00A2E2B3E0C3E2D6E097E0899142
:106EC000E82FFF27EE0FFF1FE75BF84F0190F081DF
:106ED000E02DE259FF4F1E161F061CF0E0E0F0E027
:106EE00005C0EF3FF10514F0EFEFF0E08C91282F93
:106EF0003327E217F30714F4815004C02E173F071D
:106F000014F48F5F8C939150119697FFD8CF809196
:106F10005F069927AA27BB27BC01CD0124EC39E0E5
:106F200040E050E00E942D78DC01CB018093D90134
:106F30009093DA01A093DB01B093DC0180916006AD
:106F40009927AA27BB27BC01CD010E942D78DC011F
:106F5000CB018093D5019093D601A093D701B09334
:106F6000D801DF91CF910895A0E0B0E0EAEBF7E31C
:106F70000C94C278882EC0E0D0E07E016E011092A1
:106F80004704469AD0938103C0938003D0937F0334
:106F9000C0937E03D0937B03C0937A03D0938B037B
:106FA000C0938A03D0938903C0938803D093870347
:106FB000C09386031092C2011092C10110923B024D
:106FC0000E94133784E690E00E943C170E9413371A
:106FD00080912B0680FF10C08091140190911501C3
:106FE000875B934038F480911401909115018E5E77
:106FF000924010F40E94B91A0FE18AE090E00E94DA
:107000003C178091470290914802C80FD91F809188
:107010004B0290914C02E80EF91E8091490290912A
:107020004A02C80ED91E015007FFE7CF9701205F23
:107030003F4F369527953695279530938B032093B0
:107040008A03C60140969695879596958795909365
:107050008903809388036096F5E0D695C795FA95E5
:10706000E1F7D0938703C0938603909385038093C1
:1070700084033093830320938203882009F441C062
:10708000809103089091040897FF03C09095819523
:107090009F4F6CE070E00E946C789B0170938103BD
:1070A00060938003809113089091140897FF03C0A8
:1070B000909581959F4F6CE070E00E946C78709382
:1070C0007F0360937E038091100690911106909348
:1070D0007B0380937A03B90184E090E00E94902CB6
:1070E00060917E0370917F0386E090E00E94902C77
:1070F00060917A0370917B0388E090E00E94902C6D
:1071000065C084E090E00E948B2C90938103809373
:10711000800386E090E00E948B2C90937F03809305
:107120007E0388E090E00E948B2C9C0190937B036F
:1071300080937A03809180039091810381509840DD
:1071400050F480917E0390917F038150984018F411
:1071500021503440D8F187E19AE09F938F9384EFD8
:1071600092E19F938F93E0912E04F0912F04099563
:10717000809103089091040897FF03C09095819532
:107180009F4F6CE070E00E946C7870938103609375
:107190008003809113089091140897FF03C0909585
:1071A00081959F4F6CE070E00E946C7870937F0334
:1071B00060937E03809110069091110690937B035B
:1071C00080937A030F900F900F900F901092CA0740
:1071D0001092C9071092BB071092BA0710920908C3
:1071E0001092080884E690E00E943C1780914302C8
:1071F000909144029C01220F331F220F331F280F4E
:10720000391F280F391F30930408209303088091F9
:107210004502909146028C01000F111F000F111FB3
:10722000080F191F080F191F109314080093130853
:1072300080913A06C82EDD24EE24FF24442737FD32
:107240004095542FC701B6010E942D784B015C0177
:10725000609375037093760380937703909378031C
:107260009801442737FD4095542FC701B6010E946D
:107270002D78DC01CB0180936D0390936E03A09376
:107280006F03B09370038092510390925203A092C7
:107290005303B09254038093490390934A03A093FD
:1072A0004B03B0934C031092450310924603109287
:1072B0004703109248038091160190911701A09105
:1072C0001801B09119019093130680931206109241
:1072D0003A0210923902109235031092360310923E
:1072E00037031092380380913303909134039093C5
:1072F0003203809331030E94DE6282E390E0909338
:1073000029028093280280915F069927AA27BB272C
:10731000BC01CD0124EC39E040E050E00E942D7822
:10732000DC01CB018856954CAF4FBF4F8093D901FC
:107330009093DA01A093DB01B093DC0180916006A9
:107340009927AA27BB27BC01CD010E942D78DC011B
:10735000CB018856954CAF4FBF4F8093D50190938A
:10736000D601A093D701B093D80110929F0110923B
:107370009E018091330390913403AA2797FDA09535
:10738000BA2F20919A0130919B0140919C0150911C
:107390009D01BC01CD010E942D78DC01CB018093C1
:1073A0000F0890931008A0931108B0931208109240
:1073B0002C0310922B0381E0809301010E945567FA
:1073C0008091ED0284608093ED028FEF80938108BD
:1073D0001092820880E280938308C2E2D3E0A3E2A5
:1073E000B6E007E08D91E82FFF27EE0FFF1FE75B68
:1073F000F84F8081918182598993015007FFF2CF24
:1074000084E68093210380912602882311F0469A16
:10741000579A80918A0390918B0380569940815CA2
:107420009B4228F0809147048160809347048091BB
:1074300088039091890380569940815C9B4228F093
:1074400080914704826080934704809186039091E5
:1074500087038C5291408957954028F080914704CA
:1074600084608093470480918003909181038C52C3
:107470009140835C914028F080914704886080931C
:10748000470480917E0390917F038C529140835CEE
:10749000914028F080914704806180934704809157
:1074A0007A0390917B03805092408355914028F05D
:1074B00080914704806280934704ECE0CDB7DEB74B
:1074C0000C94DE78A3E1B0E0E8E6FAE30C94BC7833
:1074D0008091860390918703209147023091480262
:1074E000821B930B909309088093080880915102A6
:1074F0009091520297FD07969C0113E035952795D0
:107500001A95E1F73093CA072093C90780914F027B
:107510009091500297FD0796B3E095958795BA959F
:10752000E1F79093BB078093BA073093D507209378
:10753000D4079093CD078093CC0780910308909156
:107540000408AC01440F551F480F591F20914302F6
:1075500030914402C901880F991F880F991F820F2B
:10756000931F820F931F480F591F57FF02C04D5F93
:107570005F4F55954795559547955093040840930F
:1075800003088091130890911408AC01440F551F13
:10759000480F591F2091450230914602C901880FBA
:1075A000991F880F991F820F931F820F931F480FF7
:1075B000591F57FF02C04D5F5F4F55954795559531
:1075C000479550931408409313082091430230913B
:1075D0004402C901880F991F880F991F820F931FBA
:1075E000820F931F9C01442737FD4095542F8091B3
:1075F000650390916603A0916703B0916803820FC1
:10760000931FA41FB51F8093650390936603A093F7
:107610006703B09368032091450230914602C90187
:10762000880F991F880F991F820F931F820F931F36
:107630009C01442737FD4095542F80916103909120
:107640006203A0916303B0916403820F931FA41F90
:10765000B51F8093610390936203A0936303B0937B
:1076600064038091DE079091DF07209143023091FF
:107670004402820F931F9093DF078093DE0780916F
:107680000B0890910C082091450230914602820F20
:10769000931F90930C0880930B0880917C0390912A
:1076A0007D03019690937D0380937C038091100667
:1076B0009091110620917A0330917B03821B930BEA
:1076C0009C01442737FD4095542F80915D03909194
:1076D0005E03A0915F03B0916003820F931FA41F0C
:1076E000B51F80935D0390935E03A0935F03B093F7
:1076F00060038FEC80937A001092100120914D036B
:1077000030914E0340914F035091500329873A879F
:107710004B875C8729543B46414050402CF028E47D
:107720003BE641E050E00DC089859A85AB85BC857C
:10773000885B9449AE4FBF4F4CF428EB34E94EEFD1
:107740005FEF2D833E834F83588708C089859A85D4
:10775000AB85BC858D839E83AF83B887209155030D
:107760003091560340915703509158032D873E871F
:107770004F87588B29543B46414050402CF028E419
:107780003BE641E050E00DC08D859E85AF85B88910
:10779000885B9449AE4FBF4F4CF428EB34E94EEF71
:1077A0005FEF29833A834B835C8308C08D859E8578
:1077B000AF85B88989839A83AB83BC83A09108087D
:1077C000B0910908BB8BAA8BFD01CF01AA2797FDB9
:1077D000A095BA2FA0904503B0904603C0904703F0
:1077E000D0904803A80EB91ECA1EDB1EA092450306
:1077F000B0924603C0924703D0924803E0900F082E
:10780000F09010080091110810911208E80EF91E6E
:107810000A1F1B1FE0920F08F09210080093110836
:1078200010931208F0910803F98BFF2309F098C117
:1078300080910703882309F093C180912B0686FF6E
:107840008FC18091BA079091BB07AA2797FDA09599
:10785000BA2FBC01CD0129813A814B815C810E9404
:107860002D789B01AC0197FF04C02150384F4F4F3A
:107870005F4FBBE05595479537952795BA95D1F75A
:107880008091C101682E772488249924CA01B90106
:10789000A40193010E942D78DC01CB018093960313
:1078A00090939703A0939803B0939903B7FF04C0F4
:1078B0008150904FAF4FBF4F1C012D01ACE055944C
:1078C000479437942794AA95D1F720929603309243
:1078D000970340929803509299038091C907909121
:1078E000CA07AA2797FDA095BA2FBC01CD012D810B
:1078F0003E814F8158850E942D7897FF04C06150CA
:10790000784F8F4F9F4FFBE09595879577956795BB
:10791000FA95D1F7A40193010E942D78DC01CB01E7
:1079200080939A0390939B03A0939C03B0939D0331
:10793000B7FF04C08150904FAF4FBF4F9C01AD01C6
:10794000ECE05595479537952795EA95D1F7209323
:107950009A0330939B0340939C0350939D03809123
:107960009603909197039093B2078093B10780910B
:107970009A0390919B039093B6078093B5072219C1
:1079800033094409550920939A0330939B0340938C
:107990009C0350939D03E20EF31E041F151FE092FB
:1079A0000F08F092100800931108109312088091AC
:1079B000C0018823B1F457FF04C02F5F3F4F4F4FE2
:1079C0005F4F5595479537952795A21AB30AC40A74
:1079D000D50AA0924503B0924603C0924703D092C5
:1079E00048032A893B8979010027F7FC0095102F6D
:1079F00080919A0390919B03A0919C03B0919D0369
:107A0000E80EF91E0A1F1B1FC801B70129813A8120
:107A10004B815C810E942D789B01AC0197FF04C0D3
:107A20002150384F4F4F5F4F6BE055954795379535
:107A300027956A95D1F78091C201A82EBB24CC244A
:107A4000DD24CA01B901A60195010E942D78DC014F
:107A5000CB0180938E0390938F03A0939003B093F8
:107A60009103B7FF04C08150904FAF4FBF4F3C010F
:107A70004D013CE095948794779467943A95D1F7BB
:107A800060928E0370928F03809290039092910384
:107A9000C801B7012D813E814F8158850E942D7804
:107AA00097FF04C06150784F8F4F9F4F2BE0959503
:107AB0008795779567952A95D1F7A60195010E943C
:107AC0002D78DC01CB018093920390939303A093D4
:107AD0009403B0939503B7FF04C08150904FAF4F0C
:107AE000BF4FAC01BD018CE07595679557954795E3
:107AF0008A95D1F740939203509393036093940334
:107B0000709395032A893B8937FF03C030952195EF
:107B10003F4F21343105E4F1D401C30197FE07C082
:107B2000B095A095909581959F4FAF4FBF4F8138ED
:107B30009105A105B10584F4DB01CA0177FF07C0F7
:107B4000B095A095909581959F4FAF4FBF4F8138CD
:107B50009105A105B105E4F081E080932D0318C0E3
:107B60001092B6071092B5071092B2071092B107A3
:107B70001092920310929303109294031092950323
:107B800010928E0310928F03109290031092910323
:107B90008091920390919303A0919403B0919503E7
:107BA000BC01CD0124E630E040E050E00E94A17825
:107BB000E0908E03F0908F03E21AF30AF092C80768
:107BC000E092C70780918E0390918F03A09190035C
:107BD000B0919103BC01CD0124E630E040E050E0DB
:107BE0000E94A178DA01C901209192033091930398
:107BF0008C01021B130B1093BD070093BC078091EF
:107C00009A0190919B01A0919C01B0919D01BC01B2
:107C1000CD0128E631E040E050E00E942D7820912F
:107C20000F08309110084091110850911208261742
:107C300037074807590764F0261B370B480B590BC9
:107C400020930F08309310084093110850931208A6
:107C500020910F083091100840911108509112089E
:107C600057FF0CC0260F371F481F591F20930F08BE
:107C70003093100840931108509312086091BA078E
:107C80007091BB076E0D7F1D9B01442737FD40950A
:107C9000542F8091490390914A03A0914B03B091D6
:107CA0004C03820F931FA41FB51F80934903909329
:107CB0004A03A0934B03B0934C0380910D03909122
:107CC0000E03681B790BCB01AA2797FDA095BA2F4D
:107CD00029853A854B855C85820F931FA41FB51FAC
:107CE00080934D0390934E03A0934F03B0935003A2
:107CF000C090D501D090D601E090D701F090D80186
:107D0000C816D906EA06FB06C4F488EA91E6A0E0A4
:107D1000B0E08C199D09AE09BF0980934D03909383
:107D20004E03A0934F03B093500380934903909365
:107D30004A03A0934B03B0934C0322273327A90196
:107D40002C193D094E095F0980914D0390914E0316
:107D5000A0914F03B091500382179307A407B50772
:107D6000B4F4D701C601885A9146A040B040809330
:107D70004D0390934E03A0934F03B0935003809311
:107D8000490390934A03A0934B03B0934C03609133
:107D9000C9077091CA07600F711F9B01442737FD07
:107DA0004095542F8091510390915203A091530319
:107DB000B0915403820F931FA41FB51F80935103EA
:107DC00090935203A0935303B093540380910B03F9
:107DD00090910C03681B790BCB01AA2797FDA09506
:107DE000BA2F2D853E854F855889820F931FA41F7A
:107DF000B51F8093550390935603A0935703B093F8
:107E00005803E090D901F090DA010091DB01109164
:107E1000DC01E816F9060A071B07C4F488EA91E6B4
:107E2000A0E0B0E08E199F09A00BB10B8093550321
:107E300090935603A0935703B09358038093510334
:107E400090935203A0935303B093540322273327F4
:107E5000A9012E193F09400B510B809155039091B8
:107E60005603A0915703B091580382179307A407B4
:107E7000B507B4F4D801C701885A9146A040B04074
:107E80008093550390935603A0935703B0935803E0
:107E90008093510390935203A0935303B0935403E0
:107EA0008091450390914603A0914703B091480308
:107EB0008093590390935A03A0935B03B0935C03A0
:107EC0008091550390915603A0915703B0915803A8
:107ED0008093750390937603A0937703B093780310
:107EE00080914D0390914E03A0914F03B0915003A8
:107EF00080936D0390936E03A0936F03B093700310
:107F00008091510390915203A0915303B091540377
:107F10008093710390937203A0937303B0937403DF
:107F20008091490390914A03A0914B03B0914C0377
:107F30008093690390936A03A0936B03B0936C03DF
:107F400080911C0190911D0197FD079603E0959586
:107F500087950A95E1F79093CA078093C9078091A6
:107F60001A0190911B0197FD079613E0959587954F
:107F70001A95E1F79093BB078093BA0780914B0263
:107F800090914C020F9734F488E19CEF9093CA07CC
:107F90008093C90780914B0290914C02079734F46B
:107FA00080E398EF9093CA078093C907209102015C
:107FB0002A30A9F480914B0290914C02835F934048
:107FC00034F088EE93E09093CA078093C9078091BC
:107FD0004B0290914C028A5F9340DCF014C0809178
:107FE0004B0290914C02815D974034F088EE93E013
:107FF0009093CA078093C90780914B0290914C02DD
:10800000805E974034F080ED97E09093CA078093AC
:10801000C9078091490290914A020F9734F488E190
:108020009CEF9093BB078093BA078091490290918F
:108030004A02079734F480E398EF9093BB0780934C
:10804000BA072A30A9F48091490290914A02835FCD
:10805000934034F088EE93E09093BB078093BA0787
:108060008091490290914A028A5F9340DCF014C0EB
:108070008091490290914A02815D974034F088EEE8
:1080800093E09093BB078093BA0780914902909147
:108090004A02805E974034F080ED97E09093BB07F2
:1080A0008093BA076091CC01662309F4AFC0409178
:1080B0001C0150911D0180919E0390919F03481BCC
:1080C000590B5093A5034093A40320911C013091B8
:1080D0001D01280F391F37FF02C02F5F3F4F359515
:1080E000279530939F0320939E03413851051CF040
:1080F00080E890E005C040585F4F34F480E89FEF7F
:108100009093A5038093A40340911A0150911B0101
:108110008091A0039091A103481B590B5093A30396
:108120004093A20320911A0130911B01280F391F9F
:1081300037FF02C02F5F3F4F359527953093A1033E
:108140002093A003413851051CF080E890E005C061
:1081500040585F4F34F480E89FEF9093A3038093DF
:10816000A203462F55278091A4039091A503849FD5
:10817000B001859F700D949F700D11249B0177FFB6
:1081800002C0215F3F4FF4E035952795FA95E1F75E
:108190008091C9079091CA07820F931F9093CA07D5
:1081A0008093C9078091A2039091A303849FD0017B
:1081B000859FB00D949FB00D1124AD019D01B7FFB7
:1081C00002C0215F3F4FE4E035952795EA95E1F73E
:1081D0008091BA079091BB07820F931F9093BB07C2
:1081E0008093BA0780911C0190911D01860F971F03
:1081F00090931D0180931C0180911A0190911B01A5
:10820000840F951F90931B0180931A010091CC0756
:108210001091CD078091B1079091B2071016110609
:108220005CF59C0197FF04C022273327281B390BDC
:10823000C901AA2797FDA095BA2F2091C001332725
:1082400044275527BC01CD010E942D789B01AC012C
:1082500097FF04C0215C3F4F4F4F5F4F76E055952D
:108260004795379527957A95D1F78091C7079091D3
:10827000C807820F931F27C097FF03C09095819571
:108280009F4FAA2797FDA095BA2F2091C0013327B1
:1082900044275527BC01CD010E942D789B01AC01DC
:1082A00097FF04C0215C3F4F4F4F5F4F66E05595ED
:1082B0004795379527956A95D1F78091C707909193
:1082C000C807821B930B9093C8078093C707E09061
:1082D000D407F090D5078091B5079091B6071E148A
:1082E0001F045CF59C0197FF04C022273327281B3D
:1082F000390BC901AA2797FDA095BA2F2091C0017B
:10830000332744275527BC01CD010E942D789B01BE
:10831000AC0197FF04C0215C3F4F4F4F5F4F96E089
:1083200055954795379527959A95D1F78091BC0734
:108330009091BD07820F931F27C097FF03C09095B0
:1083400081959F4FAA2797FDA095BA2F2091C00134
:10835000332744275527BC01CD010E942D789B016E
:10836000AC0197FF04C0215C3F4F4F4F5F4F86E049
:1083700055954795379527958A95D1F78091BC07F4
:108380009091BD07821B930B9093BD078093BC0710
:1083900080912B0687FF44C0B989BB2309F040C0F8
:1083A000809107038823E1F5E1E0EE16E1E0FE06A7
:1083B0004CF08091C9079091CA078E0D9F1D805087
:1083C00091400DC0F0E0EF16FFEFFF0664F48091DE
:1083D000C9079091CA078E0D9F1D80509F4F9093A3
:1083E000CA078093C90721E0013012074CF0809141
:1083F000BA079091BB07800F911F805091400CC02D
:108400003FEF0030130764F48091BA079091BB07E7
:10841000800F911F80509F4F9093BB078093BA07A6
:10842000E2E1CD5E0C94D87880911803882301F5A1
:108430008091ED028C7F8093ED02ACE4B4E0E8EE35
:10844000F6E09BE080910702882309F48C938D91DC
:10845000818312829150389697FFF4CF8091070262
:10846000882359F08091070281508093070205C04C
:108470008091ED0281608093ED02809172028823E9
:1084800019F010927202089580937402809376021C
:10849000809170028E7F8093700285EA8093BC0089
:1084A0000895CF93DF93A2E2B3E0C3E2D6E057E0B2
:1084B0008991E82FFF27EE0FFF1FE75BF84F019030
:1084C000F081E02DE259FF4FEF3FF10521F01CF064
:1084D000EFEFF0E004C0F7FF02C0E0E0F0E04C9105
:1084E000242F3327E217F307A9F0CF01821B930B48
:1084F00097FD03969595879595958795242F280F39
:108500002C93822F9927E817F90714F4215001C002
:108510002F5F2C935150119657FFCACF80912D0693
:10852000883F38F0EFEFF0E0E81BF109EE5DFC4F1B
:1085300080818093D2018091D201882329F08436F2
:1085400018F084E68093D20180912F06883F38F09E
:10855000EFEFF0E0E81BF109EE5DFC4F80818093C6
:10856000D0018091D001882329F0843618F084E668
:108570008093D00180913C06883F38F0EFEFF0E027
:10858000E81BF109EE5DFC4F80818093CB01809167
:10859000CB018B3010F48AE002C08F3F11F480933E
:1085A000CB0180916906883F38F0EFEFF0E0E81BDF
:1085B000F109EE5DFC4F80818093E0078091E00738
:1085C000823010F481E002C08F3F11F48093E00705
:1085D00080916B06883F38F0EFEFF0E0E81BF1097F
:1085E000EE5DFC4F80818093060880910608823002
:1085F00010F481E002C08F3F11F48093060880914F
:108600005606883F38F0EFEFF0E0E81BF109EE5D29
:10861000FC4F80818093DD0780915706883F38F0BA
:10862000EFEFF0E0E81BF109EE5DFC4F80818093F5
:10863000B70780915806883F38F0EFEFF0E0E81B6D
:10864000F109EE5DFC4F80818093E50790912E0645
:10865000983F18F49093D10109C0EFEFF0E0E91BC7
:10866000F109EE5DFC4F80818093D101983F18F4B1
:108670009093D10109C0EFEFF0E0E91BF109EE5D45
:10868000FC4F80818093D10180913106883F38F082
:10869000EFEFF0E0E81BF109EE5DFC4F8081809385
:1086A000CF0180913306883F38F0EFEFF0E0E81B10
:1086B000F109EE5DFC4F80818093CD0180913B06F6
:1086C000883F38F0EFEFF0E0E81BF109EE5DFC4F7A
:1086D00080818093CE0180913D06883F38F0EFEF96
:1086E000F0E0E81BF109EE5DFC4F80818093CA0148
:1086F00080913E06883F38F0EFEFF0E0E81BF1098B
:10870000EE5DFC4F80818093CC0180913F06883FD5
:1087100038F0EFEFF0E0E81BF109EE5DFC4F8081EF
:108720008093C90180914006883F38F0EFEFF0E078
:10873000E81BF109EE5DFC4F80818093C8018091B8
:108740004606883F38F0EFEFF0E0E81BF109EE5DF8
:10875000FC4F80818093C60180914706883F38F0A6
:10876000EFEFF0E0E81BF109EE5DFC4F80818093B4
:10877000020380914806883F38F0EFEFF0E0E81BF5
:10878000F109EE5DFC4F80818093010380914906E1
:10879000883F38F0EFEFF0E0E81BF109EE5DFC4FA9
:1087A00080818093000380914A06883F38F0EFEF84
:1087B000F0E0E81BF109EE5DFC4F80818093FF0241
:1087C00080916406883F38F0EFEFF0E0E81BF10994
:1087D000EE5DFC4F80818093FE0280916506883FAC
:1087E00038F0EFEFF0E0E81BF109EE5DFC4F80811F
:1087F0008093FD0280916606883F38F0EFEFF0E04D
:10880000E81BF109EE5DFC4F80818093FC028091B2
:108810006706883F38F0EFEFF0E0E81BF109EE5D06
:10882000FC4F80818093FB0280914B06883F38F09B
:10883000EFEFF0E0E81BF109EE5DFC4F80818093E3
:10884000C50180914F06883F38F0EFEFF0E0E81B5C
:10885000F109EE5DFC4F80818093C401809159063F
:10886000883F38F0EFEFF0E0E81BF109EE5DFC4FD8
:1088700080818093C30180915C06883F38F0EFEFE0
:10888000F0E0E81BF109EE5DFC4F80818093C201AE
:1088900080915D06883F38F0EFEFF0E0E81BF109CA
:1088A000EE5DFC4F80818093C10180915E06883F20
:1088B00038F0EFEFF0E0E81BF109EE5DFC4F80814E
:1088C0008093C00180916306883F38F0EFEFF0E0BD
:1088D000E81BF109EE5DFC4F80818093BF01809120
:1088E0007E06883F38F0EFEFF0E0E81BF109EE5D1F
:1088F000FC4F8081809316088091C601282F332772
:108900002F5F3F4F8CE398E2B9010E946C7870931F
:10891000D4016093D3018091390680930708809138
:1089200038068093CE0780910203813011F08430A5
:1089300049F481E090E0909398018093970183E05F
:1089400090E008C083E090E09093980180939701B5
:1089500081E090E09093960180939501909180063C
:10896000933320F181E08093FA02983F58F0EFEFC3
:10897000F0E0E91BF109EE5DFC4F8081823310F4D9
:108980001092FA02809154089091550897FF08C000
:108990008091FA02882321F080914704806803C007
:1089A000809147048F778093470402C01092FA02A7
:1089B000809154089091550897FF1DC0809118032D
:1089C0008823C9F08091FA028823A9F080910801D8
:1089D000909109018F5F9F4F71F488E99AE390931A
:1089E00029028093280280E094EA90930901809301
:1089F00008011092FA028091FA02882339F08091DE
:108A0000C201823D18F4825E8093C201DF91CF9152
:108A10000895A8E1B0E0EFE0F5E40C94BC780E9482
:108A2000623A309102013C3010F4299A01C0299831
:108A3000E0901903F0901A03FA82E9828091CE0740
:108A400099270A96E816F90614F49A838983809187
:108A50002103843608F05CC08091BA039091BB0377
:108A6000009731F001979093BB038093BA0307C03E
:108A7000109218038091ED028F7E8093ED023A30C0
:108A800011F0343110F0289A01C028988091EE023C
:108A90009091EF02895E9340C0F180914306282FA8
:108AA00033273A8329838091ED0280618093ED0220
:108AB00080911F06A82FBB27AA0FBB1FFD01E358FB
:108AC000F84F1182108280912006282F3327220F21
:108AD000331FC9018358984FFC0111821082A75B94
:108AE000B84F11961C921E92275B384FD9011196F0
:108AF0001C921E9280912206E82FFF27EE0FFF1F87
:108B0000E75BF84F11821082F4C210921803F1C291
:108B1000809121038D3808F4ECC28091ED028F7EA4
:108B20008093ED029091440682E3989FC001112446
:108B30009093BB038093BA03E981FA81B9978CF0D3
:108B400080911803882369F08091EE029091EF02E2
:108B5000FFEF8F3F9F0729F001969093EF028093DC
:108B6000EE028091EE029091EF028F3F910509F0A5
:108B700038F510923D0310923E0310923F0310927D
:108B800040031092390310923A0310923B03109263
:108B90003C031092A6031092A7031092A803109210
:108BA000A9031092450310924603109247031092B6
:108BB00048038A3F910549F481E08093C00305C0D2
:108BC0008091ED0282608093ED0280912106E82F72
:108BD000FF27EE0FFF1FE75BF84F80819181813502
:108BE00091050CF462C120911803222309F05DC1A4
:108BF000E0919701F0919801E25EF94F8181E82FB1
:108C0000FF27EE0FFF1FE75BF84F808191818C34C7
:108C100091050CF422C18091BC038F5F8093BC034B
:108C2000893C08F442C13C3010F4299801C0299ACB
:108C3000109218031092BC031092EF021092EE02F1
:108C400020911F06E22FFF27EE0FFF1FE75BF84F73
:108C50008081918187349105DCF4E0919501F09158
:108C60009601E25EF94F8181E82FFF27EE0FFF1F8B
:108C7000E75BF84F808191810190F081E02DF7FF53
:108C800003C0F095E195FF4FE734F1050CF48AC07D
:108C900031E04091950150919601FA01E25EF94F61
:108CA0008181A82FBB27AA0FBB1FA75BB84F8D914F
:108CB0009C9111978734910544F0E22FFF27EE0F26
:108CC000FF1FE75BF84F808191818D919C918734E4
:108CD000910574F080911F06E82FFF27EE0FFF1F0C
:108CE000E75BF84F80819181873491050CF032E089
:108CF000FA01E25EF94F8181E82FFF27EE0FFF1F97
:108D0000E75BF84F808191818634910574F48091FE
:108D10001F06E82FFF27EE0FFF1FE75BF84F80814C
:108D20009181873491050CF033E0FA01E25EF94F4E
:108D30008181E82FFF27EE0FFF1FE75BF84F80814F
:108D400091818A5B9F4F74F480911F06E82FFF2763
:108D5000EE0FFF1FE75BF84F80819181873491050B
:108D60000CF034E0425E594FFA018181E82FFF2771
:108D7000EE0FFF1FE75BF84F808191818A5B9F4F69
:108D800074F480911F06E82FFF27EE0FFF1FE75BAB
:108D9000F84F80819181863491050CF435E0832F62
:108DA0000E94CC2CE0919501F0919601E25EF94F82
:108DB0008181E82FFF27EE0FFF1FE75BF84F8081CF
:108DC00091810190F081E02DF7FF03C0F095E195CE
:108DD000FF4F7E97BCF480911F06E82FFF27EE0F10
:108DE000FF1FE75BF84F808191818A5B9F4F54F4AE
:108DF00081E08093620488EE93E09093290280934F
:108E0000280253C00E94A22D0E94952C80E00E944F
:108E10003607809145060E94A17580912B0680FF40
:108E200010C08091140190911501875B934038F434
:108E300080911401909115018E5E924010F40E9471
:108E4000B91A1092260280E00E94B43781E0809324
:108E5000BF0380932602579A1FC080819181855B52
:108E60009F4F0CF58091BC038F5F8093BC03893CBE
:108E7000E0F03C3010F4299801C0299A10921803B0
:108E80001092BC031092EF021092EE0281E00E9459
:108E9000B43781E08093BF030E94A22D68E770E0A1
:108EA0000E94F23602C02093BC0380912106E82F75
:108EB000FF27EE0FFF1FE75BF84F808191818B5AF0
:108EC0009F4F0CF016C130911803E0919701F0917B
:108ED0009801332309F0DEC0E25EF94F8181E82F6B
:108EE000FF27EE0FFF1FE75BF84F80819181855BC5
:108EF0009F4F0CF0CCC020918106E22FFF27EE0F90
:108F0000FF1FE75BF84F80819181855B9F4F1CF0CD
:108F1000222309F0BCC08091BD038F5F8093BD0305
:108F2000893C08F4E6C03093BD0380914704882350
:108F300009F0A6C08091BF03882309F4A1C081E095
:108F400090E09093EF028093EE0281E0809318030B
:108F50001092A6031092A7031092A8031092A903DF
:108F60001092450310924603109247031092480353
:108F70001092410310924203109243031092440353
:108F800080913A06E82EFF240027112780910308DC
:108F9000909104089C01442737FD4095542FC80147
:108FA000B7010E942D78DC01CB018093550390938B
:108FB0005603A0935703B0935803809113089091E0
:108FC00014089C01442737FD4095542FC801B70170
:108FD0000E942D78DC01CB0180934D0390934E03CA
:108FE000A0934F03B0935003809175039091760343
:108FF000A0917703B091780380935103909352032B
:10900000A0935303B093540380916D0390916E032A
:10901000A0916F03B09170038093490390934A032A
:10902000A0934B03B0934C0310923D0310923E0368
:1090300010923F03109240031092390310923A03AA
:1090400010923B0310923C038091ED028860809364
:10905000ED0290917F068FE0989F900111248091FE
:10906000330390913403820F931F68E671E00E94EE
:109070006C7897FD0196959587958093790339C013
:109080008CED95E0909329028093280232C01092D3
:10909000BD032FC0E25EF94F8181E82FFF27EE0F5D
:1090A000FF1FE75BF84F808191818C349105FCF0C4
:1090B00020918106E22FFF27EE0FFF1FE75BF84F9D
:1090C00080819181855B9F4F14F0222381F48091F0
:1090D000BE038F5F8093BE03893C58F01092180343
:1090E0001092BE031092EF021092EE0202C0109294
:1090F000BE038091940181508093940180919401EA
:109100008F3F21F08091ED0284FF72C30E94514293
:109110008091C9039091CA039C01220F331F280F2D
:10912000391FC0901F06AC2DBB27AA0FBB1FFD0126
:10913000E75BF84FB09035064B2D55278081918124
:10914000849FF001859FF00D949FF00D11242E0F48
:109150003F1F37FF02C02D5F3F4FB90175956795DF
:1091600075956795A358B84F80913606082F11273B
:109170008D919C91809F7001819FF00C909FF00CCD
:1091800011246E0D7F1D7093CA036093C9038091F3
:10919000CB039091CC039C01220F331F280F391F62
:1091A000D0902006AD2DBB27AA0FBB1FFD01E75BAA
:1091B000F84F80819181849FF001859FF00D949FED
:1091C000F00D11242E0F3F1F37FF02C02D5F3F4FC0
:1091D000A9015595479555954795A358B84F8D9139
:1091E0009C91809F7001819FF00C909FF00C112446
:1091F0004E0D5F1D5093CC034093CB038091FA0238
:10920000882309F448C0CB0177FD0396DC01B595AE
:10921000A795B595A795CA0157FD0396FC01F5954D
:10922000E795F595E7958091EE01682F772767FD23
:1092300070956A9F90016B9F300D7A9F300D1124BD
:1092400080910104482F552747FD50954E9FC0013E
:109250004F9F900D5E9F900D1124280F391F37FFEF
:1092600002C0295F3F4F03E0359527950A95E1F746
:109270003093200320931F036E9F90016F9F300D4A
:109280007E9F300D11244A9FC0014B9F900D5A9F25
:10929000900D11243FC080917F06E82FFF27E056F4
:1092A000FE4F86818093EE01908190930104A82F58
:1092B000BB27A7FDB095A69F9001A79F300DB69F35
:1092C000300D1124E92FFF27E7FDF095E49FC00141
:1092D000E59F900DF49F900D1124280F391F37FF43
:1092E00002C0295F3F4F13E0359527951A95E1F7A6
:1092F0003093200320931F03A49F9001A59F300D5E
:10930000B49F300D1124E69FC001E79F900DF69F9A
:10931000900D1124281B390B37FF02C0295F3F4FE6
:10932000F3E035952795FA95E1F730931E032093E6
:109330001D0380912206E82FFF27EE0FFF1FE75B3A
:10934000F84F80819181909581959F4F90931C0358
:1093500080931B038330910514F0029705C00FEF33
:109360008E3F900734F4029690931C0380931B0366
:1093700004C010921C0310921B038091FD03909176
:10938000FE032091F9033091FA03820F931F00919D
:109390001F0310912003081B190B10932003009347
:1093A0001F038091FB039091FC032091F703309100
:1093B000F803820F931F80901D0390901E03881A5C
:1093C000990A90921E0380921D0380912106E82F36
:1093D000FF27EE0FFF1FE75BF84FE080F18028E7E3
:1093E00030E0E20EF31EF0921A03E092190380912E
:1093F000CB019927AA2797FDA095BA2FBC01CD01D3
:109400000E94D577DC01CB0120E030E040E251E45E
:10941000BC01CD010E947677DC01CB01BC01CD01FE
:109420000E94B877DC01CB0180930D088091CA01BE
:109430008093E6078091C9019927AA2797FDA095F7
:10944000BA2FBC01CD010E94D577DC01CB0120E011
:1094500030E040E251E4BC01CD010E947677DC01AE
:10946000CB01BC01CD010E94B877DC01CB01809318
:10947000C1078091C8018093D60780916E0480FF58
:1094800059C080911608813808F454C0809167044F
:10949000992787FD90952B2D3327829FA001839FCD
:1094A000500D929F500D1124040F151F109320038F
:1094B00000931F0380916804992787FD9095829FF0
:1094C000B001839F700D929F700D1124860E971E20
:1094D00090921E0380921D0380916904282F3327E8
:1094E00027FD309580911B0390911C03820F931FE1
:1094F00090931C0380931B0380916B04282F3327C8
:1095000027FD3095809130069927289FD001299F0B
:10951000B00D389FB00D1124B0939F01A0939E0110
:1095200080916A0499278E159F0524F490931A035D
:10953000809319038091190390911A0397FF04C037
:1095400010921A031092190380912B0682FF02C019
:109550001092E60740911F0350912003CA0157FD66
:1095600003969C01359527953595279537FF03C0C0
:10957000309521953F4F8091F2029091F30282172E
:109580009307B4F4CA0157FF03C0909581959F4F8C
:1095900097FD039695958795959587959093F302FA
:1095A0008093F2028536910544F084E690E001C094
:1095B00001979093F3028093F20240911D03509122
:1095C0001E03CA0157FD03969C01359527953595D5
:1095D000279537FF03C0309521953F4F8091F002CA
:1095E0009091F10282179307B4F4CA0157FF03C0A8
:1095F000909581959F4F97FD0396959587959595A5
:1096000087959093F1028093F0028536910544F09E
:1096100084E690E001C001979093F1028093F002FC
:109620008091ED0284FF08C01092F3021092F202C2
:109630001092F1021092F002ED2DFF27EE0FFF1FA6
:10964000E75BF84F40915A06242F332780819181A0
:109650002817390744F48091820682FF04C081E014
:109660008093060313C0ED2DFF27EE0FFF1FE75B6E
:10967000F84F842F992720915B06821B9109208146
:1096800031812817390714F41092060340912006FF
:10969000E42FFF27EE0FFF1FE75BF84F50915A06AC
:1096A000852F992722273327281B390B8081918109
:1096B0008217930744F48091820683FF04C081E0FF
:1096C0008093050316C080910503882391F0E42F51
:1096D000FF27EE0FFF1FE75BF84F80915B0699278E
:1096E000851B9109208131818217930714F4109210
:1096F0000503EC2DFF27EE0FFF1FE75BF84F4091AE
:109700005A06242F3327808191812817390744F482
:109710008091820680FF04C081E08093030317C01C
:1097200080910303882399F0EC2DFF27EE0FFF1F94
:10973000E75BF84F842F992720915B06821B9109E4
:10974000208131812817390714F4109203034091C6
:109750001F06E42FFF27EE0FFF1FE75BF84F509126
:109760005A06852F992722273327281B390B8081FA
:1097700091818217930744F48091820681FF04C08F
:1097800081E08093040316C080910403882391F044
:10979000E42FFF27EE0FFF1FE75BF84F80915B067A
:1097A0009927851B9109208131818217930714F431
:1097B0001092040380910603882319F48091050315
:1097C000811181E08093070380910303882321F4B2
:1097D00080910403882351F081E080930803109264
:1097E0000703109206031092050302C0809308033A
:1097F00080910703882321F480910803882369F06E
:10980000809159069927E981FA818E179F0714F4F0
:109810009A83898381E080932D038091ED0284FFF8
:109820001AC010921C0310921B0310922003109276
:109830001F0310921E0310921D039AE590930D08CA
:1098400088E78093E6079093C1078093D60710922C
:109850000703109208038091D9079091DA07A0912D
:10986000DB07B091DC0720917503309176034091BE
:10987000770350917803820F931FA41FB51F809325
:10988000D9079093DA07A093DB07B093DC078091A8
:10989000E1079091E207A091E307B091E4072090DF
:1098A0006D0330906E0340906F0350907003820DF3
:1098B000931DA41DB51D8093E1079093E207A0932B
:1098C000E307B093E4078091D0079091D107A0916E
:1098D000D207B091D307E0907103F090720300912A
:1098E000730310917403EB82FC820D831E838E0D33
:1098F0009F1DA01FB11F8093D0079093D107A09305
:10990000D207B093D3078091C2079091C307A0916B
:10991000C407B091C507E0906903F0906A03009115
:109920006B0310916C03EF82F88609871A878E0DFE
:109930009F1DA01FB11F8093C2079093C307A093E0
:10994000C407B093C507F0900803FB86FF2029F4F5
:1099500080910703882309F460C010926503109278
:1099600066031092670310926803109261031092CD
:10997000620310926303109264031092D90710924D
:10998000DA071092DB071092DC071092E1071092C1
:10999000E2071092E3071092E4071092D0071092AA
:1099A000D1071092D2071092D3071092C2071092DB
:1099B000C3071092C4071092C50780915503909178
:1099C0005603A0915703B09158038093510390938D
:1099D0005203A0935303B093540380914D0390918D
:1099E0004E03A0914F03B09150038093490390938D
:1099F0004A03A0934B03B0934C0310923802109289
:109A0000370210920C0310920B0310920E03109267
:109A10000D030B85002309F0F2C180910703882311
:109A200009F0EDC18091100690911106815092408D
:109A30002CF480911803882309F4E1C190908108E7
:109A4000A0903A066091030870910408788F6F8B9C
:109A500080911308909114089A8B898B9FEF991627
:109A600009F4D9C0BB24CC24DD24CA01B901A60164
:109A700095010E94A17879018A01EF89F88DCF01C3
:109A8000AA2797FDA095BA2FE81AF90A0A0B1B0B13
:109A9000C201B101A60195010E94A17859016A0194
:109AA00029893A89C901AA2797FDA095BA2FA81A32
:109AB000B90ACA0ADB0A292C332427FC3094432C28
:109AC000532CC801B701A20191010E942D7897FF84
:109AD00004C061507E4F8F4F9F4F3B014C0109E006
:109AE00095948794779467940A95D1F7C601B50148
:109AF000A20191010E942D7897FF04C061507E4F12
:109B00008F4F9F4F5B016C0119E0D594C794B794B8
:109B1000A7941A95D1F78091F2029091F3028134C3
:109B200091053CF48091F0029091F102813491050D
:109B3000D4F0D401C30197FE03C00196A11DB11D4D
:109B40003C014D019594879477946794D601C501A3
:109B5000D7FE03C00196A11DB11D5C016D01D59416
:109B6000C794B794A79480912206E82FFF27EE0FA1
:109B7000FF1FE75BF84F808191810190F081E02D1C
:109B8000F7FF03C0F095E195FF4F7A97A4F0C40169
:109B9000B30123E030E040E050E00E94A1783901B9
:109BA0004A01C601B50123E030E040E050E00E94E8
:109BB000A17859016A0180918308282F332727FD56
:109BC0003095432F532F261537054805590514F4B2
:109BD00039014A01992787FD9095909581959F4F6E
:109BE000AA2797FDA095BA2F681679068A069B06C4
:109BF00014F43C014D012A153B054C055D0514F498
:109C000059016A01A816B906CA06DB060CF0CFC0D6
:109C10005C016D01CCC0EA2CFF2400271127CA018A
:109C2000B901A80197010E94A17839014A014F8921
:109C3000588DCA01AA2797FDA095BA2F681A790AEC
:109C40008A0A9B0AC201B101A80197010E94A1786A
:109C500059016A0169897A89CB01AA2797FDA095E4
:109C6000BA2FA81AB90ACA0ADB0AD401C30197FE9F
:109C700003C00F96A11DB11D3C014D01F4E0959468
:109C8000879477946794FA95D1F7D601C501D7FEEA
:109C900003C00F96A11DB11D5C016D01E4E0D594D8
:109CA000C794B794A794EA95D1F78091F202909166
:109CB000F302813491053CF48091F0029091F1021D
:109CC00081349105A4F0C401B30123E030E040E009
:109CD00050E00E94A17839014A01C601B50123E094
:109CE00030E040E050E00E94A17859016A01809183
:109CF0002206E82FFF27EE0FFF1FE75BF84F80815A
:109D000091810190F081E02DF7FF03C0F095E1957E
:109D1000FF4F7A97A4F0C401B30123E030E040E0A4
:109D200050E00E94A17839014A01C601B50123E043
:109D300030E040E050E00E94A17859016A0171E2F0
:109D400067167104810491042CF070E2672E712C67
:109D5000812C912C80EE68168FEF78068FEF8806A5
:109D60008FEF980644F460EE662E6FEF762E6FEF5D
:109D7000862E6FEF962E91E2A916B104C104D1048C
:109D80002CF050E2A52EB12CC12CD12CA0EEAA169D
:109D9000AFEFBA06AFEFCA06AFEFDA0644F440EE13
:109DA000A42E4FEFB42E4FEFC42E4FEFD42E809140
:109DB000550390915603A0915703B091580386190B
:109DC0009709A809B9098093550390935603A09366
:109DD0005703B093580380914D0390914E03A09187
:109DE0004F03B09150038A199B09AC09BD098093B8
:109DF0004D0390934E03A0934F03B0935003809173
:109E00003702909138028F3F910509F008F4C4C5DC
:109E1000BB85BB2309F04EC580910703882309F059
:109E200049C580912D03882309F044C5E09162065D
:109E3000EC87EE2309F43EC58091D9079091DA07AB
:109E4000A091DB07B091DC07B7FF04C081509F4FA2
:109E5000AF4FBF4FE92EFA2E0B2F112707FD1A9592
:109E6000E092D907F092DA070093DB071093DC0742
:109E70008091E1079091E207A091E307B091E40798
:109E8000B7FF04C081509F4FAF4FBF4F892F9A2F0C
:109E9000AB2FBB27A7FDBA958D879E87AF87B88B61
:109EA0008093E1079093E207A093E307B093E40760
:109EB00080913A06A82EBB24CC24DD242091650392
:109EC000309166034091670350916803C601B50164
:109ED0000E942D7897FF04C061507F4F8F4F9F4F96
:109EE000672E782E892E992487FC9A9460926503B8
:109EF00070926603809267039092680320916103D9
:109F0000309162034091630350916403C601B5012F
:109F10000E942D7897FF04C061507F4F8F4F9F4F55
:109F2000272E382E492E552447FC5A94209261033F
:109F300030926203409263035092640380915D0308
:109F400090915E03A0915F03B0916003B7FF04C0DE
:109F500081509F4FAF4FBF4F892F9A2FAB2FBB27F9
:109F6000A7FDBA9580935D0390935E03A0935F0372
:109F7000B0936003D801C70186199709A809B909E8
:109F80008093B2039093B303A093B403B093B5034B
:109F900020916106E22EFF2400271127BC01CD018C
:109FA000A80197010E94A17859016A012093C10379
:109FB0003093C2034093C3035093C4038D859E85A1
:109FC000AF85B88982199309A409B5098093B603AE
:109FD0009093B703A093B803B093B903BC01CD012C
:109FE000A80197010E94A1782093C5033093C6036E
:109FF0004093C7035093C803D601C501D7FE04C0E0
:10A0000081509F4FAF4FBF4F892F9A2FAB2FBB2748
:10A01000A7FDBA9590930C0380930B0357FF04C0E0
:10A0200021503F4F4F4F5F4FBB2757FDBA95A52F8C
:10A03000942F832F90930E0380930D038091F2024F
:10A040009091F30281349105DCF48091F0029091BB
:10A05000F10281349105A4F480912206E82FFF27B4
:10A06000EE0FFF1FE75BF84F808191810190F08137
:10A07000E02DF7FF03C0F095E195FF4F7A97E4F0EC
:10A08000809181088F3FC1F480910B0390910C0364
:10A0900097FD01969595879590930C0380930B03FC
:10A0A00080910D0390910E0397FD019695958795EC
:10A0B00090930E0380930D038091D0079091D10768
:10A0C000A091D207B091D307B7FF04C081509F4F32
:10A0D000AF4FBF4F892F9A2FAB2FBB27A7FDBA9544
:10A0E0008093D0079093D107A093D207B093D30762
:10A0F0008091C2079091C307A091C407B091C50792
:10A10000B7FF04C081509F4FAF4FBF4F892F9A2F89
:10A11000AB2FBB27A7FDBA958093C2079093C307C7
:10A12000A093C407B093C5078091750390917603FF
:10A13000A0917703B09178032B813C814D815E81A2
:10A14000281B390B4A0B5B0B2093AA033093AB03FC
:10A150004093AC035093AD0380916D0390916E03D7
:10A16000A0916F03B0917003EF80F88409851A8580
:10A17000E81AF90A0A0B1B0BE092AE03F092AF0348
:10A180000093B0031093B1032093B2033093B30351
:10A190004093B4035093B503E092B603F092B70333
:10A1A0000093B8031093B903809151039091520327
:10A1B000A0915303B0915403821B930BA40BB50BD6
:10A1C0008093510390935203A0935303B09354038D
:10A1D0008091490390914A03A0914B03B0914C03A5
:10A1E0008E199F09A00BB10B8093490390934A03EA
:10A1F000A0934B03B0934C03FC85FF23E1F0209127
:10A200002B0330912C03213831054CF080918603CB
:10A21000909187030196909387038093860320583B
:10A220003F4F4CF480918603909187030197909360
:10A2300087038093860310922C0310922B0381E0F6
:10A2400090E09093CE038093CD03E090B203F09022
:10A25000B3030091B4031091B503D801C70117FFF0
:10A2600007C088279927DC018E199F09A00BB10B25
:10A2700081509240A040B04034F084E090E0909350
:10A28000CE038093CD038091D3039091D403A0910A
:10A29000D503B091D6032091D9073091DA074091C8
:10A2A000DB075091DC07821B930BA40BB50B815E7F
:10A2B000914BAF4FBF4F8F539C49A040B04028F007
:10A2C0008091820889310CF4FFC041E0E41640E13E
:10A2D000F40640E0040740E014070CF473C08091DA
:10A2E000CF03882309F46AC0D801C70117FF07C04C
:10A2F00088279927DC018E199F09A00BB10B9C01BF
:10A30000AD01B7FF04C021503E4F4F4F5F4FF9E002
:10A310005595479537952795FA95D1F78091CD03B7
:10A320009091CE03820F931F9093CE038093CD0321
:10A33000D801C70117FF03C00796A11DB11DE3E0B7
:10A34000B595A79597958795EA95D1F78093C10321
:10A350009093C203A093C303B093C403895893415D
:10A36000A040B04064F088E893E1A0E0B0E08093C2
:10A37000C1039093C203A093C303B093C40320917D
:10A38000C1033091C2034091C3035091C40357FFEE
:10A3900004C021503F4F4F4F5F4F232F342F452F85
:10A3A000552747FD5A9580910B0390910C03820F1E
:10A3B000931F90930C0380930B0306C081E080935E
:10A3C000CF0302C01092CF0360E0E61660EFF606FE
:10A3D0006FEF06076FEF16070CF073C08091D00384
:10A3E000882309F46AC0D801C70117FF07C088276E
:10A3F0009927DC018E199F09A00BB10B9C01AD01BF
:10A40000B7FF04C021503E4F4F4F5F4F69E0559555
:10A410004795379527956A95D1F78091CD0390910F
:10A42000CE03820F931F9093CE038093CD03D80168
:10A43000C70117FF03C00796A11DB11D23E0B59505
:10A44000A795979587952A95D1F78093C103909307
:10A45000C203A093C303B093C40388579C4EAF4F6D
:10A46000BF4F64F488E79CEEAFEFBFEF8093C1036A
:10A470009093C203A093C303B093C4032091C1037C
:10A480003091C2034091C3035091C40357FF04C0ED
:10A4900021503F4F4F4F5F4F232F342F452F5527CC
:10A4A00047FD5A9580910B0390910C03820F931FE7
:10A4B00090930C0380930B0311C081E08093D00331
:10A4C0000DC01092D0030AC01092CE031092CD039B
:10A4D00088EE93E09093DE018093DD018C85282F38
:10A4E00033278091CD039091CE032817390724F4A8
:10A4F0003093CE032093CD0310918208112379F07D
:10A50000212F332727FD30958091CD039091CE03E5
:10A510002817390724F43093CE032093CD034091BC
:10A52000B2035091B3036091B4037091B503413805
:10A5300051056105710574F080918A0390918B0338
:10A540002091CD033091CE03820F931F90938B0304
:10A5500080938A0340585F4F6F4F7F4F74F4809110
:10A560008A0390918B032091CD033091CE03821BFF
:10A57000930B90938B0380938A0381E090E09093F8
:10A58000CE038093CD03C090B603D090B703E09084
:10A59000B803F090B903D701C601F7FE07C08827BA
:10A5A0009927DC018C199D09AE09BF0981509240A1
:10A5B000A040B04034F084E090E09093CE038093CC
:10A5C000CD038091D7039091D803A091D903B09186
:10A5D000DA032091E1073091E2074091E3075091BF
:10A5E000E407821B930BA40BB50B815E914BAF4F1D
:10A5F000BF4F8F539C49A040B04018F019310CF464
:10A60000FFC001E0C01600E1D00600E0E00600E077
:10A61000F0060CF473C08091D103882309F46AC05A
:10A62000D701C601F7FE07C088279927DC018C19DE
:10A630009D09AE09BF099C01AD01B7FF04C02150BF
:10A640003E4F4F4F5F4F09E05595479537952795FA
:10A650000A95D1F78091CD039091CE03820F931F7D
:10A660009093CE038093CD03D701C601F7FE03C0BC
:10A670000796A11DB11D13E0B595A79597958795F0
:10A680001A95D1F78093C5039093C603A093C7038F
:10A69000B093C80389589341A040B04064F088E863
:10A6A00093E1A0E0B0E08093C5039093C603A0932C
:10A6B000C703B093C8032091C5033091C6034091EE
:10A6C000C7035091C80357FF04C021503F4F4F4F5D
:10A6D0005F4F232F342F452F552747FD5A958091E3
:10A6E0000D0390910E03820F931F90930E0380939E
:10A6F0000D0306C081E08093D10302C01092D10304
:10A7000020E0C21620EFD2062FEFE2062FEFF2066E
:10A710000CF073C08091D203882309F46AC0D7017A
:10A72000C601F7FE07C088279927DC018C199D090F
:10A73000AE09BF099C01AD01B7FF04C021503E4FD7
:10A740004F4F5F4FE9E05595479537952795EA9527
:10A75000D1F78091CD039091CE03820F931F9093F8
:10A76000CE038093CD03D701C601F7FE03C0079641
:10A77000A11DB11D73E0B595A795979587957A951D
:10A78000D1F78093C5039093C603A093C703B093FA
:10A79000C80388579C4EAF4FBF4F64F488E79CEEC8
:10A7A000AFEFBFEF8093C5039093C603A093C70399
:10A7B000B093C8032091C5033091C6034091C703ED
:10A7C0005091C80357FF04C021503F4F4F4F5F4F78
:10A7D000232F342F452F552747FD5A9580910D0380
:10A7E00090910E03820F931F90930E0380930D039D
:10A7F00011C081E08093D2030DC01092D2030AC031
:10A800001092CE031092CD0388EE93E09093DE0178
:10A810008093DD014C85242F33278091CD039091C7
:10A82000CE032817390724F43093CE032093CD03A9
:10A8300080918208882379F0282F332727FD3095CF
:10A840008091CD039091CE032817390724F43093DB
:10A85000CE032093CD034091B6035091B70360918E
:10A86000B8037091B903413851056105710574F061
:10A8700080918803909189032091CD033091CE037C
:10A88000820F931F909389038093880340585F4FF2
:10A890006F4F7F4FCCF48091880390918903209172
:10A8A000CD033091CE03821B930B90938903809349
:10A8B00088030AC010920E0310920D0310920C032D
:10A8C00010920B0310922D038091E607882341F428
:10A8D00010920E0310920D0310920C0310920B03B2
:10A8E0008091D9079091DA07A091DB07B091DC073E
:10A8F0008093D3039093D403A093D503B093D6034E
:10A900008091E1079091E207A091E307B091E407FD
:10A910008093D7039093D803A093D903B093DA031D
:10A9200010926503109266031092670310926803F9
:10A9300010926103109262031092630310926403F9
:10A9400010925D0310925E0310925F0310926003F9
:10A950001092D9071092DA071092DB071092DC07E9
:10A960001092E1071092E2071092E3071092E407B9
:10A970001092D0071092D1071092D2071092D307ED
:10A980001092C2071092C3071092C4071092C50715
:10A990001092380210923702E0901B03F0901C03D3
:10A9A000C701F7FE04C0882799278E199F09409791
:10A9B0006CF088EE93E09093DE018093DD0180914E
:10A9C0002B0684FD03C081E08093C00310913706FD
:10A9D000A12EBB24CC24DD24B701882777FD8095E8
:10A9E000982F9701F7FE04C0222733272E193F091D
:10A9F000442737FD4095542F0E942D789B01AC01D0
:10AA0000C601B5010E942D7897FF04C061507E4FAA
:10AA10008F4F9F4F59E095958795779567955A95F4
:10AA2000D1F79B01812F99278E9DD0018F9DB00D6D
:10AA30009E9DB00D1124CD01B7FD03969595879588
:10AA400095958795280F391F442737FD4095542F3A
:10AA50002093A6033093A7034093A8035093A90320
:10AA60008091450390914603A0914703B09148031C
:10AA7000821B930BA40BB50B809345039093460365
:10AA8000A0934703B09348038155934CA040B04036
:10AA900064F080E593ECA0E0B0E0809345039093F0
:10AAA0004603A0934703B0934803809145039091D8
:10AAB0004603A0914703B0914803805B9C43AF4F8E
:10AAC000BF4F64F480EB9CE3AFEFBFEF809345038F
:10AAD00090934603A0934703B093480340903303F9
:10AAE000509034034114510409F478C180912B062D
:10AAF00083FF74C18091750390917603A0917703D1
:10AB0000B0917803B7FF04C081509E4FAF4FBF4F45
:10AB100039E0B595A795979587953A95D1F76C014A
:10AB200097FF04C0D094C194D108D39480916D0351
:10AB300090916E03A0916F03B0917003B7FF04C0B2
:10AB400081509E4FAF4FBF4F29E0B595A795979580
:10AB500087952A95D1F7BC0197FF03C07095619541
:10AB60007F4FC616D7060CF46B01B601D7FE02C0A4
:10AB7000695F7F4F3B0183E0759467948A95E1F7A5
:10AB800002E0E02EF12C6E0C7F1C0CE112E0400E76
:10AB9000511E72010027F7FC0095102F24EE3DEFA7
:10ABA000420E531E80910F0890911008A091110839
:10ABB000B091120880909A0190909B01A0909C0106
:10ABC000B0909D01BC01CD01A50194010E94A17826
:10ABD000E21AF30A040B150BC801B70128E631E0AD
:10ABE00040E050E00E94A178DC01CB011CE4E12EA2
:10ABF0001FEFF12EE80EF91E0091DD011091DE012C
:10AC00000115110589F539E1C316D1046CF5809160
:10AC10002B0390912C038E0D9F1D90932C038093FA
:10AC20002B038091C0038823F9F0C201AA2797FD66
:10AC3000A095BA2FBC01CD01A50194010E942D78E9
:10AC4000DC01CB0180930F0890931008A0931108AA
:10AC5000B0931208BC01CD010E94A1783093320359
:10AC6000209331031092C003C701B4E0880F991FED
:10AC7000BA95E1F7B3010E946C78CB01AA2797FD42
:10AC8000A095BA2F20910F0830911008409111081B
:10AC900050911208280F391F4A1F5B1F20930F087D
:10ACA000309310084093110850931208F090CE0191
:10ACB0006F2D7727C69EC001C79E900DD69E900D22
:10ACC000112497FD4F966C01A5E0D594C794AA95E1
:10ACD000E1F76C197D096B0177FD7AC0011511054B
:10ACE00009F06FC00091F2021091F3028091F0021E
:10ACF0009091F102080F191F17FF02C0095F1F4F43
:10AD0000F3E015950795FA95E1F7005C1F4FCA012E
:10AD1000B901A50194010E94A178DA01C90120912D
:10AD2000310330913203442737FD4095542F821B65
:10AD3000930BA40BB50B845E9D4FAF4FBF4FBC016F
:10AD4000CD0128E631E040E050E00E94A178DC012E
:10AD5000CB01845B90408C9DA0018D9D500D9C9DEE
:10AD6000500D1124CA01B8010E946C7883E0F89E4E
:10AD700060011124C616D70614F4B60108C088274E
:10AD800099278C199D09681779070CF4BC019B0160
:10AD9000442737FD4095542F8091450390914603F9
:10ADA000A0914703B0914803820F931FA41FB51FC2
:10ADB0008093450390934603A0934703B0934803C1
:10ADC0000DC0015010401093DE010093DD0106C05C
:10ADD00084EF91E09093DE018093DD0180912D035B
:10ADE000882381F01092390310923A0310923B03AA
:10ADF00010923C0310923D0310923E0310923F03C9
:10AE000010924003F0900803FF20F1F48091E607D0
:10AE1000282F332744275527809175039091760377
:10AE2000A0917703B0917803BC01CD010E942D78E9
:10AE3000DC01CB01BC01CD0128EF3AE240E050E05B
:10AE40000E94A178390102C066247724E0900703AC
:10AE5000EE20F1F48091E607282F33274427552769
:10AE600080916D0390916E03A0916F03B091700378
:10AE7000BC01CD010E942D78DC01CB01BC01CD01CC
:10AE800028EF3AE240E050E00E94A178290102C098
:10AE9000442455248091BC079091BD07893C9105BD
:10AEA0001CF088EC90E005C088539F4F34F488E391
:10AEB0009FEF9093BD078093BC078091C707909147
:10AEC000C807893C91051CF088EC90E005C08853C8
:10AED0009F4F34F488E39FEF9093C8078093C70790
:10AEE0008091C9079091CA07AA2797FDA095BA2F0C
:10AEF00020910D08A22EBB24CC24DD24BC01CD0161
:10AF0000A60195010E942D789B01AC018091BC07A0
:10AF10009091BD07AA2797FDA095BA2FE7E0880F6B
:10AF2000991FAA1FBB1FEA95D1F7280F391F4A1F87
:10AF30005B1F57FF04C0215C3F4F4F4F5F4F76E0D0
:10AF400055954795379527957A95D1F78301020F47
:10AF5000131F1093CA070093C9078091BA079091F5
:10AF6000BB07AA2797FDA095BA2FBC01CD01A6016A
:10AF700095010E942D789B01AC018091C7079091AB
:10AF8000C807AA2797FDA095BA2F67E0880F991FD9
:10AF9000AA1FBB1F6A95D1F7280F391F4A1F5B1FD5
:10AFA00057FF04C0215C3F4F4F4F5F4F96E05595D0
:10AFB0004795379527959A95D1F74201820E931EB2
:10AFC0009092BB078092BA07809108089091090877
:10AFD000880F991FAA2797FDA095BA2F2091C10726
:10AFE000332744275527BC01CD010E942D785B01F2
:10AFF0006C0197FF08C08FE390E0A0E0B0E0A80EDE
:10B00000B91ECA1EDB1E86E0D594C794B794A794D8
:10B010008A95D1F78091D607282F332744275527C3
:10B020008091590390915A03A0915B03B0915C0306
:10B03000BC01CD010E942D78DC01CB01BC01CD010A
:10B0400020EF35E540E050E00E94A178B501620FA5
:10B05000731F70930908609308080150104134F081
:10B0600080E090E19093CA078093C9078091C90757
:10B070009091CA078050904F34F480E090EF909305
:10B08000CA078093C907B1E08B16B0E19B0634F084
:10B0900080E090E19093BB078093BA078091BA0754
:10B0A0009091BB078050904F34F480E090EF9093E4
:10B0B000BB078093BA076150704134F080E090E1A3
:10B0C00090930908809308088091080890910908D6
:10B0D0008050904F34F480E090EF90930908809373
:10B0E000080880910001482F552780911E019091FA
:10B0F0001F014817590794F420911E0130911F0138
:10B1000069817A81649FC001659F900D749F900D45
:10B110001124B9010E9458787A83698389819A81C0
:10B12000880F991F880F991F9A83898340912B0656
:10B1300040FFBDC6EE2009F0BAC6FF2009F0B7C631
:10B14000AA24BB2445018091090390910A0390939E
:10B15000F4058093F30520918C0330918D03211524
:10B16000310509F03FC08091140190911501895972
:10B17000934058F087B5853F20F480913B02815081
:10B1800011C081E08093E6034EC08091140190913C
:10B1900015018436910508F587B58B30D0F0809184
:10B1A0003B028F5F80933B029AE089029001112459
:10B1B00080911A06821B87BD8CE291E09093290250
:10B1C000809328028EE591E090938D0380938C0309
:10B1D0002AC081E08093E50326C0F092E503F09257
:10B1E000E60321C08091130390911403A0911503ED
:10B1F000B091160314E0880F991FAA1FBB1F1A9560
:10B20000D1F780933C0290933D02A0933E02B0930D
:10B210003F02B0923A02A09239022150304030935E
:10B220008D0320938C032091D10141FF24C0223350
:10B23000D8F48091E30181508093E3018F3FD9F5E9
:10B2400010922E038091130390911403A091150383
:10B25000B091160380930F0390931003A0931103F2
:10B26000B093120381E004C081E080932E0388EC48
:10B270008093E30120C080919E0190919F01820FF5
:10B28000911D209130063327829FF001839FF00D9E
:10B29000929FF00D1124CF01AA2797FDA095BA2FF8
:10B2A00080930F0390931003A0931103B0931203A4
:10B2B00081E080932E038091750390917603A09195
:10B2C0007703B0917803E0909A01F0909B01009190
:10B2D0009C0110919D01BC01CD01A80197010E9424
:10B2E000A17859016A0180916D0390916E03A0913C
:10B2F0006F03B0917003BC01CD01A80197010E94BA
:10B30000A178B901C5010E94576F8C01CC9714F048
:10B310000CE310E0C8010E94526B8C0180E2809324
:10B32000990180912E03882309F447C48091ED028E
:10B3300099279C012071307084FD3FC46091840680
:10B3400060FD04C080912B0681FD0CC0C980DA80AD
:10B350003093DC032093DB038091ED02806C8093BB
:10B36000ED0299C18091ED0281FF6BC14091DF0137
:10B370005091E001CA010F962091190330911A03F0
:10B3800082179307BCF58091E503882399F5809196
:10B39000ED0287FF15C08091ED028F778093ED025B
:10B3A0008091130390911403A0911503B09116039B
:10B3B00080930F0390931003A0931103B093120393
:10B3C0008091ED0280648093ED02241B350B2F5099
:10B3D000304037FF03C0309521953F4F8091DB030C
:10B3E0009091DC03820F931F9093DC038093DB0327
:10B3F0008BE26EC0CA010F9728173907BCF5809100
:10B40000E603882399F58091ED0286FF15C08091AF
:10B41000ED028F7B8093ED028091130390911403D2
:10B42000A0911503B091160380930F03909310031E
:10B43000A0931103B09312038091ED028068809372
:10B44000ED02241B350B215F3F4F37FF03C03095C2
:10B4500021953F4F8091DB039091DC03821B930B7E
:10B460009093DC038093DB038DE232C08091ED0288
:10B47000807C69F18091ED028F738093ED021092D0
:10B48000DC031092DB0320911303309114034091ED
:10B4900015035091160320930F033093100340932C
:10B4A00011035093120361FF06C084EF91E0909363
:10B4B00029028093280280911703882341F42333C3
:10B4C0003105410551051CF081E0809317038DE3A0
:10B4D000809399012091DB033091DC03C90137FF90
:10B4E00004C088279927821B930B815092400CF44B
:10B4F00091C0809130069927289F7001299FF00CF8
:10B50000389FF00C1124C70160E075E00E946C7850
:10B51000CB01AA2797FDA095BA2F20910F03309158
:10B5200010034091110350911203280F391F4A1F35
:10B530005B1F20930F03309310034093110350932C
:10B5400012031092DC031092DB03C0901303D0901F
:10B550001403E0901503F0901603D701C601805044
:10B560009440A040B04082179307A407B5075CF44D
:10B57000D701C60180509C4FAF4FBF4F28173907E6
:10B580004A075B0744F080930F0390931003A09346
:10B590001103B09312038091840681FF06C084E6F4
:10B5A00090E09093290280932802809134068823AA
:10B5B00089F54091090350910A0357FF02C04D5F7E
:10B5C0005F4F559547955595479580911E019091F0
:10B5D0001F01209100013327489FB001499F700D42
:10B5E000589F700D1124CB01B9010E946C787093A3
:10B5F000E0016093DF01663471051CF486E490E09D
:10B6000005C06739710534F086E990E09093E00158
:10B610008093DF0180918C0390918D03892BB9F188
:10B620008091130390911403A0911503B091160318
:10B6300080930F0390931003A0931103B093120310
:10B6400026C08091130390911403A0911503B0912B
:10B65000160380599140A040B04080930F0390930F
:10B660001003A0931103B093120380913406882332
:10B6700011F0992702C088E790E09093E001809351
:10B68000DF0189819A8190930A0380930903C09016
:10B690000903D0900A0320911303309114034091C1
:10B6A0001503509116032B8B3C8B4D8B5E8B209199
:10B6B0000F033091100340911103509112036B89D5
:10B6C0007C898D899E89261737074807590724F0FA
:10B6D0008091840680FDB8C280918C0390918D0387
:10B6E000892B39F0C0900903D0900A03AA24BB2407
:10B6F000D9C08B899C89AD89BE89821B930BA40B11
:10B70000B50B8093AA039093AB03A093AC03B093C3
:10B71000AD03823070E897077FEFA7077FEFB70789
:10B720002CF481E090E8AFEFBFEF09C08F5F9F4737
:10B73000A040B04064F08FEF9FE7A0E0B0E08093BE
:10B74000AA039093AB03A093AC03B093AD03A09076
:10B75000AA03B090AB038091D001282F3327442750
:10B7600055278091AA039091AB03A091AC03B091AF
:10B77000AD03BC01CD010E942D7897FF04C0615E2E
:10B780007F4F8F4F9F4FA5E095958795779567954C
:10B79000AA95D1F76093AA037093AB038093AC038F
:10B7A0009093AD036530FEEF7F07FFEF8F07FFEF4C
:10B7B0009F072CF484E09EEFAFEFBFEF09C060500D
:10B7C00074408040904064F080E094E0A0E0B0E0FD
:10B7D0008093AA039093AB03A093AC03B093AD0303
:10B7E0008090AA039090AB032091390230913A02E5
:10B7F00037FF02C0295F3F4FF3E035952795FA9553
:10B80000E1F74FEF223834071CF421E83FEF05C081
:10B810002038310514F020E830E0C901AA2797FD4F
:10B82000A095BA2F2091D201332744275527BC0178
:10B83000CD010E942D7897FF04C06D5F7F4F8F4F21
:10B840009F4FE2E09595879577956795EA95D1F7B3
:10B850009B015FEF613075071CF420E03FEF06C0ED
:10B860006F3F710519F014F020E031E08091ED0296
:10B87000807C49F0C90137FD03969C0135952795D9
:10B88000359527950DC08091840680FF09C0C901B8
:10B8900037FD07969C0143E0359527954A95E1F7DA
:10B8A000820E931E2091CF01222309F454C060918F
:10B8B000350370913603809137039091380397FFD9
:10B8C00004C061587F4F8F4F9F4F37E09595879504
:10B8D000779567953A95D1F73327442755270E94E6
:10B8E0002D7897FF04C0615E7F4F8F4F9F4FB5E06B
:10B8F0009595879577956795BA95D1F76093AA0343
:10B900007093AB038093AC039093AD036138AFEFBA
:10B910007A07AFEF8A07AFEF9A072CF480E89FEF22
:10B92000AFEFBFEF0AC06F3F71058105910569F068
:10B9300064F080E091E0A0E0B0E08093AA039093EF
:10B94000AB03A093AC03B093AD038091AA03909195
:10B95000AB03880E991E8091CD01282F332780914B
:10B960008508992787FD9095289FF001299FF00D64
:10B97000389FF00D11249F01F7FF02C021583F4F5F
:10B98000220F232F221F330BFFEF21383F071CF418
:10B9900020E83FEF06C02F3F310519F014F020E0FA
:10B9A00031E0820E931EC401AA2797FDA095BA2FFD
:10B9B000E0900903F0900A039701442737FD409572
:10B9C000542FBC01CD010E942D7897FF04C0615017
:10B9D0007E4F8F4F9F4FF9E09595879577956795A7
:10B9E000FA95D1F7C61AD70A8091DB039091DC0350
:10B9F000892B09F060C01E141F040CF05CC0950177
:10BA0000B7FE03C0309521953F4F2D33310540F4EB
:10BA10008091DF039091E0038C159D0574F526C09D
:10BA20002C533040E5E036952795EA95E1F7203133
:10BA3000310510F02FE030E04091DF035091E0033A
:10BA40001A141B04E4F480E190E0821B930B489FDE
:10BA50009001499F300D589F300D112474E03695A8
:10BA600027957A95E1F72C153D0520F58091E101A8
:10BA70009091E201C816D906F4F06C011CC0205F59
:10BA80003F4F8091E1019091E201829FB001839F3D
:10BA9000700D929F700D11249B0164E036952795DF
:10BAA0006A95E1F74C155D0514F06A0104C0C216F1
:10BAB000D30608F06901C601AA2797FDA095BA2F01
:10BAC0002DE0880F991FAA1FBB1F2A95D1F7980157
:10BAD000442737FD4095542FBC01CD010E94A17829
:10BAE0002093AE033093AF034093B0035093B10360
:10BAF000C090AE03D090AF038091DD039091DE0340
:10BB00009C01220F331F280F391F2C0D3D1D37FFBD
:10BB100002C02D5F3F4FA901559547955595479513
:10BB20005093DE034093DD0380912C06282F3327AA
:10BB3000220F331F220F331F241735076CF4809117
:10BB40000708282F3327220F331F220F331F2055BA
:10BB500030404217530724F03093DE032093DD0377
:10BB60008091840680FF14C08091DD039091DE03F4
:10BB7000A981BA818A179B0724F0B093DE03A093B2
:10BB8000DD03E091DD03F091DE03FA83E9835CC01D
:10BB900029813A812E193F0937FF02C02D5F3F4F9F
:10BBA0003595279535952795E090DD03F090DE03D8
:10BBB000E20EF31EFA82E98247C0809134068823A0
:10BBC00001F56091090370910A0377FF02C06D5F70
:10BBD0007F4F759567957595679540911E015091BA
:10BBE0001F0180910001282F3327649FC001659FAA
:10BBF000900D749F900D1124B9010E946C78CB01B7
:10BC000001C099279093E0018093DF018091DF01CB
:10BC10009091E001873491051CF486E490E005C022
:10BC20008639910534F086E990E09093E0018093A5
:10BC3000DF0129813A813093DE032093DD03809177
:10BC4000ED02806C8093ED028091ED0299279C01BA
:10BC50002270307081FF1CC18091E1039091E2035A
:10BC6000A091E303B091E4030097A105B10521F091
:10BC7000809117038130B1F449815A81CA01AA2702
:10BC800097FDA095BA2F2EE0880F991FAA1FBB1F02
:10BC90002A95D1F78093E1039093E203A093E30305
:10BCA000B093E40380911703813019F482E080930C
:10BCB000170369817A81CB01AA2797FDA095BA2F36
:10BCC0009801442737FD4095542FBC01CD010E94B7
:10BCD0002D78DC01CB018093AE039093AF03A0934A
:10BCE000B003B093B103B7FF04C08150904EAF4F83
:10BCF000BF4F7C018D01FDE015950795F794E79402
:10BD0000FA95D1F7E092AE03F092AF030093B0033F
:10BD10001093B1036091EE027091EF028FE0603AF0
:10BD2000780750F58091E1039091E203A091E3033D
:10BD3000B091E4039C01AD01EAE056954795379533
:10BD40002795EA95D1F7821B930BA40BB50BA8019D
:10BD50009701F4E0220F331F441F551FFA95D1F7C6
:10BD6000820F931FA41FB51F8093E1039093E203FA
:10BD7000A093E303B093E40360547F4118F58091EE
:10BD8000E1039091E203A091E303B091E4039C01ED
:10BD9000AD01ECE05695479537952795EA95D1F793
:10BDA000821B930BA40BB50BA801970172E0220F25
:10BDB000331F441F551F7A95D1F7820F931FA41F7D
:10BDC000B51F29C08091390290913A0280913902C1
:10BDD00090913A0297FF03C0909581959F4F8436CA
:10BDE00091050CF58091E1039091E203A091E303AA
:10BDF000B091E4039C01AD016EE0569547953795EF
:10BE000027956A95D1F7821B930BA40BB50B8E0D6A
:10BE10009F1DA01FB11F8093E1039093E203A093A5
:10BE2000E303B093E4038091E1039091E203A091D6
:10BE3000E303B091E4031EE0B695A7959795879527
:10BE40001A95D1F790930A03809309034091320623
:10BE5000442399F055279C01BA010E946C78C901CE
:10BE6000861B970B9093E0038093DF03260F371F09
:10BE70003093E2012093E1011FC01092E003109281
:10BE8000DF038FEF93E09093E2018093E10114C010
:10BE9000109217031092E1031092E2031092E30351
:10BEA0001092E40330930A032093090305C08091A4
:10BEB000ED02806C8093ED022090CE07222D332777
:10BEC000220F331F220F331F285D3F4FA981BA81F4
:10BED0002A173B0714F03A83298330900708832DF3
:10BEE0009927880F991F880F991F80559040E981E5
:10BEF000FA818E179F0714F49A83898380917102C7
:10BF0000882321F4809197088F3FA1F08091EE0261
:10BF10009091EF020297C09768F4E980FA801E14AE
:10BF20001F0444F481E090E09093EF028093EE02CE
:10BF30003A83298309811A811093D8050093D70584
:10BF40008091A6039091A703A091A803B091A903A3
:10BF5000F2E0880F991FAA1FBB1FFA95D1F7009135
:10BF6000080810910908081B190B29813A81213A08
:10BF700031058CF0C90137FD01969595879580179D
:10BF800091070CF48C01909581959F4F0817190724
:10BF90006CF48C010BC00135110514F000E510E0C4
:10BFA0003FEF003B130714F400EB1FEF232D332763
:10BFB000220F331F220F331FC90149815A81841B6D
:10BFC000950B801791070CF48C0169817A81621BB3
:10BFD000730B061717070CF48B018091C90790911A
:10BFE000CA0760911F0370912003861B970B9093E3
:10BFF000D8078093D707D090E60720913D03309172
:10C000003E0340913F0350914003DD2041F0661A0A
:10C01000770AC301AA2797FDA095BA2F04C0AA27C3
:10C0200097FDA095BA2F280F391F4A1F5B1F209339
:10C030003D0330933E0340933F0350934003809170
:10C040003D0390913E03A0913F03B0914003815086
:10C050009A4FA040B04064F080E09AEFA0E0B0E0DA
:10C0600080933D0390933E03A0933F03B09340031E
:10C0700080913D0390913E03A0913F03B091400316
:10C0800080509640AF4FBF4F64F480E096E0AFEF32
:10C09000BFEF80933D0390933E03A0933F03B09383
:10C0A0004003C09041062091D7073091D807F8E0AF
:10C0B000FC1598F08C2D9927829F7001839FF00CBE
:10C0C000929FF00C1124C701F7FC07967C0163E0F6
:10C0D000F594E7946A95E1F712C08C2D869599271F
:10C0E000829FA001839F500D929F500D1124CA0181
:10C0F00057FD03967C01F594E794F594E794A0909E
:10C10000D301B090D4019501442737FD4095542FB9
:10C1100080913D0390913E03A0913F03B091400375
:10C12000BC01CD010E94A178E20EF31E9090BF01E8
:10C13000692D772788279927980117FF04C02227A0
:10C140003327201B310B37FF02C02F5F3F4F359540
:10C150002795A981BA812A0F3B1F442737FD4095B7
:10C16000542F0E942D7897FF04C0615C7F4F8F4F42
:10C170009F4F26E095958795779567952A95D1F7F6
:10C180009B016E157F050CF47B01309521953F4F87
:10C19000E216F3060CF479018091BA079091BB077F
:10C1A00060911D0370911E03861B970B9093B90736
:10C1B0008093B8072091390330913A0340913B03B3
:10C1C00050913C03DD2041F0461A570AC201AA27CC
:10C1D00097FDA095BA2F04C0AA2797FDA095BA2F66
:10C1E000280F391F4A1F5B1F2093390330933A03EE
:10C1F00040933B0350933C038091390390913A0361
:10C20000A0913B03B0913C0381509A4FA040B040B5
:10C2100064F080E09AEFA0E0B0E08093390390935F
:10C220003A03A0933B03B0933C0380913903909170
:10C230003A03A0913B03B0913C0380509640AF4F2E
:10C24000BF4F64F480E096E0AFEFBFEF8093390317
:10C2500090933A03A0933B03B0933C032091B8071B
:10C260003091B90748E04C1598F08C2D9927829FA2
:10C27000B001839F700D929F700D1124CB0177FD4B
:10C2800007966C01B3E0D594C794BA95E1F712C054
:10C29000C6948C2D9927829FD001839FB00D929FC9
:10C2A000B00D1124CD01B7FD03966C01D594C79450
:10C2B000D594C7949501442737FD4095542F80911C
:10C2C000390390913A03A0913B03B0913C03BC0128
:10C2D000CD010E94A178C20ED31E692D7727882731
:10C2E0009927980117FF04C022273327201B310B01
:10C2F00037FF02C02F5F3F4F35952795E981FA81BF
:10C300002E0F3F1F442737FD4095542F0E942D7854
:10C3100097FF04C0615C7F4F8F4F9F4FE6E095957C
:10C32000879577956795EA95D1F79B016C157D0503
:10C330000CF46B01309521953F4FC216D3060CF4D7
:10C34000690168EE862E66E0962E5FE9A52E56E01E
:10C35000B52E4BE0542E37EE632E37E0732ED50109
:10C360002C9112160CF014C1203429F4E981FA81C1
:10C37000F88FEF8B1FC049815A81CA01AA2797FD08
:10C38000A095BA2F332727FD3095432F532FBC019B
:10C39000CD010E942D7897FF04C0615C7F4F8F4FC5
:10C3A0009F4F26E095958795779567952A95D1F7C4
:10C3B000788F6F8BF5012181203439F42F89388DE6
:10C3C0002E0D3F1D388F2F8B2AC0203C39F44F890A
:10C3D000588D4E195F09588F4F8B21C0C701AA276E
:10C3E00097FDA095BA2F332727FD3095432F532F64
:10C3F000BC01CD010E942D7897FF04C0615C7F4F86
:10C400008F4F9F4FB6E09595879577956795BA952D
:10C41000D1F7AF89B88DA60FB71FB88FAF8BF501D5
:10C420002281203439F42F89388D2C0D3D1D388F11
:10C430002F8B2AC0203C39F44F89588D4C195D0947
:10C44000588F4F8B21C0C601AA2797FDA095BA2F00
:10C45000332727FD3095432F532FBC01CD010E9478
:10C460002D7897FF04C0615C7F4F8F4F9F4FA6E0F0
:10C470009595879577956795AA95D1F7AF89B88DEA
:10C48000A60FB71FB88FAF8BF5012381203439F485
:10C490002F89388D200F311F388F2F8B2AC0203CD9
:10C4A00039F44F89588D401B510B588F4F8B21C049
:10C4B000C801AA2797FDA095BA2F332727FD3095ED
:10C4C000432F532FBC01CD010E942D7897FF04C04C
:10C4D000615C7F4F8F4F9F4FF6E0959587957795DD
:10C4E0006795FA95D1F7AF89B88DA60FB71FB88FAA
:10C4F000AF8BF301808191812F89388D821793074B
:10C5000064F4B901680F791F77FF02C06F5F7F4F36
:10C5100075956795788F6F8B08C04F89588D440F3C
:10C52000551F481B590B588F4F8B822D9927880F09
:10C53000991F880F991F6F89788D861797075CF46C
:10C54000832D9927880F991F880F991FAF89B88D60
:10C55000A817B90714F0988F8F8B8F89988D97FD46
:10C5600003969595879595958795F4018183880F16
:10C57000991F880F991F2F89388D281B390BC901E6
:10C58000880F8283EF89F88DD301ED93FC9303C06C
:10C59000F401118212825A9422E030E0620E731E7E
:10C5A00044E050E0A40EB51E68E070E0860E971ED1
:10C5B00057FED5CEE2E1C85E0C94D8788091F303A3
:10C5C0009091F403A091F503B091F6038093EB03EF
:10C5D0009093EC03A093ED03B093EE038091EF03EF
:10C5E0009091F003A091F103B091F2038093E703DF
:10C5F0009093E803A093E903B093EA03089510929F
:10C60000FE031092FD031092FC031092FB030895A9
:10C6100084B1806A84B93D9A82E58CBD1DBC459A7F
:10C6200081E0809319088AEA80932A0883E880933E
:10C630002B088AE080932C0810922E0810922D0867
:10C640001092300810922F081092840810924C0813
:10C65000089530911908332309F085C00DB407FE01
:10C6600082C084E080932702459A2EB5809102040F
:10C6700099278130910589F0823091051CF4892B2E
:10C6800021F03EC00297B9F03BC030934B08209395
:10C6900003042138A9F581E008C0253549F48091CB
:10C6A0000304820F8093030482E08093020428C075
:10C6B0003093020425C080914B08E82FFF27E959E9
:10C6C000F74F20838F5F80934B08909103048A314A
:10C6D000A0F0291769F48AE1A7E6B8E0EDE4F8E0F4
:10C6E0000D9001928A95E1F781E080934C0802C099
:10C6F00030934C081092020403C0920F90930304ED
:10C7000020912908203208F028C045980000000038
:10C710000000000000000000000000000000000019
:10C720000000000000000000000000000000000009
:10C73000000000000000000000000000E09122085E
:10C74000F0912308E20FF11D80818EBD8091490890
:10C750009081890F8093490803C081E08093190874
:10C760002F5F209329080895EF92FF920F931F9354
:10C7700080913A069927880F991F880F991F7C018D
:10C780000027F7FC0095102F809175039091760398
:10C79000A0917703B0917803BC01CD01A801970166
:10C7A0000E94A17830932E0820932D0880916D036C
:10C7B00090916E03A0916F03B0917003BC01CD0105
:10C7C000A80197010E94A1783093300820932F0888
:10C7D00020910F08309110084091110850911208D3
:10C7E000DA01C901E3E0880F991FAA1FBB1FEA9570
:10C7F000D1F7820F931FA41FB51F820F931FA41F91
:10C80000B51F20919A0130919B0140919C0150915C
:10C810009D01BC01CD010E94A17830933608209380
:10C8200035088091860390918703209147023091CB
:10C830004802821B930B90933C0880933B08E09145
:10C840007C03F0917D038091DE079091DF07BF01AB
:10C850000E946C78CB019B01220F331F220F331FE4
:10C86000280F391F280F391F37FF02C02D5F3F4F98
:10C8700035952795359527953093320820933108C3
:10C8800080910B0890910C08BF010E946C789B016D
:10C89000220F331F220F331F260F371F260F371F7C
:10C8A00037FF02C02D5F3F4F35952795359527956A
:10C8B000309334082093330810927D0310927C0348
:10C8C0001092DF071092DE0710920C0810920B08EE
:10C8D00080912C0899278D30910509F466C08E301F
:10C8E00091055CF48B30910509F48EC08C30910574
:10C8F0000CF00FC10A9761F0ADC18F30910509F4BA
:10C9000081C18F3091050CF45CC1409799F1A2C1AF
:10C910008091020380933D088091010380933E083B
:10C920008091000380933F088091FF02809340082C
:10C930008091FE02809341088091FD02809342081D
:10C940008091FC02809343088091FB02809344080D
:10C950008091ED02809345088091ED02837F809362
:10C96000ED020E94A22D8093460880917903809366
:10C97000470870C1809191089091920890933E0869
:10C9800080933D0880919508909196089093400877
:10C9900080933F0880911E0190911F018093410870
:10C9A000809100018093420855C180916E0680936A
:10C9B0003D0880916F0680933E08809170068093B9
:10C9C0003F088091710680934008809172068093A1
:10C9D0004108809176068093420880917706809383
:10C9E0004308809178068093440880917B06809369
:10C9F0004508809179068093460880917A06809355
:10CA0000470880917C06DAC0F89480912106E82FCF
:10CA1000FF27EE0FFF1FE75BF84F0190F081E02D3D
:10CA2000E038F1051CF0EFE7F0E006C02FEFE13849
:10CA3000F20714F4E1E8FFEFE0933D08809122064D
:10CA4000E82FFF27EE0FFF1FE75BF84F0190F08103
:10CA5000E02DE038F1051CF0EFE7F0E006C06FEFE5
:10CA6000E138F60714F4E1E8FFEFE0933E08809127
:10CA70002006E82FFF27EE0FFF1FE75BF84F01901E
:10CA8000F081E02DE038F1051CF0EFE7F0E006C0A2
:10CA90008FEFE138F80714F4E1E8FFEFE0933F0887
:10CAA00080911F06E82FFF27EE0FFF1FE75BF84F6F
:10CAB0000190F081E02DE038F1051CF0EFE7F0E0A7
:10CAC00006C02FEFE138F20714F4E1E8FFEF7894A5
:10CAD000E0934008809122038093410880912303D2
:10CAE000809342088091240380934308809125031A
:10CAF0008093440880912603809345088091270302
:10CB000080934608809128038093470880912903E9
:10CB100055C080916204863018F01092620485E05E
:10CB200080933D0880917D0680933E088091130399
:10CB300090911403A0911503B0911603BC01CD018F
:10CB400025E030E040E050E00E94A17830934008BA
:10CB500020933F0880910F0390911003A09111033F
:10CB6000B0911203BC01CD0125E030E040E050E07F
:10CB70000E94A17830934208209341088091730667
:10CB800080934308809174068093440880917506D1
:10CB9000809345088091210380934608809149073E
:10CBA00090914A07809347088091D7059091D805C6
:10CBB00097FD039695958795959587958093480859
:10CBC00049C010923D0882E580933E0810923F08CC
:10CBD00080E1809340088091020180934108809118
:10CBE00047048093420880914804809343088091D1
:10CBF00049048093440880914A04809345088091B9
:10CC00004B0426C08091530680933D088091830693
:10CC100080933E088091C50180933F0880914C0627
:10CC20008093400880914D068093410880914E0684
:10CC3000809342088091C4018093430880915006FC
:10CC40008093440880915106809345088091520654
:10CC50008093460880914C08882309F4D8C08AEF55
:10CC60008093ED0140914E0850914F08CA018150C8
:10CC70009E4F8F5F9340B0F420915008309151083F
:10CC8000C90181509E4F8F5F934060F480912B06C5
:10CC900085FF08C05093FE034093FD033093FC03CF
:10CCA0002093FB03809154089091550821E0893628
:10CCB000920724F4909334038093330380913303D9
:10CCC000909134032091310330913203821B930BF6
:10CCD000845E9D4F68E671E00E946C78845B9040B2
:10CCE0009093300380932F03209158083091590876
:10CCF00080912802909129028217930740F4809135
:10CD00006204882321F43093290220932802809121
:10CD10004D0899278836910549F18936910524F403
:10CD20008736910531F07BC08936910509F445C0FD
:10CD300076C080915A088093810880915B08809327
:10CD4000830880915C088093820880915D088093BD
:10CD5000840880915E088093850880915F088093A5
:10CD6000EE01809160088093010459C080915A08B7
:10CD70008093240880915B088093250880915C084B
:10CD80008093260880915D088093270880915E0833
:10CD9000809328088091C70590915F08892B809324
:10CDA000C705909160089093FF038091C805837038
:10CDB0009C70892B8093C80532C080915A0880935B
:10CDC0001A0880915B0880931B0880915C0880930F
:10CDD0001C0880915D0880931D0880915E089091E9
:10CDE0005F0890931F0880931E08809160089091BF
:10CDF0006108909321088093200880916208992708
:10CE000087FD909590937C0780937B0708C01092D4
:10CE1000FE031092FD031092FC031092FB031F917E
:10CE20000F91FF90EF90089580911908882309F4DD
:10CE30003BC045988AE298E09093230880932208AB
:10CE400090910004E92FFF27EC51FE4F9F5F9093D4
:10CE50000004808180932C08993010F01092000417
:10CE6000109219080E94B46381E0809329080000A1
:10CE700000000000000000000000000000000000B2
:10CE800000000000000000000000000000000000A2
:10CE90000000000000000000000000000000809181
:10CEA0002A08809349088EBD089587B18C6087B9A0
:10CEB000429843981092050480E88093F001109204
:10CEC00004048093EF01089580910A0481508093B7
:10CED0000A048F3F09F0FBC024E020930A048091EC
:10CEE000ED02992780739070892B21F4809148047A
:10CEF00080FF1CC080916C06882349F080910D044E
:10CF0000882311F42093050481E080930D0480911F
:10CF10006D068823B9F080910E04882319F484E00B
:10CF20008093040481E080930E040CC010920D04E1
:10CF300010920E048091680680930B0480916A061B
:10CF400080930C0480910D04882309F040C08091E7
:10CF50008206282F332724FF07C0809118038823D7
:10CF600019F425FD4DC04EC090916906983F50F0D0
:10CF70008091E0078D3D30F080910B0488230CF404
:10CF80003FC040C0983F48F08091E0078A3028F4C5
:10CF900080910B048823B4F133C080910504815043
:10CFA000809305048F3F79F58091E007815080934D
:10CFB00005048091F001813011F480E801C086956C
:10CFC0008093F0018091F00190910B0417C0809143
:10CFD00005048150809305048F3FA9F489E0809374
:10CFE00005048091F001813011F480E801C086953C
:10CFF0008093F0018091F00190916C06892311F0EB
:10D00000429A01C0429880910E04882309F043C0DF
:10D0100080918206282F332724FF07C080911803B0
:10D02000882319F426FD50C034C090916B06983FB8
:10D0300050F0809106088D3D30F080910C048823DB
:10D040000CF442C026C0983F48F0809106088A3010
:10D0500028F480910C048823E4F036C08091040405
:10D060008150809304048F3F91F580910608815090
:10D07000809304048091EF01813011F480E801C0B5
:10D0800086958093EF018091EF0190910C048923A4
:10D09000D9F4439808958091040481508093040446
:10D0A0008F3FA9F489E0809304048091EF018130DF
:10D0B00011F480E801C086958093EF018091EF0123
:10D0C00090916D06892311F0439A0895439808952D
:10D0D0004FB724E130E0F8948091C9008F778093B6
:10D0E000C9008091C9008F7B8093C9008091C900DD
:10D0F0008F7D8093C9005A9A52985B9A539A832FD6
:10D1000099278093CD002093CC008091C800826045
:10D110008093C80080E18093C9008091CA008F7716
:10D120008093CA008091CA008F7B8093CA0080914F
:10D13000CA008F7D8093CA008091CA008F7E809341
:10D14000CA008091CA00877F8093CA008091C9007D
:10D150008B7F8093C9008091CA0084608093CA004D
:10D160008091CA0082608093CA008091C80087FFC6
:10D1700003C08091CE00F9CF8091C9008068809370
:10D18000C9004FBF0895A0E0B0E0E9ECF8E60C94C8
:10D19000C678482F00E010E08091F101813061F401
:10D1A0001092F10184E48093110410921304109200
:10D1B00012041092140425C280911104882319F4DA
:10D1C00021E030E001C0980190911204992371F49C
:10D1D000232B11F081E010C084E48093110490931C
:10D1E00013049093120490931404F4C1913069F4E1
:10D1F000232B09F0E5C182E080931204809113048F
:10D200008F5F8093130483E0E3C19230D1F4232B2A
:10D2100009F0D6C183E080931104409314049091E7
:10D220001304923039F41092150447FF03C081E0D3
:10D230008093150483E0809312049F5F90931304FE
:10D24000C9C1933009F0BCC1232B09F0B9C1909337
:10D25000110482E080931204809113048F5F809305
:10D26000130420911404822F9927782F6627842F86
:10D270009927682B792B80914506813051F4737082
:10D28000CB018050924063E070E00E946C78EB012B
:10D2900019C0823069F47770CB018050944066E009
:10D2A00070E00E946C78EB012695269526950CC0BF
:10D2B000EB01D370C856D140CE01D7FD0196EC01E9
:10D2C000D595C79526952695022F11270F701070BA
:10D2D0000F5F1F4F0D30110508F06BC102301105B3
:10D2E00019F404E010E005C00430110511F402E067
:10D2F00010E06801C00ED11EF601E75BF84F808197
:10D3000091819E01281B390BC90137FF03C09095FD
:10D3100081959F4F069794F480912103883C30F4C7
:10D3200080912103865F8093210308C088EC80935D
:10D33000210380916F008F7D80936F00F601E75B82
:10D34000F84F808191819C01220F331F280F391FD4
:10D350002C0F3D1F37FF02C02D5F3F4F7901F59421
:10D36000E794F594E794CE0101968E159F0524F479
:10D370000894E108F10808C0CE010197E816F90603
:10D380001CF40894E11CF11C0630110509F0D1C011
:10D39000C536D1050CF4A8C090911004E92FFF27E1
:10D3A000EA57F74FE081ED3729F480910F0480951B
:10D3B00080930F04963061F480910F04882311F05C
:10D3C000E338B9F0882309F08BC0ED3791F088C0BD
:10D3D000993009F085C080910F04882329F4809149
:10D3E0008F08833831F07CC080918F088D3709F029
:10D3F00077C0809187088D3739F480918808833809
:10D40000B1F483E89FEF0FC0833889F480918808D6
:10D41000833829F4109254071092530708C08D37AF
:10D4200031F48DE790E090935407809353078091F7
:10D430008908992787FD9095909356078093550703
:10D4400080918A08992787FD909590936007809333
:10D450005F0780918B08992787FD909590936207CD
:10D4600080936107809110048930D1F580918D08F7
:10D470008D3749F48091590790915A0705969093FA
:10D480005A078093590780918E088D3749F480910F
:10D49000590790915A07059790935A078093590717
:10D4A0008091590790915A0783589F4F1CF483E845
:10D4B0009FEF09C08091590790915A078E379105C7
:10D4C00034F08DE790E090935A078093590780914C
:10D4D0008C08992787FD909590935E0780935D0750
:10D4E0001092100410920F04CA30D1055CF48091A0
:10D4F00010048F5F80931004E82FFF27EA57F74F3F
:10D5000083E88083809110048A3011F41092100413
:10D510008FEFCC39D8076CF480911004E82FFF27E7
:10D52000EA57F74F8DE7808380910F0480958093B1
:10D530000F0480912103843BD0F0F601E75BF84FA4
:10D5400080819181F701E81BF90BCF0163E070E066
:10D550000E946C78CB01880F991F860F971F2DE7CB
:10D5600037E0C20ED31EF6019183808307C02DE7FA
:10D5700037E0C20ED31EF60111821082053011056C
:10D5800040F4000F111F075B184FF801F182E08291
:10D5900021C00530110529F4D0935807C0935707CF
:10D5A00019C007301105B1F4D0935C07C0935B0735
:10D5B00011C00231110570F081E08093F1010AC0C1
:10D5C00081E08093F101109213041092150484E419
:10D5D0008093110480911304803198F08091150498
:10D5E000882331F48091F101882311F48093940110
:10D5F00010921304109215041092120484E4809384
:10D600001104E8E0CDB7DEB70C94E278CF93FC01CB
:10D6100097FF05C0CFEFF095E195FF4F01C0C1E046
:10D6200028E631E0CF01B9010E946C78FC018B350E
:10D63000910554F08B5590408A35910538F484EB70
:10D6400090E08E1B9F0BFC0141E00DC0CF01855B7C
:10D6500090408A35910518F4E45BF04003C02E1B1E
:10D660003F0BF9014FEFEE0FFF1FE15DF54F2591E5
:10D6700034918C2F992787FD9095289FB001299F81
:10D68000700D389F700D1124842F992787FD909578
:10D69000689FA001699F500D789F500D1124CA0109
:10D6A000CF9108952AE530E0281B390BC9010E946B
:10D6B000066B0895CF93DF9380E00E943D718091C7
:10D6C0001E0190911F016AE070E00E946C789F93A8
:10D6D0008F9380911E0190911F016AE070E00E947B
:10D6E0006C787F936F938DEF9AE09F938F93C0E355
:10D6F000D1E7DF93CF93E0912E04F0912F040995A9
:10D700002DB73EB7285F3F4F2DBF8091ED01882395
:10D71000B9F186E00E943D7180911E0890911F082A
:10D720006AE070E00E9458787F936F938FED90E0ED
:10D730009F938F9380910F0890911008A0911108EA
:10D74000B091120820919A0130919B0140919C0167
:10D7500050919D01BC01CD010E94A1783F932F9370
:10D7600086E09BE09F938F93DF93CF93E0912E040D
:10D77000F0912F0409958DB79EB70A968DBF12C000
:10D7800086E00E943D7182E19BE09F938F93DF933F
:10D79000CF93E0912E04F0912F0409950F900F90F4
:10D7A0000F900F908091FF038823C1F086E00E94C4
:10D7B0003D718091FF0399279F938F9389E19BE0AF
:10D7C0009F938F93DF93CF93E0912E04F0912F04DA
:10D7D00009952DB73EB72A5F3F4F2DBF80E10E94CC
:10D7E0003D718091F7019091F8016CE370E00E9427
:10D7F00058789F938F938091F7019091F8016CE393
:10D8000070E00E9458787F936F9380919508909173
:10D8100096089F938F9384E29BE09F938F93C0E33E
:10D82000D1E7DF93CF93E0912E04F0912F04099577
:10D8300080912B062DB73EB7265F3F4F2DBF80FF4F
:10D8400029C08AE10E943D718091990199279F9397
:10D850008F938091130390911403A0911503B091BD
:10D860001603BC01CD0124E630E040E050E00E9408
:10D87000A1783F932F9381E39BE09F938F93DF9356
:10D88000CF93E0912E04F0912F0409958DB79EB7A8
:10D8900008968DBFDF91CF910895CF93DF9380E0FD
:10D8A0000E943D7180910707992787FD90959F936E
:10D8B0008F938091FF06992787FD90959F938F9373
:10D8C0008091F706992787FD90959F938F9380917C
:10D8D000EF06992787FD90959F938F9388E39BE0B0
:10D8E0009F938F93C0E3D1E7DF93CF93E0912E0412
:10D8F000F0912F04099580E10E943D712DB73EB74C
:10D90000245F3F4F2DBF80912707992787FD909572
:10D910009F938F9380911F07992787FD90959F93E1
:10D920008F9380911707992787FD90959F938F93E9
:10D9300080910F07992787FD90959F938F9388E497
:10D940009BE09F938F93DF93CF93E0912E04F09110
:10D950002F04099580911D062DB73EB7245F3F4FD8
:10D960002DBF853098F480E10E943D7188E59BE0F1
:10D970009F938F93DF93CF93E0912E04F0912F0428
:10D9800009950F900F900F900F9018C08730B0F44A
:10D9900088E10E943D718FED90E09F938F9389E61F
:10D9A0009BE09F938F93DF93CF93E0912E04F091B0
:10D9B0002F0409958DB79EB706968DBFDF91CF9145
:10D9C00008950F931F9380E00E943D712AE030E09C
:10D9D0008091910890919208B9010E9458789F9384
:10D9E0008F938091910890919208B9010E94587884
:10D9F0007F936F9380911E0190911F01B9010E9446
:10DA00006C789F938F9380911E0190911F01B901B3
:10DA10000E946C787F936F9382E79BE09F938F9334
:10DA200000E311E71F930F93E0912E04F0912F0470
:10DA3000099580E10E943D718DB79EB70C968DBF10
:10DA400080919508909196089F938F938091930869
:10DA5000909194089F938F9385E89BE09F938F9379
:10DA60001F930F93E0912E04F0912F0409958DB729
:10DA70009EB708968DBF1F910F9108950F931F9326
:10DA8000CF93DF938091ED01C0E3D1E7882309F4C0
:10DA900078C080E00E943D7180911B0899279F9378
:10DAA0008F9380911D0899279F938F9381E99BE025
:10DAB0009F938F938E01DF93CF93E0912E04F0918B
:10DAC0002F0409958DB79EB708968DBF80911C08CD
:10DAD000833031F48CE00E943D7180EA9BE005C008
:10DAE0008CE00E943D7185EA9BE09F938F93DF93CA
:10DAF000CF93E0912E04F0912F0409950F900F9091
:10DB00000F900F9080911A0881FF12C08CE00E9444
:10DB10003D718AEA9BE09F938F931F930F93E0914F
:10DB20002E04F0912F0409950F900F900F900F90F5
:10DB300080E10E943D718FED90E09F938F938091E3
:10DB40002008909121089F938F9380911E089091B7
:10DB50001F086AE070E00E9458787F936F938FEA05
:10DB60009BE09F938F9380E391E79F938F93E09146
:10DB70002E04F0912F0409958DB79EB70A968DBF9C
:10DB800012C082E00E943D718FEB9BE09F938F93C8
:10DB9000DF93CF93E0912E04F0912F0409950F901D
:10DBA0000F900F900F90DF91CF911F910F910895DB
:10DBB000CF93C82F209116042093170499278F32F2
:10DBC000910509F1803391051CF44F97A1F02CC009
:10DBD0008F34910501F18F38910531F5222319F425
:10DBE00081E090E038C086E0289FF0011124EB51DD
:10DBF000F54F849117C086E0289FF0011124EA5167
:10DC0000F54F84910FC086E0289FF0011124E9515F
:10DC1000F54F849107C086E0289FF0011124E85158
:10DC2000F54F849180931604909116048091170407
:10DC30009813C0E00E9443719091160486E0989F6B
:10DC4000F0011124E751F54F259134918C2FF90102
:10DC5000099580E090E0CF9108951092920810927B
:10DC600091081092960810929508109294081092BC
:10DC70009308109297088AE090E00E941A179093F8
:10DC80001904809318040895CF93DF9380911804AA
:10DC9000909119040E942317882309F4AFC0809142
:10DCA0001804909119040A9690931904809318040B
:10DCB000E0E0F0E09F0190E05FEFA8EEB6E04BE01F
:10DCC000ED018B8187FF0BC09F5F8D81E80FF11DF8
:10DCD0008981280F311D8E81851708F4582F4150F6
:10DCE000189647FFEDCF50939708232B41F52091CD
:10DCF0001E0430911F044091200450912104BB2741
:10DD0000A52F942F832F90931D0480931C04AA2782
:10DD1000BB27281B390B4A0B5B0BCF01AA27BB275C
:10DD2000280F391F4A1F5B1F20931E0430931F04C6
:10DD30004093200450932104E5E0F0E013C02091CB
:10DD40001C0430911D042E173F0718F4E21BF30B3F
:10DD500002C0E0E0F0E0892F9927880F991FE80FB3
:10DD6000F91F3596F0939208E0939108EF3FF10583
:10DD700078F480911E0190911F018E9F90018F9FDA
:10DD8000300D9E9F300D1124C90164E670E013C070
:10DD9000CF01969587959695879520911E01309194
:10DDA0001F01289FA001299F500D389F500D11245D
:10DDB000CA0169E170E00E945878709394086093FA
:10DDC000930820911A0430911B042E0F3F1F3093AB
:10DDD0001B0420931A045EE02131350778F080910E
:10DDE00095089091960801969093960880939508CF
:10DDF00020513E4030931B0420931A04DF91CF91B1
:10DE00000895002422273327442751E0BB27EE271B
:10DE1000FF27A0E1660F771F881F991F001C221F94
:10DE2000331F441F660F771F881F991F001C221F76
:10DE3000331F441F2AF4050E2B1F3E1F4F1F04C023
:10DE4000051A2B0B3E0B4F0B550FBB1FEE1F587FB8
:10DE5000556047FD5250AA95E9F6E695B795579556
:10DE6000E695B7955795852F9B2F08952227332741
:10DE700041E0552768E0880F991F221F331F880F44
:10DE8000991F221F331F1AF4240F351F02C0241BB1
:10DE9000350B440F551F487F456037FD42506A954A
:10DEA00051F75695479556954795842F0895AA277B
:10DEB00097FF04C0809590958A1F9A1F77FF04C032
:10DEC000609570956A1F7A1F669F9001779FA001E9
:10DED000679F300D411D5A1F300D411D5A1F889FED
:10DEE000F001999F2E0F3F1F401D511D899F300D3E
:10DEF000411D5A1F300D411D5A1FCA01B90111247D
:10DF000080CF4FB720E430E0F8948091C9008F773C
:10DF10008093C9008091C9008F7B8093C900809154
:10DF2000C9008F7D8093C9005A9A52985B9A539A80
:10DF3000832F99278093CD002093CC008091C80037
:10DF400082608093C80088E18093C9008091CA00F4
:10DF50008F778093CA008091CA008F7B8093CA001C
:10DF60008091CA008F7D8093CA008091CA008F7E05
:10DF70008093CA008091CA00877F8093CA008091F5
:10DF8000C9008B7F8093C9008091CA008460809310
:10DF9000CA008091CA0082608093CA008091C80044
:10DFA00087FF03C08091CE00F9CF8091C9008068BF
:10DFB0008093C9004FBF08950F931F93CF93DF93B2
:10DFC000482F4F5F893108F08BC080914807841734
:10DFD00020F44F5F409348074150CB0183539B424D
:10DFE00068E170E00E946C78A42FBB27FD01EA0F66
:10DFF000FB1FE75BF84F808191819B01281B390B48
:10E00000C90137FF03C0909581959F4F069794F4FF
:10E0100080912103883C30F480912103865F8093B6
:10E02000210308C088EC8093210380916F008F7DCD
:10E0300080936F00FD01EA0FFB1FE75BF84F8081C3
:10E0400091819C01220F331F280F391F260F371F84
:10E0500037FF02C02D5F3F4FE901D595C795D59594
:10E06000C795CB0101968C179D0714F4219706C024
:10E0700061507040C617D7070CF421968091210398
:10E08000843BD8F08D010A0F1B1FF801E75BF84FA6
:10E0900080819181FE01E81BF90BCF0163E070E004
:10E0A0000E946C78CB01880F991F860F971F035829
:10E0B000184FF8019183808307C0AA0FBB1FA35894
:10E0C000B84F11961C921E92E42FFF27EE0FFF1FF0
:10E0D000E75BF84FD183C083443011F41092940170
:10E0E000DF91CF911F910F910895CF93DF932091EE
:10E0F0009808822F9927807F9070409709F06CC014
:10E100002F3109F046C08091990880932604209110
:10E110009B082093280480919C0880932704822FD9
:10E12000992790934A0780934907222309F054C006
:10E1300080911F06282F3327220F331FF901E35840
:10E14000F84F1182108280912006A82FBB27AA0FBA
:10E15000BB1FFD01E358F84F118210828091220607
:10E16000E82FFF27EE0FFF1FCF018358984FEC01D8
:10E1700019821882275B384FE90119821882A75B40
:10E18000B84F11961C921E92E75BF84F11821082D5
:10E1900023C0C22FCF70CA30F8F4809199088093C1
:10E1A000C20880919A088093C10880919B0880934F
:10E1B000C40880919C088093C3086091C108709145
:10E1C000C2088C2F0E94DC6F6091C3087091C40854
:10E1D0008C2F8F5F0E94DC6FDF91CF910895CF93DA
:10E1E000C82F8F3F49F4809129048F3F29F4109262
:10E1F0002B0410922A0432C020912B04222339F4DC
:10E20000CF3111F485E001C084E080932C0480912B
:10E210002C0490912A048217A0F4892F8095809372
:10E220002A048F3F19F48EEF80932A0480912A04E8
:10E23000C81711F40E94757010922B0410922A04D2
:10E240000BC0E22FFF27E856F74FC0832F5F2093C4
:10E250002B049C0F90932A04C0932904CF91089516
:10E2600090912504933240F4E92FFF27E256F74FAF
:10E2700080839F5F909325040895833218F48D5F07
:10E2800080932504089590E2E1EAF8E08FE191930C
:10E29000815087FFFCCF0895CF93CFB723E031E0C3
:10E2A000F8948091C9008F778093C9008091C9004C
:10E2B0008F7B8093C9008091C9008F7D8093C900B6
:10E2C0005A9A52985B9A539A832F99278093CD003C
:10E2D0002093CC008091C80082608093C80088E1C0
:10E2E0008093C9008091CA008F778093CA00809183
:10E2F000CA008F7B8093CA008091CA00806280939D
:10E30000CA008091CA0080618093CA008091CA00CF
:10E3100088608093CA008091C90084608093C9009E
:10E320008091CA0084608093CA008091CA00826094
:10E330008093CA008091C80087FF03C08091CE00FF
:10E34000F9CF8091C90080688093C9008091C9008D
:10E3500080648093C9000E944371CFBFCF9108951C
:10E36000282F99278F709070892B31F420958091F8
:10E370002404822B8093240408958091F40188233F
:10E3800009F441C08091ED0285FF0AC082E98093C3
:10E390009E0883E280939F0885E58093A00802C0D1
:10E3A00010929E088091F5018F3071F480912404C1
:10E3B0000E94D86D882341F081E980939E08809364
:10E3C0009F0881E38093A0081092F4018091C80017
:10E3D00085FFFCCF8091C9008F7E8093C90080911A
:10E3E000C9008E7F8093C90080919E08882311F414
:10E3F0008EEF01C08EE78093CE008091240480933D
:10E40000F5011092240408951F920F920FB60F92F7
:10E4100011248F939F93EF93FF939091F40199238D
:10E4200009F040C080912D04882361F480919E08FA
:10E43000882311F483E003C0813999F481E080934B
:10E440002D040FC0833099F480919E08882349F0F1
:10E4500090939E088091C9008E7F8093C9008EEFB3
:10E460001EC08091C90081608093C9000EC08332B4
:10E4700061F48091C9008E7F8093C9008FEF8093F3
:10E48000CE0081E08093F40114C080912D04E82F28
:10E49000FF27E256F74F8F5F80932D048081809392
:10E4A000CE0007C010922D048091C9008061809336
:10E4B000C900FF91EF919F918F910F900FBE0F9028
:10E4C0001F901895EF92FF920F931F93CF93DF93B6
:10E4D0007C018B01EA01452B39F0F80181918F0114
:10E4E000F70109952197C9F7E6E0CDB7DEB70C949F
:10E4F000E478EF92FF920F931F93CF93DF937C0109
:10E500008B01EA01452B41F0F8010F5F1F4F849109
:10E51000F70109952197C1F7E6E0CDB7DEB70C9476
:10E52000E4780F931F93CF938C01C62F161634F403
:10E5300080E2F8010995C1501C16D4F3CF911F91C8
:10E540000F9108950F931F93CF938C01C62F16162A
:10E5500034F480E3F8010995C1501C16D4F3CF912F
:10E560001F910F910895A5E3B0E0E9EBF2E70C9459
:10E57000BC782E96EEADFFAD2E97882499245401D9
:10E5800080912304882321F42C961FAE1EAE2C9775
:10E590005EE4452E512C4C0E5D1E6F01B60105C088
:10E5A000153239F00894C11CD11CF60114911123C5
:10E5B000B9F7A601461B570B31F02C968EAD9FADD7
:10E5C0002C970E947972112309F46AC20894C11C25
:10E5D000D11CFF24FDA6FCA64FEFE42EF9A6F60100
:10E5E0000894C11CD11C1491153721F0812F806231
:10E5F0008837B1F4F0FE0AC0F20124E030E0420EA8
:10E60000531E80809180A280B3800AC0F20142E054
:10E6100050E0440E551E808191814C01AA24BB24F8
:10E62000103221F489A58823D1F61DC0133219F4C4
:10E6300058E0F52AD4CF1A3211F01D3291F41A3273
:10E6400059F4F20182E090E0480E591EE081ECA7F7
:10E65000EE232CF6E195ECA790E1F92AAFEDFA2232
:10E66000BECF1B3211F419A7BACF1E32C1F5F60185
:10E670000894C11CD11C14911A3279F4F20122E0E1
:10E6800030E0420E531E408151813FEF4F3F530710
:10E6900014F44FEF5FEFE42EA2CF40E050E0812F63
:10E6A00080538A30A0F4CA0133E0880F991F3A954D
:10E6B000E1F7840F951F480F591F410F511D40531B
:10E6C0005040F6010894C11CD11C1491E8CF8FEF83
:10E6D0004F3F580714F44FEF5FEFE42E85CF103310
:10E6E00029F4F4FC7CCF90E2F92A79CF812F815371
:10E6F0008930D8F440E050E0CA0123E0880F991F28
:10E700002A95E1F7840F951F480F591F410F511D9E
:10E7100040535040F6010894C11CD11C1491812F24
:10E7200080538A3048F34CA75FCF183619F4A4E021
:10E73000FA2A55CF1C3619F4B1E0FB2A50CF133614
:10E7400061F43E010894611C711CF20122E030E08A
:10E75000420E531E808189833CC1143421F014364B
:10E7600011F0193651F5143411F431E0F32AF0FEAA
:10E770000AC0F20144E050E0440E551E80809180B2
:10E78000A280B3800CC0F20182E090E0480E591ED6
:10E79000808191814C01AA2497FCA094BA2CB7FEE9
:10E7A0000AC0B094A09490948094811C911CA11CE8
:10E7B000B11C8DE289A70AE06FC01F3411F01F362B
:10E7C00031F41F3411F491E0F92A08E064C01037E5
:10E7D00079F4F201A2E0B0E04A0E5B1E80819181E3
:10E7E0004C01AA24BB2400E1B0E4FB2A18E753C083
:10E7F0001337C1F5F20122E030E0420E531E608073
:10E8000071806114710489F43E010894611C711CCB
:10E8100088E289838EE6F301818385E78B838CE62A
:10E820008C838D8389E28E831F82E7FC13C08E2D3B
:10E83000992787FD9095AC0160E070E0C3010E94CC
:10E840006877009729F0382E3618E3140CF0C3C00F
:10E850003E2CC1C0F30101900020E9F731973E2E14
:10E860003618B9C0153511F0153731F4153511F4D6
:10E87000F1E0FF2A0AE00FC0183519F0183709F047
:10E88000A0C000E1F3FE07C081149104A104B1040B
:10E8900011F020E4F22A19A6EDA6E7FC02C03FED34
:10E8A000F32289E2682E712C6C0E7D1E8114910476
:10E8B000A104B10421F44DA5442309F47BC0802FA9
:10E8C0009927AA27BB278EA79FA7A8ABB9AB202E55
:10E8D000332490E0891690E0990691E0A90690E033
:10E8E000B90648F0C501B4012EA53FA548A959A90C
:10E8F0000E947F7817C0AFEF8A169104A104B1047B
:10E9000049F040F0C401B1010E9458789B014427AE
:10E91000552708C0882D602F0E944C78282F332758
:10E92000442755272AAB3BAB4CAB5DAB0A3059F4BF
:10E930008AA9880F880F880F9AA9990F890F382DF7
:10E94000381B832F10C0003139F48AA98295807F4B
:10E95000482D481B842F07C08AA9880F880F880F6D
:10E96000582D581B852F90E02EA53FA548A959A9E1
:10E9700082169306A406B50608F091E08AA89BA823
:10E98000ACA8BDA88A3010F4805D04C0895A18353F
:10E9900009F48F7DD3018E933D01992309F099CF1E
:10E9A000083041F4F3FE06C0803321F080E3FD011E
:10E9B00082933F01CE010196382E3618F8E23F0EC1
:10E9C0000BC0112309F46CC03E010894611C711C3A
:10E9D0001983B1E03B2E19A6032D2DA4231827FC83
:10E9E000222489A5882311F00F5F02C0F6FC0E5F78
:10E9F000020DEF2CFF24C70180739070892B49F41E
:10EA00008CA5801B682F2C968EAD9FAD2C970E94F5
:10EA1000917289A5882331F041E050E0BE01675D25
:10EA20007F4F0AC0E6FE0EC080E38AA71BA742E024
:10EA300050E0BE01665D7F4F2C968EAD9FAD2C974A
:10EA40000E946272C70180739070809749F48CA510
:10EA5000801B682F2C968EAD9FAD2C970E94A272C2
:10EA6000622D2C968EAD9FAD2C970E94A272832DA5
:10EA7000992787FD9095AC01B3012C968EAD9FAD83
:10EA80002C970E946272E4FE89CD2CA5201B2CA736
:10EA9000622F2C968EAD9FAD2C970E9491727ECDE9
:10EAA000E2E1CB5C0C94D8782FB740E0F894E0E03A
:10EAB000F0E081E2809357009491E2E0F0E08093EF
:10EAC00057003491E4E0F0E08093570084912FBF29
:10EAD0009E3199F4363941F4893011F441E00DC08A
:10EAE0008A3059F442E009C0373939F4863011F4DC
:10EAF00043E003C0853009F444E0842F992708954A
:10EB00009FB7F8948091C900877F8093C900809156
:10EB1000C9008F7E8093C9008091C9008F77809350
:10EB2000C9008091C9008F7B8093C9008091C90082
:10EB30008F7D8093C90052985A9A53985B9A9FBFD1
:10EB400008951F93CF93DF93182F80912304882378
:10EB500009F48DC08091F301181709F488C08091E1
:10EB60002204882321F40E9454758093220488EBA8
:10EB70009CE09F938F93C4EFD2E1DF93CF93E0911A
:10EB80002E04F0912F0409950F900F900F900F9085
:10EB9000812F99278230910501F1833091052CF462
:10EBA000009761F0019769F024C084309105D9F095
:10EBB00084309105ACF00597C9F01BC088EA9CE051
:10EBC00002C086E99CE09F938F93DF93CF93E091FF
:10EBD0002E04F0912F04099518C08DE79CE0F3CF27
:10EBE0008AE59CE0F0CF8CE49CE0EDCF84E49CE0EF
:10EBF000EACF85EC9CE09F938F93DF93CF93E091D6
:10EC00002E04F0912F04099510E00F900F900F90B3
:10EC10000F9080912204843011F0823099F40E9488
:10EC20008075812F8150833018F40E9468681DC060
:10EC3000143019F40E944C7118C01530B1F40E94C0
:10EC4000816F13C0112389F08BED9CE09F938F930C
:10EC500084EF92E19F938F93E0912E04F0912F0423
:10EC600009950F900F900F900F901093F301DF9183
:10EC7000CF911F9108950F931F9381E080932304F8
:10EC80004091F201E4EFFBE020E030E05FE48491AA
:10EC900099272F5F3F4F829FB001839F700D929FF6
:10ECA000700D112446275150319657FFF0CF4093F5
:10ECB000F201ECECFBE020E030E057E28491992790
:10ECC0002F5F3F4F829FB001839F700D929F700D09
:10ECD000112446275150319657FFF0CF4093F2014F
:10ECE00080912204882321F40E9454758093220489
:10ECF0008091F201833459F088E190E029E20FB667
:10ED0000F894A895809360000FBE2093600083EB79
:10ED100092E790932F0480932E0486EF9CE09F93BC
:10ED20008F9304EF12E11F930F93E0912E04F09163
:10ED30002F0409950F900F900F900F9081E690E0AF
:10ED40009F938F9382E590E09F938F931F921F92E2
:10ED5000809102016AE00E944C78892F99279F9345
:10ED60008F93809102010E944C7899279F938F93F3
:10ED70008CE19DE09F938F931F930F93E0912E045E
:10ED8000F0912F04099584EF9BE09F938F931F933D
:10ED90000F93E0912E04F0912F0409958CEC9BE0E9
:10EDA0009F938F931F930F93E0912E04F0912F0464
:10EDB00009958DB79EB746968DBF80E59DE09F93E0
:10EDC0008F931F930F93E0912E04F0912F040995D8
:10EDD00083EC8093810080916F00806280936F004C
:10EDE0000F900F900F900F901F910F9108958091A9
:10EDF0002304882361F08091F301843011F40E9490
:10EE0000BD718091F201833411F0109223040895B2
:10EE10001F920F920FB60F9211242F933F934F938F
:10EE20005F936F937F938F939F93AF93BF93EF9372
:10EE3000FF932091CE008091FE018823B1F02093B2
:10EE4000C6008091FE01823029F52F3F19F58FEF22
:10EE500094E3ACE0B0E0C297A109B109B7FFFBCFE2
:10EE6000809171048093CE0015C09091F301892F99
:10EE70008150833020F4822F0E94C3680BC09430ED
:10EE800021F4822F0E94B07105C0953019F4822FB1
:10EE90000E94EF70FF91EF91BF91AF919F918F9181
:10EEA0007F916F915F914F913F912F910F900FBE86
:10EEB0000F901F901895FB01DC0140FF05C002C0B8
:10EEC00005900D9205900D9242505040C8F708955C
:10EED000FC014150504030F001900616D1F73197B7
:10EEE000CF0108958827992708955058192E84D066
:10EEF00001D06AC0BA176207730784079507B1F19A
:10EF000088F40EF410940B2EBA2FA02D062E622F2B
:10EF1000202D072E732F302D082E842F402D092EE3
:10EF2000952F502DFF275523B9F0591B49F0573E17
:10EF300098F0469537952795A795F0405395C9F7D2
:10EF400076F0BA0F621F731F841F30F48795779590
:10EF50006795B795F040939517FA0F2E0895BF1B4C
:10EF6000BB27BA0B620B730B840BF6CFDEF670C0B7
:10EF700097FB4ED09F3738F0FEE9F91B982F872F6B
:10EF8000762F6B2F05C061C096958795779567950D
:10EF9000F150D0F73EF490958095709561957F4F34
:10EFA0008F4F9F4F0895E89403C097FB0EF4F3DF53
:10EFB000B62F672F782F892F9EE9002405C09A95D8
:10EFC000BB0F661F771F881F11249923A1F0882388
:10EFD000B2F79F3F59F0BB0F48F421F4002011F421
:10EFE00060FF04C06F5F7F4F8F4F9F4F881F9795C3
:10EFF000879597F9089529C0052E092607FA440F29
:10F00000551F5F3F79F0AA27A51708F051E04795F3
:10F01000880F991F9F3F31F0BB27B91708F091E087
:10F02000879508959F919F91112414C097FB880F95
:10F03000991F9F3F31F0BB27B91708F091E08795E2
:10F0400008959F919F91112405C0662777278827EF
:10F05000992708959FEF80EC0895629FD001739FD8
:10F06000F001829FE00DF11D649FE00DF11D929F64
:10F07000F00D839FF00D749FF00D659FF00D9927A3
:10F08000729FB00DE11DF91F639FB00DE11DF91FC7
:10F09000BD01CF0111240895991B79E004C0991F87
:10F0A000961708F0961B881F7A95C9F780950895E2
:10F0B000AA1BBB1B51E107C0AA1FBB1FA617B7079E
:10F0C00010F0A61BB70B881F991F5A95A9F78095BA
:10F0D0009095BC01CD01089597FB092E07260AD013
:10F0E00077FD04D0E5DF06D000201AF47095619515
:10F0F0007F4F0895F6F7909581959F4F0895A1E26F
:10F100001A2EAA1BBB1BFD010DC0AA1FBB1FEE1FA1
:10F11000FF1FA217B307E407F50720F0A21BB30BEC
:10F12000E40BF50B661F771F881F991F1A9469F768
:10F1300060957095809590959B01AC01BD01CF01C4
:10F14000089597FB092E05260ED057FD04D0D7DF72
:10F150000AD0001C38F450954095309521953F4FCA
:10F160004F4F5F4F0895F6F7909580957095619594
:10F170007F4F8F4F9F4F08952F923F924F925F92F4
:10F180006F927F928F929F92AF92BF92CF92DF92B7
:10F19000EF92FF920F931F93CF93DF93CDB7DEB71C
:10F1A000CA1BDB0B0FB6F894DEBF0FBECDBF0994B0
:10F1B0002A88398848885F846E847D848C849B8407
:10F1C000AA84B984C884DF80EE80FD800C811B8115
:10F1D000AA81B981CE0FD11D0FB6F894DEBF0FBE44
:10F1E000CDBFED010895EE0FFF1F0590F491E02DC6
:10F1F0000994F999FECFB2BDA1BDF89A119600B459
:10F200000895F7DF01921A94E1F70895F2DFE02DF7
:10F21000F0DFF02D0895F999FECFB2BDA1BD00BC7D
:10F2200011960FB6F894FA9AF99A0FBE0895F3DF83
:10F23000012CF1DF112408950190EDDF1A94E1F71C
:02F2400008952F
:10F242005E010A010164FF01FFFFC01FC01F01012F
:10F2520001737373FF03007D0000C409C4096400D5
:10F262001148656C6C6F20576F726C64000000006F
:10F27200000000000000000000000000000000008C
:10F28200000000000000000000000000000000007C
:10F29200000000000000000000000000000000006C
:10F2A200000000000000000000000000000000005C
:10F2B2000053706F727400004E6F726D616C0000CB
:10F2C200426567696E6E6572000051756164726FA6
:10F2D200000064000101000300200B050000ECFFA8
:10F2E20000020406070808080706040200FEFCFAEA
:10F2F200F9F8F8F8F9FAFCFE0002040607080864B7
:10F3020040415A4664640A02969696960840403AEC
:10F3120010FB30380190D0030090D00300F4017844
:10F3220000FF03640B0A0D0B0C0E0B0F10FA2001E9
:06F33200010170FF010F54
:00000001FF
